:020000040000FA
:200000000208540200800402003F00020008B92200000002008014000000000200801C00A2
:20002000000000020080244447532D31323136542020202020204C56332E30EB7002E72298
:2000400089828A831410E704F593E022F593E49322BB0002F722BB8000500989828A838BC1
:20006000931593F022BC000BBE0029EF8DF084FFADF022E4CCF875F008EF2FFFEE33FEEC9A
:2000800033FCEE9DEC984005FCEE9DFE0FD5F0E9E4CEFD22EDF8F5F0EE008420D21CFEADD5
:2000A000F075F008EF2FFFED33FD4007985006D5F0F222C398FD0FD5F0EA22A3F8E0C5F033
:2000C00025F0F0E582158270021583E0C838F0E822BB0006F709A7F01922BB8000500D8985
:2000E000828A838B931593F0E5F0A3F022E88FF0A4CC8BF0A42CFCE98EF0A42CFC8AF0ED79
:20010000A42CFCEA8EF0A4CDA8F08BF0A42DCC3825F0FDE98FF0A42CCD35F0FCEB8EF0A40D
:20012000FEA9F0EB8FF0A4CFC5F02ECD39FEE43CFCEAA42DCE35F0FDE43CFC22EB9FF5F0F0
:20014000EA9E42F0E99D42F0E89C45F022E8600FEFC333FFEE33FEED33FDEC33FCD8F122D5
:20016000BB0006E9F802000332BB8000500C89828A838B9315930200017B22ECF0A3EDF035
:20018000A3EEF0A3EFF022EB700C87F009E608B5F019DFF6801589828A831410E70FF59383
:2001A000E0F5F0A3E608B5F002DFF5806AF593E493F5F0A3E608B5F05EDFF4805ACB701311
:2001C00088828C838B9387F009E493A3B5F048DFF580441410E71F88848C858B9589828ACD
:2001E00083F593758620E0F5F0E493A3A3B5F024DFF4DEF2801E88848C858B9589828A83F8
:20020000F593758620E493F5F0E493A3A3B5F004DFF3DEF17586007FFFB5F0020F22400245
:200220007F012202000187809488F0EF60010E4E60F0ED60EE1410E7EECB701288828C8370
:20024000F59387F009E0A3B5F0CDDFF680C91410E71E88848C858B9589828A83F593758682
:2002600020E0F5F0E0A3A3B5F0AADFF5DEF380A488848C858B9589828A83F593758620E47F
:2002800093F5F0E0A3A3B5F08BDFF4DEF28085EB7008E709F608DFFA801B89828A831410E7
:2002A000E70AF593E0A3F608DFFA8009F593E493A3F608DFF9ECFAA9F0EDFB2288F0EF601A
:2002C000010E4E60F088F0ED60C51410E7E7CB700E88828C838B93E709F0A3DFFA80D614AF
:2002E00010E71C88848C858B9589828A83F593758620E0F0A3A3DFFADEF875860080B68875
:20030000848C858B9589828A83F593758620E493F0A3A3DFF9DEF77586008099C5F0F8A3AF
:20032000E028F0C5F0F8E582158270021583E038F022ECF608EDF608EEF608EFF62290008E
:200340007004E0F54090007005E0F541854082854183E020E7077E007F00C2D72289428A6E
:20036000435407F54512000539E02402F54450020545120003E0053AE53A7002053BE54050
:200380002544F540E541354530E604C2E6242DF5411200040090007004E540F090007005A2
:2003A000E541F0AE45AF44D2D72290007010E020E61EA3EDF0A3E9F0A3EAF0EC5407D2E6EA
:2003C00090007010F00538E53870020539D2D7227C007D00C2D72290007010E0A2E6B32247
:2003E00075F001800375F0041200040078407F06900070921200052190007090E5F0F02217
:2004000090007090E0540770F7221200046D90007008742DF0900070107508101200045861
:20042000E490007004F090007006F0742D90007005F090007007F0751D10751C10751E008B
:20044000751F2D75832D758200E4F0753800753900753A00753B0022E4A808F0A3D8FC22F2
:20046000120005171200040A120004AB22900004A175080A79707860120005287518C075CD
:2004800019A8751A00751B647510C07511A87512007513017514FF7515FF7516FF7517006E
:2004A00022000B78667788C0A800649000706AE0440CF0229000706AE054F3F02290007017
:2004C0006AE04401F0229000706AE054FEF0229000706AE04402F0229000706AE054FDF0A0
:2004E000229000706AE04440F0229000706AE054BFF02290007000E04410F0229000700045
:20050000E054EFF02290007000E04420F02290007000E05420F0229000700AF000000000F0
:2005200022E6F008A3DFFA2289A0E493A3F208B800030989A0D508F222A3E58330E6037569
:20054000832D22754300754200754100754000754508754400120003E5754308754200758E
:200560004108754000754508754400120003E51200040090000000750910750800750B00D7
:20058000750A0012000638400B9000706CE04408F0D2D722C2D7227543007542007541000E
:2005A000754000754508754400120003E5754308754200754108754000754508754400129A
:2005C0000003E51200040090000000750910750800750B00750A00120006384051754310DA
:2005E000754200754110754000754508754400120003E575431875420075411875400075D5
:200600004508754400120003E51200040090001000750910750800750B10750A00120006F2
:2006200038400B9000706CE04418F0D2D722C2D722E6F008A3DFFA22A90B89A0A80AE49397
:20064000F5F0A3E265F0701008B800030989A01200067D50E9C2D722D2D722A90B89A0A88D
:200660000AE0F5F0A3E265F0701008B800030989A01200067D50EAC2D722D2D722E50860BA
:200680000A14F50845097007D2D72215091508C2D7229000700B7418F09000700C7420F0A2
:2006A00075A06022120006927824E2E2B408157400F21200072912000721120007071200B4
:2006C000070E802E22120006927816E2E2703708E2E2B4013178281200079C5029120007F9
:2006E0003912000779120007411200078178177402F27800E2E2FC4480F208E2E2FD7918FC
:200700007A20120003AA22781AE4F208F222782680F7E2E2F5F0E3E3F2E5F0F30809DAF2BF
:20072000227A04781C792080E9790878027A0680E1E2E2F30809DAF922780879027A0680EF
:20074000F0780879227A0680E8E4F309F3227A08E480037A04E4F309DAFC22E0F3A309E013
:20076000F3227A04E0F3A309DAFA227A0280027A04E2E2F0A308DAF922900070607A068041
:20078000E3781879227A0A8089E0F5F0E2E265F0700708A3DAF3D2D722C2D7229000706605
:2007A0007A0480E59000200AE0FEA3E08E8375820075814F73220D0A205446333331465556
:2007C0003A333956463038302031364B2D626173656420426C616E6B20436865636B696E64
:2007E00067002E2E2E5B6661696C5D0A002E2E2E5B6F6B5D0A000D0A205446333331465581
:200800003A6465766963655B53535420333956463038305D000D0A20544633333146553A7F
:20082000536563746F722D62617365642832353620736563746F72732920466C61736820DD
:2008400045726173652028314D29002E2E2E5B6F6B5D2E0075C7AA75C755759D02787FE409
:20086000F6D8FD900000007F007E607D01E4F0A3DFFCDEFADDF875814F12000517D20D12DF
:200880000004B41200040A12001DD412001DF0120013EBEF7004020008A5020008B312006D
:2008A0001D36EF700EC20D120004AB1200000702000C7BD20D02008000300D040200800C16
:2008C000C0E0C0D075D00012001DACD0D0D0E0320D0A544633333146553A52657620257542
:2008E0000A54616966617465636820496E632E000D0A2849503D200025752E00257529003D
:200900000D0A284D41433D200025782E00257829000D0A54463333313A2054465450206475
:200920006F6E652E204A756D7020746F20307825782E0A000D0A436865636B204368656363
:200940006B53756D3D00307825782E2E2E4F4B21210D0A00307825782E2E2E4661696C218C
:20096000210D0A001B5B324A000D0A436865636B204D6167696320436F64652E2E2E004FE3
:200980004B2121004661696C212100496C6C6567616C206669726D77617265002E000D0A90
:2009A00020496E76616C6964206669726D776172652021000D0A20466C6173682065727204
:2009C0006F722021004387049000555574AAF090002AAA7455F09000555574A0F08F828EE5
:2009E000838D93E52EF05387FB229000262FEEF0A3EFF0E4784EF608F6D390002630E0944A
:200A0000009000262FE094005003010C7A90002620E0FF94094003010B36EF705E90002659
:200A20002FE0FEA3E0FFD39400EE94004031784EE6FC08E67B012448F974203CFA1200007A
:200A40003B643A601A90002630E024FFF09000262FE034FFF0784F06E61870C10680BEEF53
:200A60004E7003010C7A784B7601900026207401F0784F06E618704F06804C90002620E0A7
:200A8000784BF6784BE6C39409504E90002630E094009000262FE09400403E784E0806E60B
:200AA000188606700106147B012448F974203EFA1200003BFF784BE6062423F582E4342663
:200AC000F583759300EFF090002630E024FFF09000262FE034FFF080AA784BE6900026204D
:200AE000F0C394095003010C7A9000261A7426F0A37423F0120018D1EF64014E70069000A5
:200B00002620F022120018D1EF64044E7003010C2B7D027F01120018D59000261CEFF07D06
:200B2000067C007F037E00120018D990002614EEF0A3EFF0807E9000261DE0FFA3E0900043
:200B40002614CFF0A3EFF090002621E06066D390002630E094009000262FE09400405590F2
:200B600000261A7426F0A37421F0784E0806E6188606700106147B012448F974203EFA12DB
:200B800000003B90002622F090002630E024FFF09000262FE034FFF07D017C00E4FFFE12A4
:200BA0000018D912001541E490002621F09000261CE014F09000261A7420F0A37448F0A335
:200BC000E0FF784C760008A607D3784DE6940018E694004049D390002630E0940190002636
:200BE0002FE094004038784EE6FE08E6FF2401FDE43EFC120018D912001541784F74022635
:200C0000F618E436F618E6161870011690002630E024FEF09000262FE034FFF080AB784D53
:200C2000E69000261CF0E61846700890002620F00109F99000262FE07004A3E064017026D0
:200C4000784E0806E6188606700106147B012448F974203EFA1200003B90002621F0E49076
:200C600000262FF0A3F090002614E0FFA3E09000261DCFF0A3EFF00109F922900070FFE058
:200C8000784AF67E087FD0E6540FFD7C0012000E721200113C7E087FF0E4FDFC12000E72B0
:200CA000E4784AF6784AE6FDC39403501E7E087FF874042DF582E43420F583759300E0FD7D
:200CC0007C0012000E72784A0680D97E087FFC90002007E0FD7C0012000E727E097F00E458
:200CE000FDFC12000E72E4784AF6784AE6FDC39405501E7E097F0974122DF582E43420F5F8
:200D000083759300E0FD7C0012000E72784A0680D97E097F0D90002017E0FD7C0012000EE9
:200D2000727B017A2079181200033E90002608EEF0A3EFF0D39424EE940040E59000202621
:200D4000E0B4081FA3E0B4061A90002609E024F0F090002608E034FFF0120006C5784AA6D8
:200D60000780BE90002026E0B408B6A3E0B400B19000202AE0FFA3E090002608CFF0A3EFD3
:200D8000F090002034E0FCA3E0FDA3E0FEA3E0FF900020001200017BE4784AF6784AE6FF9F
:200DA0007C007B012420F9EC3420FA1200003BFE740C2FF582E43420F583759300EEF006B7
:200DC000E6B406D890002028E064456003010D219000202EE0543F6003010D2190002031E4
:200DE000E0B4010E120006A4E490002608F0A3F0805190002031E0B411499000203EE07091
:200E000004A3E06445701690002609E024E4F090002608E034FFF012000FDA802690002073
:200E20003EE064FC7004A3E064036003010D2190002609E024E4F090002608E034FFF012DA
:200E400000164D9000264DE07003010D2112001E169000200A741FF0A374FCF07E097F110D
:200E6000FD7C1F12000E72C2A9C2AF120007A4010D2190002638EEF0A3EFF0A3ECF0A3ED23
:200E8000F090002638E475F001120000BB85F082F583759300E4939000263DF07003010F09
:200EA000D9E064256003010FBA9000263C740AF090002638E475F001120000BB85F082F572
:200EC00083759300E49324DB7003010FBA800090002639E024FFF090002638E034FFF090F1
:200EE000002638E475F001120000BB85F082F583759300E4939000263DF0E0249D60142473
:200F0000EE601924FD6003010FBA9000263C7410F080099000263BE0FF010FD29000263E87
:200F2000740AF09000263AE07002A3E0605A9000263CE0FBFD7C009000263AE0FEA3E0FF2E
:200F400012000065AA059000263AE0FEA3E0FFEBFD7C00120000659000263AEEF0A3EFF0F0
:200F6000D3EA64809489EA40052457FF80032430FF9000263EE014F0244EF582E43426F540
:200F800083759300EFF0809B9000263EE0B40A047F30803E9000263EE0C3940A4003010E42
:200FA00081E0FF04F0744E2FF582E43426F583759300E0FF12001E2880DA9000263DE0FF54
:200FC00012001E289000263DE0640A6003010E817F0D12001E28010E812290002044E0FE1D
:200FE000A3E0FFEE600301113BEF24FD606404600301113B12001C509000203CE0FFA3E07D
:2010000090002643CFF0A3EFF09000203EE0FEA3E0FF90002641EEF0A3EFF090002044E419
:20102000F0A37404F0E4A3F0A3F09000203CEEF0A3EFF090002643E0FFA3E09000203ECF47
:20104000F0A3EFF090002608E4F0A37404F0020012949000203EE0FEA3E0FF90002641E0B4
:201060006E7003A3E06F60030111339000263FE0FEA3E0FF90002046E0B50608A3E0B507C8
:201080000301112F90002640E02401FF9000263FE03400FE90002046E06E7003A3E06F6002
:2010A000030111339000203CE0FFA3E090002643CFF0A3EFF07E097F9CE4FDFC12000E724F
:2010C000C390002609E09404FF90002608E09400FE120009EA9000262EE0702B90002617B6
:2010E000E0C3941450067E097F9E80047E097FB4E4FDFC12000E727F047E0012001BE4905C
:2011000000264D7401F02290002640E004F070079000263FE004F0C390002609E094049041
:20112000002608E0940250079000264D7401F002001D72E490002608F0A3F022D2A9D2AF78
:20114000E49000262FF0A3F09000262FE0FEA3E0FFC39402EE9400505BEF2404FFE43EFE42
:2011600012001A7D90002631EEF0A3EFF0E0FD90002630E025E0FB9000262FE033FA740472
:201180002BF58274203AF583759300EDF090002631E0FF74052BF58274203AF58375930053
:2011A000EFF090002630E004F0709D9000262FE004F08094E49000262FF0A3F09000262F8B
:2011C000E0FEA3E0FFC39403EE9400505412001A7D90002631EEF0A3EFF0E0FD900026307C
:2011E000E025E0FB9000262FE033FA74122BF58274203AF583759300EDF090002631E0FF04
:2012000074132BF58274203AF583759300EFF090002630E004F070A49000262FE004F08071
:201220009BE4784BF6784BE6FF2404F582E43420F583759300E0FEEF2466FDE434708D828C
:20124000F583759300EEF006E6B404D9E4784BF6784BE6FF2412F582E43420F58375930009
:20126000E0FEEF2460FDE434708D82F583759300EEF006E6B406D99000706CE054FDF0908F
:20128000007001743FF0900070007410F0900070DAE4F02290002609E02408FE900026086F
:2012A000E0340090002040F0A3CEF0E4A3F0A3F090002000E0FCA3E0FDA3E0FEA3E0FF9030
:2012C0000020381200017B90002004E0FCA3E0FDA3E0FEA3E0FF900020341200017B900013
:2012E0002609E0241CF090002608E03400F0900020287445F0E4A3F09000202E7440F0E48F
:20130000A3F0A37410F0A304F090002608E0FFA3E09000202ACFF0A3EFF090002009E004B4
:20132000F0700790002008E004F090002008E09000202CF090002009E09000202DF0E4907C
:20134000002032F0A3F0900020187490F090002609E02412F090002608E03400F0C3A3E02F
:20136000944090002608E094005006E4F0A37440F090002018E054F8FE90002608E04EFF19
:20138000A3E090002018CFF0A3EFF0E4FF740C2FF582E43420F583759300E0FEEF7C007B3C
:2013A00001241AF9EC3420FAEE120000510FEFB406DBE4FF74122FF582E43420F583759310
:2013C00000E0FE74202FF582E43420F583759300EEF00FEFB406DD900020267408F0A3E401
:2013E000F07B017A207918020003AAE4FFFEFDFC9000262F1200017BE490002633F07E0916
:201400007F64FDFC12000E727E097F69E4FDFC12000E727FFC7EFF7D0F7C00900026341284
:2014200000017B9000262FE0F8A3E0F9A3E0FAA3E0FBC000C001C002C003A3E0FFE4FDFE95
:20144000A3A3E0F9A3E0FAA3E02FFFEE3AFEED39FDE42FFFE43EFEED3481FDA907AA06AB1A
:20146000051200003BFFD003D002D001D000EB4FFFEAFEE9FDE8FC9000262F1200017B90E7
:2014800000262FE0FCA3E0FDA3E0FEA3E0FF78081200014D9000262F1200017B900026335C
:2014A000E004F0E0C3940350030114239000262FE0F8A3E0F9A3E0FAA3E0FBC000C001C01E
:2014C00002C003A3E0FFE4FDFEA3A3E0F9A3E0FAA3E02FFFEE3AFEED39FDE42FFFE43EFE1E
:2014E000ED3481FDA907AA06AB051200003BFFD003D002D001D000EB4FFFEAFEE9FDE8FCC0
:201500009000262F1200017B7F557EAA7D557CAA9000262FE0F8A3E0F9A3E0FAA3E0FBC36D
:201520001200013C700D7E097F7FFDFC12000E727F01227E097F84E4FDFC12000E727F00B5
:201540002290002618EEF0A3EFF090002614E475F001120000BBAFF090002631F0A3EFF062
:2015600090002619E0FF9000262CF090002046E07004A3E0640160030115FC90002631E07D
:20158000FCA3E0FDC39427EC9400403CD3ED943AEC9400503390002617E004F08D828C8305
:2015A000759300E4936F6006E49000262DF090002617E0B414129000262DE07004A3F0804F
:2015C000079000262E7401F090002616E0702DA3E0641470279000262EE06020E4F52F1282
:2015E0000005971200173912001810EF70069000262EF022900026167401F022900026311E
:20160000E0FEA3E04E7002052F9000262EE06401703A90002616E0640170319000262CE02E
:20162000FDF46028E52F7011C3EE9440401E90002631E0FEA3E0FF800F90002631E0FEA37B
:20164000E0FF9000262CE0FD12001B76227FE07E5A7D947C0190002054E0F8A3E0F9A3E087
:20166000FAA3E0FBC31200013C600301173890002046E0FEA3E0FF64014E6007EF4E60031D
:20168000011738E490002052F0A3F090002050E0FEA3E0FFEE6003011738EF24FB600B24F3
:2016A000FB600924096003011738802D78127C207D017B017A2079487E007F06120002297E
:2016C000EF707590002608E4F0A37428F090002050E4F0A3740BF0800E12001CA390002080
:2016E00050E4F0A3740CF078487C207D017B017A2079127E007F06120002BC90002044E48D
:20170000F0A37402F0A3E4F0A304F09000204EE4F0A304F09000203EE0FEA3E0FF9000205B
:201720003CE0FDA3E0A3CDF0A3EDF09000203CEEF0A3EFF012001294227E077FF6E4FDFC30
:2017400012000E727E087F15E4FDFC12000E72E4F52FF523752408AE23AF24E4FCFDFB7AB7
:2017600010F9F8120000ED8F288E278D268C25A2AFE433F522C2AF4387049000555574AA83
:20178000F090002AAA7455F0900055557480F074AAF090002AAA7455F0E47FFF7EFFFDFC1B
:2017A000AB28AA27A926A825D31200013C401BE42528FFE43527FEE5263401FDA907AA0661
:2017C000AB05743012000051800C8528828527837593007430F05387FBE52224FF92AFAEDE
:2017E00023AF24E4FCFDFB7A10F9F8120000ED120019FB0524E52470020523C3E52394014F
:2018000050030117577E087F4BE4FDFC02000E727E077FB6E4FDFC12000E72E4752502F5B9
:2018200024F523F522E47F3FFEFDFCAB25AA24A923A822D31200013C40030118C3E4F52648
:20184000F527E4FF7E40FDFCAB25AA24A923A822120000ED8F2B8E2A8D298C28E4FCFDE501
:201860002B2527F52BE52A3526F52AED3529F529EC3528F528E4252BFFE4352AFEE52934C3
:2018800081FDA907AA06AB051200003BF4600D7E077FE2E4FD12000E727F00220527E527DA
:2018A00070020526C3E52694404097E5252401F525E43524F524E43523F523E43522F522CD
:2018C0000118257E077FEDE4FDFC12000E727F01227D087F077C007E0090002631ECF0A35D
:2018E000EDF0E4A3F0A3F0AD07AC06C390002632E09D90002631E09C40629000261AE0FEC0
:20190000A3E08E837593002DF582E5833CF583759300E0F990002634E0C4F8540FC868F081
:2019200090002633E0C454F048F0E9D39439500BE9C39430FFE49400FE8013C3E99441FFC2
:20194000E49400CF240ACF3400FE90002633E04EF0A3E04FF00DBD00010C808F9000263379
:20196000E0FEA3E0FF2290002635EEF0A3EFF09000265C7408F0F5C84402F0F5C87F327E3D
:201980000012001E159000265CE04404F0F5C87F647E0012001E1512001E079000265A74BA
:2019A00008F0A3E4F09000265AE0FCA3E0FD4C6043A3E054FAF090002635E0FEA3E0FFEC65
:2019C0005EFEED5F4E60089000265CE04404F09000265CE012001E0F12001E119000265CFB
:2019E000E04401F0F5C89000265AE0C313F0A3E013F080B19000265CE0FF22900026361297
:201A000000017B752901E4F52CF52D90002636A3E0FDA3E0FEA3E02400FFE43EFEED34812F
:201A2000FDA907AA06AB051200003BF52A532A40E529604090002636A3E0FDA3E0FEA3E052
:201A40002400FFE43EFEED3481FDA907AA06AB051200003BF52B532B40E52AB52B03E4F59E
:201A600029852B2A052DE52D7002052CB4FFC1E52CB4FFBCE5297F0060027F0122C2AFEE98
:201A80004408FE120019669000265CEFF0E490002633F0A3F09000265A7480F0A3E4F0902F
:201AA00000265AE07002A3E060379000265CE054FA12001E0E12001E07AFC8EF30E3149068
:201AC00000265AE0FEA3E0FF90002633E04EF0A3E04FF09000265AE0C313F0A3E013F080A1
:201AE000BE9000265CE054F8F0F5C87F907E0112001E15D2AF90002633E0FEA3E0FF2290EE
:201B000000262FEBF0A3EAF0A3E9F0E490002637F0A3F09000263574FFF5F0120000BB45F3
:201B2000F0604690002632E0FBA3E0FAA3E0F91200003BFF9000262FE0FBA3E0FAA3E0F94E
:201B400090002637E475F001120000BBFCE925F0F9EA3CFAEF1200005160B890002633E437
:201B600075F0011200031C80AA9000262FE0FBA3E0FAA3E0F92290002633EEF0A3EFF0A3DD
:201B8000EDF0AF2FE4FCFDFEFBFA7901F8120000ED8F268E258D248C2390002633E0FEA317
:201BA000E0FFE4FCFDE5262FF526E5253EF525ED3524F524EC3523F523A3E0F52EA2AFE41C
:201BC00033F522C2AFAF26AE25AD24AC23120009C5AF26AE25AD24AC23120019FBE5222489
:201BE000FF92AF22900070007429F090002044E4F0A37405F0A3EEF0A3EFF064044E7020D9
:201C0000900026327481F0A37409F0A3748BF0A3E4F0A37411F07B017A20794812001AFFC4
:201C200090002641E0FFA3E09000203CCFF0A3EFF090002643E0FFA3E09000203ECFF0A373
:201C4000EFF090002608E4F0A37415F002001294E49000263FF0A3F090002000E0FCA3E0E4
:201C6000FDA3E0FEA3E0FF900026451200017BE490002641F0A3F0A3F0A3F09000264DF064
:201C80009000262EF090002617F090002616F09000262D04F0900070007421F0900070DAC1
:201CA000E4F0227B017A20796CE475F004120000D1740229F9E43AFAE475F008120000D11F
:201CC000740229F9E43AFA90002004E0FCA3E0FDA3E0FEA3E0FF12000160740429F9E43A16
:201CE000FEC3E99444FFEE942090002608F0A3EFF0229000262FEEF0A3EFF0E4F523D3ED6E
:201D00009400EC9400402C9000262FE0FEA3E0AA06F97B811200003B2523F523ED1D700130
:201D20001C90002630E004F070D49000262FE004F080CBAF23227E097F34E4FDFC12000E5A
:201D400072E4F522FD7C80FF7E8012001CF28F22E522B4FF0E7E097F46FD7C0012000E7230
:201D60007F01227E097F54AD227C0012000E727F002290002044E4F0A37404F0900026411F
:201D8000E0FFA3E09000203CCFF0A3EFF090002643E0FFA3E09000203ECFF0A3EFF090009A
:201DA0002608E4F0A37404F002001294C0D0C2A9C2AFE5492401F549E43548F548E4354773
:201DC000F547E43546F546758C5D758A3DD2AFD2A9D0D022E58954F04401F589758C5D758D
:201DE0008A3DE4F549F548F547F546D2B9D28C227598504387805389CF438920758DF37593
:201E00008CF3D28ED299229000265CE04401F0F5C87FF47E01229000706CE054E7F022AF16
:201E200049AE48AD47AC46223099FDC2998F9922FFFFFFFFFFFFFFFFFFFFFFFFFFFFFFFF00
:201E4000FFFFFFFFFFFFFFFFFFFFFFFFFFFFFFFFFFFFFFFFFFFFFFFFFFFFFFFFFFFFFFFFA2
:201E6000FFFFFFFFFFFFFFFFFFFFFFFFFFFFFFFFFFFFFFFFFFFFFFFFFFFFFFFFFFFFFFFF82
:201E8000FFFFFFFFFFFFFFFFFFFFFFFFFFFFFFFFFFFFFFFFFFFFFFFFFFFFFFFFFFFFFFFF62
:201EA000FFFFFFFFFFFFFFFFFFFFFFFFFFFFFFFFFFFFFFFFFFFFFFFFFFFFFFFFFFFFFFFF42
:201EC000FFFFFFFFFFFFFFFFFFFFFFFFFFFFFFFFFFFFFFFFFFFFFFFFFFFFFFFFFFFFFFFF22
:201EE000FFFFFFFFFFFFFFFFFFFFFFFFFFFFFFFFFFFFFFFFFFFFFFFFFFFFFFFFFFFFFFFF02
:201F0000FFFFFFFFFFFFFFFFFFFFFFFFFFFFFFFFFFFFFFFFFFFFFFFFFFFFFFFFFFFFFFFFE1
:201F2000FFFFFFFFFFFFFFFFFFFFFFFFFFFFFFFFFFFFFFFFFFFFFFFFFFFFFFFFFFFFFFFFC1
:201F4000FFFFFFFFFFFFFFFFFFFFFFFFFFFFFFFFFFFFFFFFFFFFFFFFFFFFFFFFFFFFFFFFA1
:201F6000FFFFFFFFFFFFFFFFFFFFFFFFFFFFFFFFFFFFFFFFFFFFFFFFFFFFFFFFFFFFFFFF81
:201F8000FFFFFFFFFFFFFFFFFFFFFFFFFFFFFFFFFFFFFFFFFFFFFFFFFFFFFFFFFFFFFFFF61
:201FA00075C7AA75C755759D02787FE4F6D8FD900000007F007E607D01E4F0A3DFFCDEFA5B
:201FC000DDF875814F12000517C20D120004B41200040A12001DD412001DF0C20D120004F9
:201FE000AB02000C7BFFFFFFFFFFFFFFFFFFFFFFFFFFFFFFFFFFFFFFFFFFFFFF0200085466
:20200000020020C0C5F0F8A3E028F0C5F0F8E582158270021583E038F022EB9FF5F0EA9EC0
:2020200042F0E99D42F0E89C45F022E8600FECC313FCED13FDEE13FEEF13FFD8F122E86096
:202040000FEFC333FFEE33FEED33FDEC33FCD8F122BB0006E9F8020020B4BB8000500C89B3
:20206000828A838B9315930200206C22ECF0A3EDF0A3EEF0A3EFF022D093D083D082E4935B
:202080007012740193700DA3A393F8740193F5828883E4737402936C70127403936D700C9D
:2020A0007404936E70067405936F60DDA3A3A3A3A3A380CAECF608EDF608EEF608EFF62295
:2020C00002002FF6E490002005F0A3F0E0FF12003492E490002004F090002004E0FF04F0F7
:2020E000EFC3940A5069E47F807E80FDFC9000200F1200206C90002006E0FFC00790002094
:202100000FE0FCA3E0FDA3E0FEA3E0FF900020161200206CD0077D147C00120032D790005E
:202120002006E0FF7B017A20790F7D147C00120033E5E47F807E80FDFC9000200FE0F8A3B1
:20214000E0F9A3E0FAA3E0FBC31200201A708990002004E0B40A0280FEE47F81FEFDFC9066
:2021600000200F1200206C90002006E0FFC0079000200FE0FCA3E0FDA3E0FEA3E0FF900088
:2021800020161200206CD0077D177C00120032D7E4FF7E04FDFC9000200F1200206C90001E
:2021A0002006E0FFC0079000200FE0FCA3E0FDA3E0FEA3E0FF900020161200206CD0077D7D
:2021C000187C00120032D7E490002004F090002004E0FF245AF582E43420F583759300E0A8
:2021E000FE74092FF582E43420F583759300EEF090002004E004F0E0B406D2E4900020049C
:20220000F090002004E0FBC39403506DE0FD25E02409F582E43420F583759300E0FEED25FA
:20222000E0240AF582E43420F583759300E0FDEDFFE4FCFD9000200F1200206C90002006A8
:20224000E0FFC007EB2419FDE433FCC004C0059000200FE0FCA3E0FDA3E0FEA3E0FF900069
:2022600020161200206CD005D004D007120032D790002004E004F08088E47F747E88FDFC89
:202280009000200F1200206C90002006E0FFC0079000200FE0FCA3E0FDA3E0FEA3E0FF90D7
:2022A0000020161200206CD0077D1C7C00120032D7E47F807E19FDFC9000200F1200206C73
:2022C00090002006E0FFC0079000200FE0FCA3E0FDA3E0FEA3E0FF900020161200206CD050
:2022E000077D1D7C00120032D7E47F2C7E01FDFC9000200F1200206C90002006E0FFC007E6
:202300009000200FE0FCA3E0FDA3E0FEA3E0FF900020161200206CD0077D1E7C0012003209
:20232000D7E4FFFEFDFC9000200F1200206C90002006E0FFC0079000200FE0FCA3E0FDA375
:20234000E0FEA3E0FF900020161200206CD0077D267C00120032D7E47FFF7EFFFDFC900040
:20236000200F1200206CE490002004F090002004E0FEC39424503D90002006E0FFC007EE24
:202380002427FDE433FCC004C0059000200FE0FCA3E0FDA3E0FEA3E0FF9000201612002043
:2023A0006CD005D004D007120032D790002004E004F080B8E47FFFFEFDFC9000200F12002C
:2023C000206C90002006E0FFC0079000200FE0FCA3E0FDA3E0FEA3E0FF90002016120020FF
:2023E0006CD0077D4B7C00120032D7E47FFF7EFFFDFC9000200F1200206C90002006E0FF71
:20240000C0079000200FE0FCA3E0FDA3E0FEA3E0FF900020161200206CD0077D4C7C001245
:202420000032D7E47FFF7E01FDFC9000200F1200206C90002006E0FFC0079000200FE0FC65
:20244000A3E0FDA3E0FEA3E0FF900020161200206CD0077D4D7C00120032D7E47FFF7EFF7E
:20246000FDFC9000200F1200206C90002006E0FFC0079000200FE0FCA3E0FDA3E0FEA3E08B
:20248000FF900020161200206CD0077D4E7C00120032D7E47FA07EC0FDFC9000200F120095
:2024A000206C90002006E0FFC0079000200FE0FCA3E0FDA3E0FEA3E0FF900020161200201E
:2024C0006CD0077D687C00120032D7E47F417EFAFDFC9000200F1200206CE490002004F043
:2024E00090002004E0FEC39402503D90002006E0FFC007EE2469FDE433FCC004C005900064
:20250000200FE0FCA3E0FDA3E0FEA3E0FF900020161200206CD005D004D007120032D7909E
:20252000002004E004F080B8E47F417EFAFDFC9000200F1200206CE490002004F0900020C1
:2025400004E0FEC39402503D90002006E0FFC007EE246BFDE433FCC004C0059000200FE0A2
:20256000FCA3E0FDA3E0FEA3E0FF900020161200206CD005D004D007120032D79000200429
:20258000E004F080B8E47F107E20FDFC9000200F1200206C90002006E0FFC0079000200FAD
:2025A000E0FCA3E0FDA3E0FEA3E0FF900020161200206CD0077D6D7C00120032D7E47F0499
:2025C0007E08FDFC9000200F1200206C90002006E0FFC0079000200FE0FCA3E0FDA3E0FE27
:2025E000A3E0FF900020161200206CD0077D6E7C00120032D7E47F107E20FDFC9000200FD3
:202600001200206C90002006E0FFC0079000200FE0FCA3E0FDA3E0FEA3E0FF9000201612CA
:2026200000206CD0077D6F7C00120032D7E47F047E08FDFC9000200F1200206C90002006BB
:20264000E0FFC0079000200FE0FCA3E0FDA3E0FEA3E0FF900020161200206CD0077D707C12
:2026600000120032D7E490002004F090002004E0FBC39404400301271DE47FFF7E01FDFC6B
:202680009000200F1200206CEB75F002A42471FDE435F0FCC004C00590002006E0FFC0076B
:2026A0009000200FE0FCA3E0FDA3E0FEA3E0FF900020161200206CD007D005D004120032D4
:2026C000D7E47FFF7EFFFDFC9000200F1200206C90002004E075F002A42471FFE435F0CFE3
:2026E0002401FDE43FFCC004C00590002006E0FFC0079000200FE0FCA3E0FDA3E0FEA3E095
:20270000FF900020161200206CD007D005D004120032D790002004E004F001266BE47F0836
:202720007E08FDFC9000200F1200206C90002006E0FFC0079000200FE0FCA3E0FDA3E0FEC5
:20274000A3E0FF900020161200206CD0077D797C00120032D7E47F1E7E14FDFC9000200F64
:202760001200206C90002006E0FFC0079000200FE0FCA3E0FDA3E0FEA3E0FF900020161269
:2027800000206CD0077D7A7C00120032D7E4FFFEFDFC9000200F1200206C90002006E0FF7C
:2027A000C0079000200FE0FCA3E0FDA3E0FEA3E0FF900020161200206CD0077D7B7C001273
:2027C0000032D7E47F207E40FDFC9000200F1200206C90002006E0FFC0079000200FE0FC62
:2027E000A3E0FDA3E0FEA3E0FF900020161200206CD0077D817C00120032D7E47F507EFA5B
:20280000FDFC9000200F1200206C90002006E0FFC0079000200FE0FCA3E0FDA3E0FEA3E0E7
:20282000FF900020161200206CD0077D827C00120032D7E4FF7E40FDFC9000200F1200203D
:202840006C90002006E0FFC0079000200FE0FCA3E0FDA3E0FEA3E0FF900020161200206C2E
:20286000D0077D8C7C00120032D7E47F11FEFDFC9000200F1200206C90002006E0FFC007BD
:202880009000200FE0FCA3E0FDA3E0FEA3E0FF900020161200206CD0077D957C001200320D
:2028A000D7E47F337E22FDFC9000200F1200206C90002006E0FFC0079000200FE0FCA3E03B
:2028C000FDA3E0FEA3E0FF900020161200206CD0077D967C00120032D7E47F557E44FDFCA0
:2028E0009000200F1200206C90002006E0FFC0079000200FE0FCA3E0FDA3E0FEA3E0FF9071
:202900000020161200206CD0077D977C00120032D7E490002007F0A3F090002007E0FAA30F
:20292000E0FBC39419EA648094804003012BF9E47F837E04FDFC9000200F1200206C9000B4
:202940002006E0FFC007EBAE027803C333CE33CED8F92400FDEE3401FCC004C00590002086
:202960000FE0FCA3E0FDA3E0FEA3E0FF900020161200206CD005D004D007120032D790005A
:202980002007E0FAA3E0FB64184A6003012A547F817E16FDFC9000200F1200206C90002076
:2029A00006E0FFC007EBAE027803C333CE33CED8F92402FDEE3401FCC004C0059000200F35
:2029C000E0FCA3E0FDA3E0FEA3E0FF900020161200206CD005D004D007120032D7E47F80B6
:2029E0007E36FDFC9000200F1200206C90002006E0FFC007A3E0FEA3E07803C333CE33CE2D
:202A0000D8F92401FDEE3401FCC004C0059000200FE0FCA3E0FDA3E0FEA3E0FF9000201637
:202A20001200206CD005D004D007120032D7E4FFFEFDFC9000200F1200206C90002006E090
:202A4000FFC007A3E0FEA3E07803C333CE33CED8F9012B1AE47FF17E17FDFC9000200F12A2
:202A600000206C90002006E0FFC007A3E0FEA3E07803C333CE33CED8F92402FDEE3401FC17
:202A8000C004C0059000200FE0FCA3E0FDA3E0FEA3E0FF900020161200206CD005D004D0B2
:202AA00007120032D7E47F807ED6FDFC9000200F1200206C90002006E0FFC007A3E0FEA3E7
:202AC000E07803C333CE33CED8F92401FDEE3401FCC004C0059000200FE0FCA3E0FDA3E09D
:202AE000FEA3E0FF900020161200206CD005D004D007120032D7E47F01FEFDFC9000200F3D
:202B00001200206C90002006E0FFC007A3E0FEA3E07803C333CE33CED8F92403FDEE34015F
:202B2000FCC004C0059000200FE0FCA3E0FDA3E0FEA3E0FF900020161200206CD005D004E5
:202B4000D007120032D7E4FFFEFDFC9000200F1200206C90002006E0FFC007A3E0FEA3E0EC
:202B60007803C333CE33CED8F92404FDEE3401FCC004C0059000200FE0FCA3E0FDA3E0FEDB
:202B8000A3E0FF900020161200206CD005D004D007120032D7E47F017E10FDFC9000200F0A
:202BA0001200206C90002006E0FFC007A3E0FEA3E07803C333CE33CED8F92405FDEE3401BD
:202BC000FCC004C0059000200FE0FCA3E0FDA3E0FEA3E0FF900020161200206CD005D00445
:202BE000D007120032D790002008E004F0700790002007E004F0012919229000201EEFF043
:202C00007B017A2079427D107C0012002EEB90002042A3A3A3E05480FFEF60037F0022909E
:202C200000201FA3A3A3E05407FFE4FEFDFC120020782C91000000012C420000000500007C
:202C40002C8E9000204EE0FCA3E0FDA3E0FEA3E0FF9000202D1200206C9000201EE0FF7DB8
:202C6000037C001200339E9000204AE0FCA3E0FDA3E0FEA3E0FF9000202D1200206C90008E
:202C8000201EE0FF7D027C001200339E80037F002290002023E0FCA3E0FDA3E0FEA3E0FFE3
:202CA0009000202D1200206C9000201EE0FF7D017C001200339E9000201FE0FCA3E0FDA341
:202CC000E0FEA3E0FF9000202D1200206C9000201EE0FFE4FDFC1200339E9000201EE0FFFF
:202CE0007B017A2079427D107C0012002EEB90002042A3A3A3E05480FFEF70DE9000201F35
:202D0000A3A3A3E05478FFE4FEFDFC78031200202B120020782D43000000002D57000000CE
:202D2000012D6B000000032D6B000000042D6B000000052D6B000000062D6B000000070081
:202D4000002D819000201EE0FF7B017A2079527D047C0012002EEB9000201EE0FF7B017A6C
:202D600020794E7D037C0012002EEB9000201EE0FF7B017A20794A7D027C0012002EEB8019
:202D8000037F00227F012290002021EFF07B017A2079427D107C0012002EEB90002042A3A3
:202DA000A3A3E05480FFEF60037F002290002022A3A3A3E05407FFE4FEFDFC120020782D80
:202DC000D8000000022DD8000000042DD80000000600002DD57F002290002022A3A3A3E0C7
:202DE0005478FFE4FEFDFC78031200202B120020782E19000000002E36000000012E53007E
:202E00000000032E53000000042E53000000062E530000000700002E7A90002052E0FCA3F2
:202E2000E0FDA3E0FEA3E0FF9000202D1200206C7D04120033969000204EE0FCA3E0FDA3DE
:202E4000E0FEA3E0FF9000202D1200206C7D03120033969000204AE0FCA3E0FDA3E0FEA3C2
:202E6000E0FF9000202D1200206C90002021E0FF7D027C001200339E80037F002290002096
:202E800026E0FCA3E0FDA3E0FEA3E0FF9000202D1200206C90002021E0FF7D017C00120076
:202EA000339E90002022E0FCA3E0FDA3E0FEA3E0FF9000202D1200206C90002021E0FFE401
:202EC000FDFC1200339E90002021E0FF7B017A2079427D107C0012002EEB90002042A3A329
:202EE000A3E05480FFEF70DE7F01229000202AEFF0A3ECF0A3EDF0A3EBF0A3EAF0A3E9F06E
:202F0000E4A3F0A3F0E4FFFEFDFC9000203E1200206C9000202BE0FCA3E0FD9000202AE050
:202F2000FF120031F29000202AE0FFE4FD1200348CE0FF0D120034DFE0FF120032CAE0FF14
:202F4000E4FD120034DFE4FFFEFC900020371200206CE490002032F0120034AC12003267B6
:202F600090002032E004F0E0C3942040EB90002037E0FCA3E0FDA3E0FEA3E0FF9000202DF6
:202F8000E0FBA3E0FAA3E0F912002051E4FFFEFDFC900020371200206CE490002032F012B3
:202FA0000034AC1200326790002032E004F0E0C3940940EB90002037A3A3E0FEA3E0FBEEEE
:202FC000FAE4F9F89000202BE0FEA3E0FFE4FCFDC31200201A601E90002030E475F0011241
:202FE000002004FED3741E95F0EE6480F87480984003012F0522E490002000F0A3F090002E
:203000002000E0FEA3E0FFC39402EE9400505BEF2404FFE43EFE1200317090002002EEF031
:20302000A3EFF0E0FD90002001E025E0FB90002000E033FA74562BF58274203AF583759329
:2030400000EDF090002002E0FF74572BF58274203AF583759300EFF090002001E004F07073
:203060009D90002000E004F08094E490002000F0A3F090002000E0FEA3E0FFC39403EE9418
:203080000050541200317090002002EEF0A3EFF0E0FD90002001E025E0FB90002000E03396
:2030A000FA745A2BF58274203AF583759300EDF090002002E0FF745B2BF58274203AF58333
:2030C000759300EFF090002001E004F070A490002000E004F0809B020020C490002006EE47
:2030E000F0A3EFF0900020647408F0F5C84402F0F5C87F327E00120034D290002064E044AF
:2031000004F0F5C87F647E00120034D2120034C4900020627408F0A3E4F090002062E0FC98
:20312000A3E0FD4C6043A3E054FAF090002006E0FEA3E0FFEC5EFEED5F4E600890002064EB
:20314000E04404F090002064E0120034CC120034CE90002064E04401F0F5C890002062E065
:20316000C313F0A3E013F080B190002064E0FF22C2AFEE4408FE120030DB90002064EFF004
:20318000E490002004F0A3F0900020627480F0A3E4F090002062E07002A3E0603790002079
:2031A00064E054FA120034CB120034C4AFC8EF30E31490002062E0FEA3E0FF90002004E0CF
:2031C0004EF0A3E04FF090002062E0C313F0A3E013F080BE90002064E054F8F0F5C87F9077
:2031E0007E01120034D2D2AF90002004E0FEA3E0FF229000203CECF0A3EDF0AB07E4FA1297
:20320000003477120032CA9000203EE0FCA3E0FDA3E0FEA3E0FF78011200202B9000203EE4
:203220001200206C0AEAB420D69000203CE0FEA3E0FFE4FCFDA31200206CE4FA120034774D
:20324000120032CA9000203EE0FCA3E0FDA3E0FEA3E0FF78011200202B9000203E1200201D
:203260006C0AEAB409D622E4FCFDFE900020331200206C90002033E0FCA3E0FDA3E0FEA37A
:20328000E0FF90002032E0F9F81200203EA31200206C90002037E0FCA3E0FDA3E0FEA3E0A4
:2032A000FF90002033E0F8A3E0F9A3E0FAA3E0FBEF4BFFEE4AFEED49FDEC48FC9000203724
:2032C0001200206C9000202AE0FFAE077D01120034D91D020034D990002013EFF0A3ECF0F8
:2032E000A3EDF0C3EC94015027A3E0FCA3E0FDA3E0FEA3E0FF9000202D1200206C90002066
:2033000014E0FCA3E0FD90002013E0FF0200339E90002016E0FCA3E0FDA3E0FEA3E0FF9013
:2033200000201D1200206C90002014E0FCA3E0FD90002013E0FF120034332290002019ECA0
:20334000F0A3EDF0A3EBF0A3EAF0A3E9F0C007E47F21FEFDFC9000201F1200206C90002027
:2033600019E0FEA3E0FFE4FCFD900020231200206CD00712002BFA9000204AE0FCA3E0FD22
:20338000A3E0FEA3E0FF9000201BE0FBA3E0FAA3E0F90200205190002021E0FF7C0090005C
:2033A000202AEFF0C007C004C0059000202DE0FCA3E0FDA3E0FEA3E0FF9000203E12002038
:2033C0006CD005D004D007120031F29000202AE0FFE4FD1200348CE0FF0D120034E5E0FF6A
:2033E0001D020034E590002013EFF090002016EBF0A3EAF0A3E9F090002014ECF0A3EDF039
:20340000C3EC940190002013E0FF5013A3E0FCA3E0FDA3E0FBA3E0FAA3E0F902002EEBA32F
:20342000E0FCA3E0FDA3E0FBA3E0FAA3E0F91200333B22AB05AA04A9079000201DE0FCA3BD
:20344000E0FDA3E0FEA3E0FF9000204A1200206CAF01C007E47F22FEFDFC9000202212001D
:20346000206CAE02AF03E4FCFD900020261200206CD00702002D879000203EE0FCA3A3E090
:20348000FEA3E05401FFA907AF03AD01ED24FF929122AE07E4FD1200348C0D120034D31D47
:2034A000120034D9120034DF020034E59000202AE0FFA290E4339000203BF09000203BE005
:2034C0005401FF2290002064E04401F0F5C87FF47E0122ED24FF929022ED24FF929222EDE5
:2034E00024FF929522ED24FF929322FFFFFFFFFFFFFFFFFFFFFFFFFFFFFFFFFFFFFFFFFF1E
:20350000FFFFFFFFFFFFFFFFFFFFFFFFFFFFFFFFFFFFFFFFFFFFFFFFFFFFFFFFFFFFFFFFCB
:20352000FFFFFFFFFFFFFFFFFFFFFFFFFFFFFFFFFFFFFFFFFFFFFFFFFFFFFFFFFFFFFFFFAB
:20354000FFFFFFFFFFFFFFFFFFFFFFFFFFFFFFFFFFFFFFFFFFFFFFFFFFFFFFFFFFFFFFFF8B
:20356000FFFFFFFFFFFFFFFFFFFFFFFFFFFFFFFFFFFFFFFFFFFFFFFFFFFFFFFFFFFFFFFF6B
:203F0000120020C022FFFFFFFFFFFFFFFFFFFFFFFFFFFFFFFFFFFFFFFFFFFFFFFFFFFFFFA8
:203F2000FFFFFFFFFFFFFFFFFFFFFFFFFFFFFFFFFFFFFFFFFFFFFFFFFFFFFFFFFFFFFFFFA1
:203F4000FFFFFFFFFFFFFFFFFFFFFFFFFFFFFFFFFFFFFFFFFFFFFFFFFFFFFFFFFFFFFFFF81
:203F6000FFFFFFFFFFFFFFFFFFFFFFFFFFFFFFFFFFFFFFFFFFFFFFFFFFFFFFFFFFFFFFFF61
:203F8000FFFFFFFFFFFFFFFFFFFFFFFFFFFFFFFFFFFFFFFFFFFFFFFFFFFFFFFFFFFFFFFF41
:208000000200B3016D64350025730000020461E5257800220205958B3098FDAF99C2987EF5
:208020000022740002008FFF416E6F00416EBA01516E91694C6F7645446C696E4B5377695E
:2080400054634800446EA40000012C467EDE0010184500034A814B00000000000000000076
:20806000004878D401020408102040804187CB01427727000A42772F0000427723000042E9
:208080007725000042771F00004277310000427729FFFF427721800044771B000000004230
:2080A0007715000042771700004277190000C11F4185FC004485FD00000000415D1E00422C
:2080C00081A3000042819B0000426D160000426D1800004275BE0000527B3C872FBC872FEC
:2080E000C8872FD9872FEB872FD9872FEB43874E86FFEA4C7FAF877CEA877CF2877CF587F6
:208100007CF858761587259387259B8725A58725AF8725B88725C18725C68725CE46760954
:208120008725C68725D346760F8725DA8725DE6040714500081018202830380A121A220CD9
:20814000141C240E161E262E01020304050607090B0D0F11131517191B1D1F212325272970
:208160002A2B2C2D2F31323334353637393A3B3C3D3E3F467DDE87AD2787AD2E497DD58792
:20818000AD3387AD4287AD5248789E00010009001100194878AE000800100018001A4982EE
:2081A000C5878DFF878E07878E0C436EBF00000062F74B3286A2526367695F64756D790099
:2081C00000000000000000000000008523A26367695F6C6F67696E000000000000000000AA
:2081E00000008617106367695F706F727400000000000000000000000082EDF36367695F87
:20820000736574706F72740000000000000000008615526367695F766C616E00000000001D
:208220000000000000000084D82C6367695F736574766C616E00000000000000000084BBE8
:208240001B6367695F64656C766C616E000000000000000000869A046367695F716F730082
:208260000000000000000000000000008603E26367695F7170626173650000000000000085
:2082800000000085FC166367695F716473637000000000000000000000008600FF636769E2
:2082A0005F7131700000000000000000000000000085EBEB6367695F7076696400000000AD
:2082C0000000000000000000833F5C6367695F766964000000000000000000000000008427
:2082E00016436367695F6164647669640000000000000000000081B5A96367695F64657677
:208300006963650000000000000000000082606D6367695F64657461696C000000000000D8
:208320000000000084091E6367695F737461746973740000000000000000008513996367F9
:20834000695F7472756E6B000000000000000000000083B9776367695F6D6972726F720041
:20836000000000000000000000857F5D6367695F7061737300000000000000000000000053
:20838000834C076367695F737973000000000000000000000000008315F76367695F74720F
:2083A00061700000000000000000000000008681156367695F6261636B75700000000000C8
:2083C00000000000008584256367695F62616B5F64617461000000000000000086816263EA
:2083E00067695F7265736574000000000000000000000083BEB86367695F73747000000049
:208400000000000000000000000083E7EF6367695F736E6D705F636D7574797365740000D6
:208420000085F11D6367695F736E6D705F636D75747964656C0000008400076367695F7303
:208440006E6D705F74726170736574000000008610056367695F736E6D705F74726170640A
:20846000656C0000000085AEB66367695F736E6D70000000000000000000000000868A29B9
:208480006367695F6A756D626F00000000000000000000000000000000000000000000002D
:2084A00000000000000000000000004286DC0000423729000042356B00004231AE00004231
:2084C00037250000423727000049348681B1A181B1AF81B1D752366D81B1EB81B20281B266
:2084E0001881B22E81B24681B2624C371581B27F81B29C81B2BA81B2D16032372B000000F7
:2085000000000000000000000000000000000000000000000000000000000000000000005B
:208520000000000000000000000000000000006064314A00010003000600010004000100EC
:20854000AB000A004C00010005000100000000000000000000000000000000000000000013
:20856000000000000D000000000000000000000000000000000000000000000000000000EE
:208580000000000000000000000000000000000000000000000000606434220001000300BD
:2085A0000600010004000100AB000A004C00010005000200000000000000000000000000A6
:2085C0000000000000000000000000000D000000000000000000000000000000000000008E
:2085E00000000000000000000000000000000000000000000000000000000000000000601B
:2086000096338C000100030006000100020001000200020001000100FF00000000000000F2
:2086200000000000000000000000000000000000000000000B000100030006000100040020
:208640000100AB000A004C000100050003000000000000000000000000000000000000000F
:208660000000000000000D00000000000000000000000000000000000000000000000000ED
:20868000000000000000000000000000000000000000000000000000006096367F0001002E
:2086A000030006000100020001000200020001000100FF00000000000000000000000000A8
:2086C00000000000000000000000000000000B00010003000600010004000100AB000A00CA
:2086E0004C0001000500040000000000000000000000000000000000000000000000000024
:208700000D000000000000000000000000000000000000000000000000000000000000004C
:2087200000000000000000000000000000000000000000606430E200010003000600010058
:2087400004000100AB000A004C000100050005000000000000000000000000000000000008
:2087600000000000000000000D0000000000000000000000000000000000000000000000EC
:208780000000000000000000000000000000000000000000000000000000006064307E0067
:2087A000010003000600010004000100AB000A004C0001000500060000000000000000009C
:2087C000000000000000000000000000000000000D0000000000000000000000000000008C
:2087E000000000000000000000000000000000000000000000000000000000000000000079
:2088000000000060642FFA00010003000600010004000100AB000A004C000100050007004D
:208820000000000000000000000000000000000000000000000000000D000000000000002B
:20884000000000000000000000000000000000000000000000000000000000000000000018
:208860000000000000000000000000606431B400010003000600010004000100AB000A008A
:208880004C000100050008000000000000000000000000000000000000000000000000007E
:2088A0000D00000000000000000000000000000000000000000000000000000000000000AB
:2088C00000000000000000000000000000000000000000606432E0000100030006000100B7
:2088E00004000100AB000A004C000100050009000000000000000000000000000000000063
:2089000000000000000000000D00000000000000000000000000000000000000000000004A
:2089200000000000000000000000000000000000000000000000000000000044336809311E
:208940004A0044349F0934220044349B09338C0144372109367F014433440930E2004431D5
:20896000B009307E00443146092FFA004434930931B4004434970932E000422FF800004ACD
:2089800081CDFC06FC03FC0400A120004247E20001438763818022545F95000100030006B9
:2089A00000010004000100AB000A004C0001410400004286FC00004286FE000043476F8166
:2089C000B57A6028429200000000000000000000000000000000000000000000000000000C
:2089E000000000000000000000000000000062104559000000000000000000000000000067
:208A0000000000000000000000000000000000000000000000000000000000000000000056
:208A2000000000000000000000000000000000000000000000000000000000000000000036
:208A4000000000000000000000000000000000000000000000000000000000000000000016
:208A60000000000000000000000000000000000000000000000000000000000000000000F6
:208A80000000000000000000000000000000000000000000000000000000000000000000D6
:208AA0000000000000000000000000000000000000000000000000000000000000000000B6
:208AC000000000000000000000000000000000000000000000000000000000000000000096
:208AE000000000000000000000000000000000000000000000000000000000000000000076
:208B0000000000000000000000000000000000000000000000000000000000000000000055
:208B2000000000000000000000000000000000000000000000000000000000000000000035
:208B4000000000000000000000000000000000000000000000000000000000000000000015
:208B60000000000000000000000000000000000000000000000000000000000000000000F5
:208B80000000000000000000000000000000000000000000000000000000000000000000D5
:208BA0000000000000000000000000000000000000000000000000000000000000000000B5
:208BC000000000000000000000000000000000000000000000000000000000000000000095
:208BE000000000000000000000000000000000000000000000000000000000000000000075
:208C00000000621042BA0000000000000000000000000000000000000000000000000000E6
:208C2000000000000000000000000000000000000000000000000000000000000000000034
:208C4000000000000000000000000000000000000000000000000000000000000000000014
:208C60000000000000000000000000000000000000000000000000000000000000000000F4
:208C80000000000000000000000000000000000000000000000000000000000000000000D4
:208CA0000000000000000000000000000000000000000000000000000000000000000000B4
:208CC000000000000000000000000000000000000000000000000000000000000000000094
:208CE000000000000000000000000000000000000000000000000000000000000000000074
:208D0000000000000000000000000000000000000000000000000000000000000000000053
:208D2000000000000000000000000000000000000000000000000000000000000000000033
:208D4000000000000000000000000000000000000000000000000000000000000000000013
:208D60000000000000000000000000000000000000000000000000000000000000000000F3
:208D80000000000000000000000000000000000000000000000000000000000000000000D3
:208DA0000000000000000000000000000000000000000000000000000000000000000000B3
:208DC000000000000000000000000000000000000000000000000000000000000000000093
:208DE000000000000000000000000000000000000000000000000000000000000000000073
:208E0000000000000000000000000000000000000000000000005045490000000000000074
:208E2000000000000000000000602047B300000000000000000000000000000000000000B8
:208E40000000000000000000000000000060204772000000000000000000000000000000D9
:208E60000000000000000000000000000000000000602044D100000000000000000000005D
:208E8000000000000000000000000000000000000000000000602047930000000000000078
:208EA00000000000000000000000000000000000000000000000000000605044F5000000C9
:208EC000000000000000000000000000000000000000000000000000000000000000000092
:208EE000000000000000000000000000000000000000000000000000000000000000000072
:208F0000000000000000000000000000004144CE014647690180C200000041479200527CDC
:208F200008871A5C871A64871A6A871A71871A7A871A82447B8C00000000447B9000000032
:208F400014447B8800000001004E7C30097C30097C30097C30000000000068656C6C6F3F49
:208F60003F3F0068696869232323006D616320777269746500676F206C6F6164657200631C
:208F80006C6F7365746D006D61632072656164002573006D6163006D6F64656C207265611E
:208FA00064006D6F64656C3A004447532D3132313654006677766572207265616400667716
:208FC0007665723A00332E30302E313700726263686B004661696C004F6B003153657442D4
:208FE0007566663A25640A0032536574427566663A25640A00900887F1EFF0D2212222325D
:2090000049434D500A000180C200000F3C74723E3C746820636F6C7370616E3D343E2573FC
:209020000A3C74723E0A203C74643E3C623E42797465730A203C746420636F6C7370616E19
:209040003D333E256C750A0A003C74723E0A203C74643E3C623E25730A203C74643E256CEB
:20906000750A203C74643E3C623E25730A203C74643E256C750A0A0087302487302C873080
:209080002F87303287380987381187381787381E87382787382F76636200203C74643E0AE2
:2090A000203C73656C656374206E616D653D25733E0A203C6F7074696F6E2076616C7565C4
:2090C0003D25643E25730A000A3C7472206865696768743D33303E0A203C746420616C69B3
:2090E000676E3D63656E7465723E3C623E25730A203C74643E3C623E0A0087937087937EA7
:2091000087938C87939F8793B38793CA8793E28793F68793CA20203C696E70757420747996
:2091200070653D636865636B626F78206E616D653D25732076616C75653D25642025733E47
:209140002025733C62723E0A00000000010A3C7472206865696768743D33303E0A203C7481
:209160006420616C69676E3D6C6566743E3C623E266E6273703B25730A203C74643E3C6298
:209180003E0A0086E9CD86E9DB20203C696E70757420747970653D726164696F206E616DCB
:2091A000653D25732076616C75653D256425733E2025733C62723E0A000A3C747220686573
:2091C000696768743D33303E0A203C746420616C69676E3D6C6566743E3C623E266E627331
:2091E000703B25730A203C74643E3C623E0A0086EDC300000086EDD186EDE486EDF886EE1A
:209200000F86EE2786EE3B86EE0F20203C696E70757420747970653D636865636B626F7860
:20922000206E616D653D25732076616C75653D25642025733E2025733C62723E0A004E6FD2
:2092400074653A3C62723E0A53313A2064657669636520626F6F7475703C62723E0A4632CC
:209260003A206C696E6B207570202F206C696E6B20646F776E3C62723E0A46333A206162FE
:209280006E6F726D616C2072656365697665206572726F723C62723E0A46343A2061626E9B
:2092A0006F726D616C207472616E736D6974206572726F723C62723E0A54313A206C696E3D
:2092C0006B207570202F206C696E6B20646F776E3C62723E0A54323A2061626E6F726D6111
:2092E0006C2072656365697665206572726F723C62723E0A54333A2061626E6F726D616C30
:20930000207472616E736D6974206572726F723C62723E0A0000027400000000000000EBB8
:209320007008E709F608DFFA801B89828A831410E70AF593E0A3F608DFFA8009F593E493BC
:20934000A3F608DFF9ECFAA9F0EDFB2288F0EF60010E4E60F088F0ED60C51410E7E7CB70E0
:209360000E88828C838B93E709F0A3DFFA80D61410E72A89828A83F593ECFAE0A3C8C582A9
:20938000C8CCC583CCCBC593CBF0A3C8C582C8CCC583CCCBC593CBDFE2DEE080AA89828AC1
:2093A00083F593ECFAE493A3C8C582C8CCC583CCCBC593CBF0A3C8C582C8CCC583CCCBC523
:2093C00093CBDFE1DEDF02009347EB7002E72289828A831410E704F593E022F593E493229E
:2093E000F8EB7006E7C828F3E82289828A831410E708F593E0C828F0E822F593E49322BBE7
:20940000000327F722F8EB89828A831410E706F593E028F022F593E4932822BB0002F7223C
:20942000BB8000500989828A838B931593F022EF8DF0A4A8F0CF8CF0A428CE8DF0A42EFECE
:2094400022BC000BBE0029EF8DF084FFADF022E4CCF875F008EF2FFFEE33FEEC33FCEE9D97
:20946000EC984005FCEE9DFE0FD5F0E9E4CEFD22EDF8F5F0EE008420D21CFEADF075F008BE
:20948000EF2FFFED33FD4007985006D5F0F222C398FD0FD5F0EA22C2D5EC30E709B2D5E43E
:2094A000C39DFDE49CFCEE30E716B2D5E4C39FFFE49EFE12009441C3E49DFDE49CFC800444
:2094C0001200944130D507C3E49FFFE49EFE22C5F0F8A3E028F0C5F0F8E582158270021538
:2094E00083E038F022A3F8E0C5F025F0F0E582158270021583E0C838F0E822EB7007E7F56A
:20950000F009E7192289828A831410E708F593E0F5F0A3E022F593E493F5F074019322F80D
:20952000EB700C09E5F027C7F5F019E837C72289828A831410E707F593E8020094E5F59355
:20954000E4740193F5F0E49322BB000B09C5F027F7C5F01937F722F8EB89828A831410E7DB
:2095600007F593E8020094CFF59374019325F0F5F0E4933822BB0006F709A7F01922BB80E6
:2095800000500D89828A838B931593F0E5F0A3F022E88FF0A4CC8BF0A42CFCE98EF0A42CC1
:2095A000FC8AF0EDA42CFCEA8EF0A4CDA8F08BF0A42DCC3825F0FDE98FF0A42CCD35F0FC83
:2095C000EB8EF0A4FEA9F0EB8FF0A4CFC5F02ECD39FEE43CFCEAA42DCE35F0FDE43CFC221E
:2095E00075F008758200EF2FFFEE33FECD33CDCC33CCC58233C5829BED9AEC99E58298408C
:209600000CF582EE9BFEED9AFDEC99FC0FD5F0D6E4CEFBE4CDFAE4CCF9A88222B800C1B912
:209620000059BA002DEC8BF084CFCECDFCE5F0CBF97818EF2FFFEE33FEED33FDEC33FCEB11
:2096400033FB10D703994004EB99FB0FD8E5E4F9FA227818EF2FFFEE33FEED33FDEC33FCCD
:20966000C933C910D7059BE99A4007EC9BFCE99AF90FD8E0E4C9FAE4CCFB2275F010EF2F07
:20968000FFEE33FEED33FDCC33CCC833C810D7079BEC9AE899400AED9BFDEC9AFCE899F8A7
:2096A0000FD5F0DAE4CDFBE4CCFAE4C8F922CFF4CFCEF4CECDF4CDCCF4CC22EB9FF5F0EA28
:2096C0009E42F0E99D42F0EC6480C864809845F022EB9FF5F0EA9E42F0E99D42F0E89C45ED
:2096E000F022E8600FECC313FCED13FDEE13FEEF13FFD8F122E8600FEFC333FFEE33FEED14
:2097000033FDEC33FCD8F122EB7006E9F802009CBF89828A831410E706F59302009CCBF565
:209720009302009CD7BB0006E9F802009D30BB8000500C89828A838B931593020097E4229C
:20974000EB7006E9F802009D1989828A831410E706F593020097B8F59302009CD7EB7006AF
:20976000E9F802009CE789828A831410E706F59302009CF4F59302009D007401FF3395E0FD
:20978000FEFDFCA3A3A3E0CF2FF0E582158270021583E0CE3EF0E582158270021583E0CD82
:2097A0003DF0E582158270021583E0CC3CF0227401FF3395E0FEFDFCA3A3A3E02FFFF0E59B
:2097C00082158270021583E03EFEF0E582158270021583E03DFDF0E582158270021583E060
:2097E0003CFCF022ECF0A3EDF0A3EEF0A3EFF022F5F0C582A4C582C5F0C583A42583F583C6
:2098000022A42582F582E5F03583F58322EB7006E9F802009D3C89828A831410E706F5936F
:2098200002009D4EF59302009D8EBB001CD093D0F0D0E0F8D0E0C9FBD0E0FAD0E0CBC8C0C3
:20984000E0C0F0C09302009D45BB80005022D093D0F0D0E0F8D0E0C9F582D0E0CAF583D017
:20986000E0CB14C8C0E0C0F0C093889302009D85D093D083D082D0E0D0E0D0E0E473D093AD
:20988000D083D082F8E4937012740193700DA3A393F8740193F5828883E47374029368602A
:2098A000EFA3A3A380DFD093D083D082F8E4937012740193700DA3A393F8740193F582881B
:2098C00083E473740293B5F0067403936860E9A3A3A3A380D8D093D083D082E493701274E6
:2098E0000193700DA3A393F8740193F5828883E4737402936C70127403936D700C740493B0
:209900006E70067405936F60DDA3A3A3A3A3A380CA8B938A838982159353937FE4737593ED
:2099200008E5512582F582E5503583F583B550048582512210AF06858251F5502285825107
:20994000F550D2AF22759308E5512582F582E5503583F58322EB700C87F009E608B5F04179
:20996000603F80F489828A831410E70FF593E0F5F0A3E608B5F02A602880F3F593E493F506
:20998000F0A3E608B5F01A601880F2CB701588828C838B9387F009E493A3B5F004600280F1
:2099A000F380611410E72E89828A83F593ECFAE0F5F0A3C8C582C8CCC583CCCBC593CBE423
:2099C00093A3C8C582C8CCC583CCCBC593CBB5F033603180DA89828A83F593ECFAE493F5F7
:2099E000F0A3C8C582C8CCC583CCCBC593CBE493A3C8C582C8CCC583CCCBC593CBB5F004C7
:209A0000600280D97F00F845F0600EE863F0806480D395F01F40027F012202009955020085
:209A2000998BED60F51410E7F5CB701488828C83F59387F009E0A3B5F0CA60C880F480C47E
:209A40001410E72D89828A83F593ECFAE0F5F0A3C8C582C8CCC583CCCBC593CBE0A3C8C52B
:209A600082C8CCC583CCCBC593CBB5F097609580DB89828A83F593ECFAE493F5F0A3C8C530
:209A800082C8CCC583CCCBC593CBE0A3C8C582C8CCC583CCCBC593CBB5F0A360A180DAEBF8
:209AA0007008E709F60870FA801B89828A831410E70AF593E0A3F60870FA8009F593E49313
:209AC000A3F60870F9ECFAA9F0EDFB2288F0ED60CE1410E7F0CB700E88828C83F593E7098B
:209AE000F0A370FA80DF1410E72889828A83F593ECFAE0A3C8C582C8CCC583CCCBC593CB29
:209B0000F0A3C8C582C8CCC583CCCBC593CB70E280B589828A83F593ECFAE493A3C8C582D7
:209B2000C8CCC583CCCBC593CBF0A3C8C582C8CCC583CCCBC593CB70E1808CEB700C87F01C
:209B400009E608B5F019DFF6801589828A831410E711F593E0F5F0A3E608B5F002DFF50257
:209B6000009BECF593E493F5F0A3E608B5F07DDFF48079CB701388828C838B9387F009E412
:209B800093A3B5F067DFF580631410E73089828A83F593ECFAE0F5F0A3C8C582C8CCC583B8
:209BA000CCCBC593CBE493A3C8C582C8CCC583CCCBC593CBB5F035DFDCDEDA802F89828A9B
:209BC00083F593ECFAE493F5F0A3C8C582C8CCC583CCCBC593CBE493A3C8C582C8CCC583EB
:209BE000CCCBC593CBB5F004DFDBDED97FFFB5F0020F2240027F012202009B3B02009B736F
:209C000088F0EF60010E4E60EEED60EC1410E7ECCB701288828C83F59387F009E0A3B5F00C
:209C2000CBDFF680C71410E72F89828A83F593ECFAE0F5F0A3C8C582C8CCC583CCCBC5933B
:209C4000CBE0A3C8C582C8CCC583CCCBC593CBB5F09ADFDDDEDB809489828A83F593ECFAC3
:209C6000E493F5F0A3C8C582C8CCC583CCCBC593CBE0A3C8C582C8CCC583CCCBC593CBB563
:209C8000F004DFDCDEDA02009BECEF4E6022EF60010EEDBB0007F709DFFCA9F022BB800037
:209CA000500E89828A838B931593F0A3DFFCDEFA22C3E49FFFE49EFEE49DFDE49CFC22E639
:209CC000FC08E6FD08E6FE08E6FF22E0FCA3E0FDA3E0FEA3E0FF22E493FC740193FD740233
:209CE00093FE740393FF22E6FB08E6F908E6FA08E6CBF822E0F8A3E0F9A3E0FAA3E0FB22B4
:209D0000E493F8740193F9740293FA740393FB227401FF3395E0FEFDFC080808E62FFFF674
:209D200018E63EFEF618E63DFDF618E63CFCF622ECF608EDF608EEF608EFF622E6FB08E6E0
:209D4000FA08E6F922EBF608EAF608E9F622E0FBA3E0FAA3E0F922F8E0FBA3A3E0F925F031
:209D6000F0E582158270021583E0FA38F022F8E0FBA3A3E025F0F9F0E582158270021583C8
:209D8000E038FAF022EBF0A3EAF0A3E9F022E493FB740193FA740293F92270253032643D79
:209DA000002564005761726E696E6700546F2073657420516F5320737570706F7274206F16
:209DC0006E20616E7920706F72742C204A756D626F204672616D6520737570706F72742017
:209DE0006D7573742062652064697361626C65642E006367695F716F7300706F72743D0046
:209E0000706F72743D253032640073706565643D0073706565643D2564007072696F72699B
:209E200074793D007072696F726974793D2564007365745F666C6F773D007365745F666C93
:209E40006F773D2564006367695F736574706F72743D256400506F72742053657474696EB1
:209E600067004D656469612074797065206973206368616E6765642E3C62723E43757272BB
:209E8000656E742073706565642073657474696E67206973206E6F74207375697461626CAB
:209EA000652E00766C616E5F69643D00766C616E5F69643D256400646573633D00260076DA
:209EC00063623D007663623D25303264006367695F736574766C616E3D256400564C414E97
:209EE0002053657474696E67004174206C65617374206F6E6520564C414E2067726F757076
:209F0000206D75737420696E636C7564656420746865207472756E6B696E6720706F727418
:209F200073207768656E20656E61626C6520746865207472756E6B696E672066756E637422
:209F4000696F6E2E006E756D3D006E756D3D2564007663623D2564006367695F64656C76AC
:209F60006C616E0076747970653D0076747970653D25640044656661756C74007379733DD2
:209F8000006C6F633D006C6F67696E3D0053797374656D2053657474696E6700496E7661DF
:209FA0006C6964206C6F67696E2074696D656F75742076616C7565006367695F73797300DA
:209FC00069703D00496E76616C69642049502041646472657373006D6B3D00496E76616CF6
:209FE0006964205375626E6574204D61736B0067773D00496E76616C69642047617465775D
:20A000006179204950004950207375626E6574206D75737420626520657175616C20746F58
:20A020002067617465776179207375626E65742E006F6C645F706173733D006E65775F7084
:20A040006173733D0072656E65775F706173733D004368616E67652050617373776F72644F
:20A060000050617373776F7264206C656E6774682063616E2774206265207A65726F2E0009
:20A080006367695F70617373004F6C642070617373776F72642069732077726F6E672E004E
:20A0A0004E65772070617373776F726420697320696E636F6E73697374656E742E005472B2
:20A0C00061702053657474696E6700496E76616C69642054726170204950006367695F7474
:20A0E000726170006669623D00636F703D00257325256400656E61626C65253032643D005B
:20A10000746B70253032643D002530326426005472756E6B2053657474696E670054686584
:20A12000205472756E6B696E6720706F727473206D7573742073657420746F20746865207C
:20A1400073616D6520564C414E2067726F75702E006367695F7472756E6B006D6F64653DE5
:20A16000006D6F64653D2530326400736E69666665723D00736E69666665723D25303264D3
:20A1800000736F757263653D00736F757263653D2530326400647669643D00505649442001
:20A1A00053657474696E6700496E76616C6964205649442076616C7565006367695F707642
:20A1C0006964005649442025303264206973206E6F742065786973742C206F7220506F728C
:20A1E000742025303264206973206E6F7420746865206D656D626572206F66205649442062
:20A20000253032642E00276367695F7076696427007669643D005649442053657474696E98
:20A220006700564944206D757374206265206265747765656E203220616E64203430393464
:20A24000006367695F6164647669640054686520564944207461626C652069732066756C51
:20A260006C005468652056494420697320657869737420696E20564944207461626C6500E3
:20A280007025643D007461675F69643D007461675F69643D256400546865206D616E616770
:20A2A000656D656E7420564944206F6620706F727420253032642069732025642C20736FCA
:20A2C0002069742063616E206E6F7420626520756E73656C65637465642E00276367695FA4
:20A2E0007365747669643D256427005468652056494420697320746865206D616E616765D8
:20A300006D656E7420564944206F6620706F727420253032642C20736F2069742063616E24
:20A32000206E6F742062652064656C657465642E006367695F7365747669643D2564005267
:20A34000656D6F766520564C414E00656E61626C65645F666C61673D00656E61626C6564C4
:20A360005F666C61673D256400546F20736574204A756D626F204672616D652073746174EB
:20A3800075732C516F532049454545203830322E315120737570706F727420737461747566
:20A3A00073206D757374206265207468652073616D65206F6E20616E7920706F72742E00BB
:20A3C0006367695F6A756D626F007061737377643D00716F73747970653D00716F7374796D
:20A3E00070653D256400666C61673D00666C61673D256400625F7072693D005370616E6E42
:20A40000696E6720547265652053657474696E6700496E76616C69642042726964676520FC
:20A420005072696F72697479006367695F73747000625F6167653D00496E76616C696420BF
:20A44000427269646765204D61782041676500625F68656C6C6F3D00496E76616C69642043
:20A460004272696467652048656C6C6F2054696D6500625F64656C61793D00496E76616CC5
:20A4800069642042726964676520466F72776172642044656C61790064636F73743D0049DB
:20A4A0006E76616C6964205061746820436F73742076616C756500647072693D00496E7662
:20A4C000616C6964205072696F726974792076616C756500736E6D705F6D6F646966793D41
:20A4E00000736E6D705F6D6F646966793D25642E25642E0047436F6D3D007379733D256444
:20A5000000534E4D5020436F6E66696775726500457863656564206D6178696D756D20436C
:20A520006F6D6D756E6974792047726F75702E006367695F736E6D7000436F6D6D756E6916
:20A540007479204E616D652043616E204E6F74204265204475706C69636174652E000063D7
:20A560006D7574793D0025642E25642E0061757468656E3D0054436F6D3D00547261702038
:20A58000436F6D6D756E697479204E616D65204D75737420457869737420496E20534E4D7A
:20A5A0005020436F6D6D756E697479204E616D65732E00496E76616C696420534E4D5020DF
:20A5C000547261702049502E00457863656564206D6178696D756D205472617020436F6D9B
:20A5E0006D756E6974792047726F75702E002854726170204950202B205472617020436F0E
:20A600006D6D756E697479204E616D65292043616E204E6F74204265204475706C69636131
:20A6200074652E00747261703D00E525244CF582E43475F583759308E00525229008754997
:20A640003017049008754CE475F00112009D57020093CA2010E57F2ED2108018EF540F24F5
:20A6600090D43440D4FF30140BEF24BFB41A0050032461FFE526600215260529E529700213
:20A68000052830171190087549E475F00112009D57EF0200941B0200B4DC7403D21780037A
:20A6A000E4C217F5259008754912009D85E4F526F528F529E52660087F201200A67480F44D
:20A6C0007527FFC211C210C212C213C215C216C2181200A63CFF700E3017067F001200A613
:20A6E00085AF29AE2822B42563C2D5C2141200A63CFF24D0B40A00501A75F00A782630D53B
:20A700000508B6FF0106C6A426F620D5047002D21380D824CFB41A00EF5004C2E5D21402AF
:20A7200000A8B2D21180C4D21080BED21280BAD2D580B8D21580B27F201200A6742012075E
:20A740007401B5260040F01200A62AFF1200A6740200A6B4D218D216808F1200A62AFB1240
:20A7600000A62AFA1200A62AF94A4B700679897AA97B8120123DE52660397E00E9C0E02EC0
:20A78000F9EAC0E03400FA120093CAF9D0E0FAD0E0C960060EEE652770E2C2D5EBC0E0EA31
:20A7A000C0E0E9C0E0EE1200A8FAD0E0F9D0E0FAD0E0FB120093CAFF6096EBC0E0EAC0E057
:20A7C000E9C0E01200A674D0E02401F9D0E03400FAD0E0FBE5270460DAD527D70200A75057
:20A7E0007BFF7AA879F6D2128089791080027908C216C2188008D2D5790A8004790AC2D5D3
:20A80000E527047002F527E4FAFDFEFF1200A62AFC7B082011161200A62AFD7B1030100C64
:20A820001200A62AFE1200A62AFF7B20EC3382D592D55013C3E43010069FFFE49EFEE4206D
:20A8400011039DFDE49CFCE4CBF8C211EC700CCFCECDCCE824F8F870F38017C3EF33FFEEEE
:20A8600033FEED33FDEC33FCEB33FB994002FB0FD8E9EB301105F8D0E0C448B211C0E00A5E
:20A88000EC4D4E4F78207B0070C2EAB5270040BCC0E01200A8FCD0F0D0E0201104C4C0E07C
:20A8A000C4B211C0F01200A65DD0F0D5F0EA0200A6B41200987EA75A53A7EA58A7274CA75B
:20A8C0002342A7EE4FA7F644A7F649A73D43A7FC55A7E046A7E045A7E047A9A650A72B2D44
:20A8E000A72F2EA7562BA73323A75420A9922AA6E9480000A74C3F3F3F00790AA2D52013FB
:20A9000014301509B910020404B9080104A2D520160250010420126D9212B526005036C0D4
:20A92000E07F2030131A7F30A2127216721550101200A955C212C216C215C2187F308010BD
:20A94000301503E9C0E01200A674301503D0E0F9D0E0B526CA3015197F30B9100D1200A619
:20A96000747F583014077F788003B908041200A6743012067F2D0200A6747F202018F77F79
:20A980002B2016F222921280CC286E756C6C2900D2111200A62A3011F7C211782630D501D2
:20A9A00008F60200A6E91200A62A7F4960087F4310E7027F5814C0E0EF1200A665743A12E4
:20A9C00000A665D0E0600DC0E0C41200A65DD0E01200A65DD2137526040200A7EAE52A30BB
:20A9E0001C0104F8232824F6F582E43473F58375930822900873F3301C04900873F6E47585
:20AA0000F00112009D57020093CA60E6C52E7002152D14C52E201C05FF02008FF59008731B
:20AA2000F374FFF5F002009D6EFF02059CFAE52B6006D52B037F0022201C101200B537EFCF
:20AA40006008052EE52E7002052D22900873F312009D4E120093CAFF60E5900873F3E4757D
:20AA6000F00112009D5780D71200AA38EFC0E01200AA29D0E040F18091D21C8002C21C9050
:20AA80000873F312009D85E4F52CF52AF52DF52E752B00C21BC219C21AC21D1200A9F3FFEB
:20AAA0007005AF2C7E0022B425321200A9F3FF24D0B40A00500C75F00AC52BA4252BF52B6D
:20AAC00080E824CFB41A00EF5002C2E50200AD13D21A80D6D21980D2D21D80CEEF1200AA3C
:20AAE0002950091200AA68EF600F80A4EFC0E01200AA38D0E06F6098EF70040200AB8312EF
:20AB000000AA0A809D1200AA38EF6077E52B7008052B80041200AA38EF6017201D111200B4
:20AB2000A9DDE475F00112009D57EF1200941BD52BE2201D04052A052C80AF1200AA2EEF04
:20AB4000C0E01200AA29D0E050051200AA0AE4FF201D111200A9DDE475F00112009D57EF9D
:20AB60001200941BEF70D4201D04052A052C0200AAEAE52B6002052B1200AA681200AA2EFA
:20AB8000EF70BD301C05E41200AA0AE52C60030200AAA27EFF7FFF22201D1474FFFCFDFE04
:20ABA000FF1200A9DD12009D4E12009725052A0200AA90D0E080CC7900800A791080067941
:20ABC000088002790AD21EE52B6002052BE9C0E01200AA68EF60DC1200AA38BF2D04D21B2D
:20ABE0008003BF2B0B1200AA68EF60C71200AA2ED0E0B40A028034B40802802FBF302870A1
:20AC0000027408C21EC0E01200AA2ED0E0BF78028003BF5816052BD52B028007D52B04D224
:20AC20001E800B7410801B7002740ABF000BEFF8E4FCFDFEFF0200ACBBC0E0EF1200AA0A13
:20AC4000D0E0F9E4FCFDFEFFE9C0E0ECC0E0EDC0E0EEC0E0EFC0E01200AA2EEFF8D0E0FF32
:20AC6000D0E0FED0E0FDD0E0FCD0F0E8604DB461004007B47B005002C2E524D0503DFA2455
:20AC8000F6500724F95034240AFAEAB5F000502BCFA9F0A42FFF92D5E9C5F0CEA4A2D53E2E
:20ACA000FE92D5E9C5F0CDA4A2D53DFD92D5E9C5F0CCA4A2D53CFCC21E808DE8C0E0201D99
:20ACC00030201E09052C301B0412009CB11200A9DD12009D4E052A20190C201A0FEE8FF05F
:20ACE00012009575800B120097258005EF1200941BD0E01200AA0A0200AA90201D13120096
:20AD0000A9DD12009D4E052AE52D852EF01200957580E41200987EAB7253ABBB58AAD44C2C
:20AD2000AAD042AAAA48ABBF4FABC344AB0543ABB749ABC355AB9846AB9845AB9847AAD8D2
:20AD40002AACFB4E0000AADC4745542000696E6465782E68746D00706F73745F75726C3D0A
:20AD6000002E006367695F6C6F676F757400636F6E6669672E62696E006367695F62616BDC
:20AD80005F64617461006367695F006367695F6C6F67696E004C6F67696E004F6E6C7920C2
:20ADA0006F6E6520757365722063616E206C6F67696E006367695F6465766963650057721C
:20ADC0006F6E672070617373776F7264004C6F67696E2074696D656F7574006367695F707A
:20ADE0006F7274006367695F716F73006367695F717062617365006367695F713170006304
:20AE000067695F7164736370006367695F64656C766C616E006367695F766C616E00636763
:20AE2000695F7472756E6B006367695F6D6972726F72006367695F6A756D626F5F656E61A7
:20AE4000626C6564006367695F737973006367695F737470006367695F706173730063676E
:20AE6000695F74726170006367695F61757468656E736574006367695F736E6D705F74725B
:20AE80006170006367695F736E6D705F656E61626C6564006367695F736E6D705F74726171
:20AEA00070736574006367695F736E6D705F7472617064656C006367695F736E6D705F6329
:20AEC0006D757479736574006367695F736E6D705F636D757479006367695F736E6D705FC7
:20AEE000636D75747964656C006367695F7365747674797065006367695F7076696400632D
:20AF000067695F736574766964006367695F766964006367695F616464766964006367696D
:20AF20005F64656C766964006367695F7265736574006367695F636C72737461740063672C
:20AF4000695F73746174697374006367695F616464766C616E006367695F736574766C6190
:20AF60006E006367695F7365747669643D2564006367695F736E6D705F636D7574796164D6
:20AF800064006367695F736E6D70006367695F736E6D705F7472617061646400900070046A
:20AFA000E0F54090007005E0F541854082854183E020E7077E007F00C2D72289428A43543F
:20AFC00007F5451200B197E02402F544500205451200B03E053AE53A7002053BE54025445D
:20AFE000F540E541354530E604C2E62404F5411200B05E90007004E540F090007005E541F8
:20B00000F0AE45AF44D2D72290007010E020E61EA3EDF0A3E9F0A3EAF0EC5407D2E6900073
:20B020007010F00538E53870020539D2D7227C007D00C2D72290007010E0A2E6B32275F065
:20B0400001800375F0041200B05E78407F06900070921200B17F90007090E5F0F0229000CB
:20B060007090E0540770F7221200B0CB900070087404F0900070107508101200B0B6E49086
:20B08000007004F090007006F0740490007005F090007007F0751D10751C10751E00751F88
:20B0A00004758304758200E4F0753800753900753A00753B0022E4A808F0A3D8FC221200BA
:20B0C000B1751200B0681200B109229000B0FF75080A797078601200B1867518C07519A8DF
:20B0E000751A00751B647510C07511A87512007513017514FF7515FF7516FF751700220001
:20B100000B78667788C0A800649000706AE0440CF0229000706AE054F3F0229000706AE0E2
:20B120004401F0229000706AE054FEF0229000706AE04402F0229000706AE054FDF022902B
:20B1400000706AE04440F0229000706AE054BFF02290007000E04410F02290007000E054B6
:20B16000EFF02290007000E04420F02290007000E05420F0229000700AF00000000022E610
:20B18000F008A3DFFA2289A0E493A3F208B800030989A0D508F222A3E58330E603758304DE
:20B1A0002253797374656D20626F6F747570004C6F67696E20696E76616C696420706173CB
:20B1C00073776F72642066726F6D2025642E25642E25642E25640041757468656E746963F9
:20B1E0006174696F6E206661696C00506F727420256420666962657220696E7365727465E8
:20B200006400506F72742025642066696265722072656D6F76656400506F727420256420D4
:20B220006669626572206C696E6B20757000506F7274202564206669626572206C696E6BEF
:20B2400020646F776E00506F72742025642066696265722072656365697665206572726FC5
:20B260007200506F7274202564206669626572207472616E736D6974206572726F720050BA
:20B280006F727420256420636F707065722072656365697665206572726F7200506F727415
:20B2A00020256420636F70706572207472616E736D6974206572726F7200506F7274202576
:20B2C0006420636F70706572206C696E6B20757000506F727420256420636F707065722077
:20B2E0006C696E6B20646F776E004447532D3132313654002825642900506F727420256477
:20B300000075C7AA75C755759D0275C7AA75C75575C600787FE4F6D8FD7550047551007546
:20B320008151D20D0200B35202026464E493A3F85407240CC8C333C4540F4420C883400414
:20B34000F456800146F6DFE4800C010204081020408090008028E47E019360CCA3FF543F09
:20B3600030E509541FFEE493A360010ECF54E0B4E02AE493FBA3E493FAA3E493F9A3E49341
:20B38000C083C082C0931200941BD093D082D083A309E970010ADFE6DEE480BA54C025E022
:20B3A000602B4088E493A3FAE493A3F8E493A3C8C582C8CAC583CA759308F0759300A3C8D4
:20B3C000C582C8CAC583CADFE3DEE18089E493A3F8E493A34003F68001F208DFF40200B390
:20B3E000560A454550524F4D2052656D61696E65642053697A653A2025640A00496E6974A4
:20B400002066696E69736865642E0A000A4D414320496C6C6567616C00456E746572204374
:20B420006865636B5F506B745F4C6F6F7021210A00696E6465782E68746D006C6566742E36
:20B4400068746D00746F702E68746D0062756C6C65742E67696600666F726D2E63737300C2
:20B460006C6F676F2E676966006D6F64656C2E676966002A67085C44656661756C74006127
:20B48000646D696E007075626C6963007072697661746500004D444C3A4447532D313231D4
:20B4A00036542D56332E30302E303000416C6C205265676973746572733A0A005B522530F9
:20B4C00032583A253034585D0048575F52657365745F506F72743A2532640A00EFB40A08B1
:20B4E000740D1200B4E8740A309811A899B8130CC2983098FDA899C298B811F63099FDC2AD
:20B5000099F5992246455F2564004762455F256400566C616E31007075626C6963002573C0
:20B5200020562573004447532D313231365400332E30302E31370010210D12008018BF0DC9
:20B54000027F0A0200B4DC900887F1E0FF22332E30302E313700256C6400300044656661D1
:20B56000756C7400E4FFFE120093CA600C0FEF70010E09E970F10A80EE22740000000000DC
:20B580000000000000000000000000004447532D3132313654000012233445FE25730044FA
:20B5A00047532D31323136540078947C6C7D097B817A9079787E007F0C1200934C90084E55
:20B5C00029E0FBA3E0FAA3E0F9120094FBFFAEF0E5F0600301CCCBEF14B40B00400301CC8E
:20B5E000CB9000B5F075F004A4C58325F0C583730200B61C0200B6490200BA9B0200BB82BB
:20B600000200C00C0200C2EC0200C6560200CA3C0200CC090200C4E90200CC9A9008754C3F
:20B620007487F0A37430F0A37437F0900847D6E0FBA3E0FAA3E0F91200A69A90084B26EED8
:20B64000F0A3EFF07F0101CCC49008754C7487F0A37431F0A37456F0900847D6E0FBA3E07B
:20B66000FAA3E0F91200A69A90084B26EEF0A3EFF0E490086C4FF0A3F090086C4FE475F043
:20B6800001120094CFAFF0FE600301B949EF14B40D00400301B9499000B6A675F004A4C569
:20B6A0008325F0C583730200B6DA0200B6F80200B7160200B7490200B7590200B76E0200E9
:20B6C000B7830200B7980200B7B60200B84C0200B8670200B8870200B8B490086C65748736
:20B6E000F0A37431F0A37473F078687C6C7D097B877A31798001B88090086C657487F0A384
:20B700007431F0A3748AF078687C6C7D097B877A31799B01B88090086C657487F0A374311F
:20B72000F0A374A3F09008754C7487F0A37431F0A374B4F0A3E4F0A37402F0A3E4F0A3049A
:20B74000F0A3E4F0A30401BA0890086C50E004F0700790086C4FE004F090086C657487F0FE
:20B76000A37431F0A374C1F012059DE5803D90086C657487F0A37431F0A374CCF012059D60
:20B78000F5802890086C657487F0A37431F0A374D8F012059E05801390086C657487F0A35D
:20B7A0007431F0A374E8F012059E1590086CA0120097E401B98A90086C657487F0A374312A
:20B7C000F0A374F0F07B097A6C7968120591B39008754C7487F0A37431F0A374FCF09008C5
:20B7E0006C68E0FF3395E09008754FE4F0A3EFF090086C69E0FF3395E090087551E4F0A373
:20B80000EFF090086C6AE0FF3395E090087553E4F0A3EFF090086C6BE0FF3395E09008759B
:20B8200055E4F0A3EFF090086C6CE0FF3395E090087557E4F0A3EFF090086C6DE0FF339594
:20B84000E090087559E4F0A3EF01BA0890086C657487F0A37432F0A3741AF01205A1857816
:20B86000687C6C7D09801990086C657487F0A37432F0A37426F01205A18C78687C6C7D090D
:20B8800012009ACC01BA1390086C657487F0A37432F0A37434F01205A09D9008754FEEF00C
:20B8A000A3EFF09008754C7487F0A37432F0A3744C01BA0890086C657487F0A37432F0A333
:20B8C000744FF090087F827409F0A3746CF0A374A6F0A37409F0A3746CF0A374A8F0A37446
:20B8E00009F0A3746CF0A374AAF07B097A6C79A4120575C79008754C7487F0A37432F0A331
:20B90000745DF090086CA4E0FFA3E09008754FCFF0A3EFF090086CA6E0FFA3E09008755155
:20B92000CFF0A3EFF090086CA8E0FFA3E090087553CFF0A3EFF090086CAAE0FFA3E090086F
:20B940007555CFF0A3EF01BA08900847D6E0FBA3E0FAA3E0F990084B26E0FEA3E0FFE92FFF
:20B96000F9EA3EFA9008754C7487F0A37432F0A37481F01200A69A90084B27E02FF09008B4
:20B980004B26E03EF07F0201CCC49008754C7487F0A37432F0A37493F090086CA0E0FCA3DC
:20B9A000E0FDA3E0FEA3E0FF7818120096E2E49008754FF0A3EFF090086CA0E0FCA3E0FDDB
:20B9C000A3E0FEA3E0FF7810120096E2E490087551F0A3EFF090086CA0E0FCA3E0FDA3E01B
:20B9E000FEA3E0FF7808120096E2E490087553F0A3EFF090086CA0E0FCA3E0FDA3A3E0FEE3
:20BA0000E490087555F0A3CEF07B097A6C79681200A69A7B097A6C79681200B564EF4E70CF
:20BA20001078687C6C7D097B877A32799F12009ACC900847D6E0FBA3E0FAA3E0F990084BFE
:20BA400026E0FEA3E0FFE92FF9EA3EFAC002C0019008754C7487F0A37432F0A374A6F090F0
:20BA6000086C65E0F9A3E0FAA3E09008754FC9F0A3EAF0A3E9F0A37409F0A3746CF0A3746C
:20BA800068F0D001D0021200A69A90084B27E02FF090084B26E03EF001B67990087B4EE0C8
:20BAA00070289008754C7487F0A37432F0A374C0F0900847D6E0FBA3E0FAA3E0F91200A669
:20BAC0009A90084B26EEF0A3EFF090084E34E0FBA3E0FAA3E0F9120094FB45F07054900843
:20BAE00047D6E0FBA3E0FAA3E0F990084B26E0FEA3E0FFE92FF9EA3EFA9008754C7487F075
:20BB0000A37432F0A374C2F01200A69A90084B27E02FF090084B26E03EF01204B84E9008FD
:20BB20004E34E0FBA3E0FAA3E0F9E475F00112009575E4FFFE12030D8FEF4E6042900847F9
:20BB4000D6E0FBA3E0FAA3E0F990084B26E0FEA3E0FFE92FF9EA3EFA9008754C7487F0A3B8
:20BB60007432F0A374D8F01200A69A90084B27E02FF090084B26E03EF07F03120586877FB9
:20BB8000002290087B4EE070289008754C7487F0A37432F0A374C0F0900847D6E0FBA3E053
:20BBA000FAA3E0F91200A69A90084B26EEF0A3EFF01205A0A6EF64014E600301BC5B900842
:20BBC0007B4EE07056900847D6E0FBA3E0FAA3E0F990084B26E0FEA3E0FFE92FF9EA3EFAD1
:20BBE0009008754C7487F0A37432F0A374EBF01200A69A90084B27E02FF090084B26E03E54
:20BC0000F090087B4E7401F090084E34E0FBA3E0FAA3E0F9E4F5F012009575E4FFFE1203A5
:20BC2000C11FEF4E6032900847D6E0FBA3E0FAA3E0F990084B26E0FEA3E0FFE92FF9EA3E2A
:20BC4000FA9008754C7487F0A37432F0A374D8F01200A69A120586777F002290087B4EE046
:20BC6000703F900847D6E0FBA3E0FAA3E0F990084B26E0FEA3E0FFE92FF9EA3EFA900875E3
:20BC80004C7487F0A37433F0A3740CF01200A69A90084B27E02FF090084B26E03EF001C7E6
:20BCA000DF90087B4EE0B40114E4FFFE1203EDE3EF4E7002FF2290087B4E7402F090087B2B
:20BCC0004EE06402600301BDBB900847D6E0FBA3E0FAA3E0F990084B26E0FEA3E0FFE92FEA
:20BCE000F9EA3EFA9008754C7487F0A37433F0A3744CF0C390086E8CE09401FE90086E8BFF
:20BD0000E094009008754FF0A3CEF01200A69A90084B27E02FF090084B26E03EF090086C8C
:20BD20004FE4F0A304F0C390086E8CE09401FF90086E8BE09400FE90086C4FE0FCA3E0FDCE
:20BD4000D39FEE6480F8EC6480985054900847D6E0FBA3E0FAA3E0F990084B26E0FEA3E0A8
:20BD6000FFE92FF9EA3EFA9008754C7487F0A37434F0A37403F0A3ECF0A3EDF01200A69AB7
:20BD800090084B27E02FF090084B26E03EF090086C50E004F0708F90086C4FE004F080862F
:20BDA00090087B4E7403F090084E34E0FBA3E0FAA3E0F9E475F0011200957590087B4EE026
:20BDC0006403600301C00790084E34E0FBA3E0FAA3E0F9120094FBC39401FFE5F09400FE84
:20BDE0007B097A6C795B12056F88EF4E7049900847D6E0FBA3E0FAA3E0F990084B26E0FE91
:20BE0000A3E0FFE92FF9EA3EFA9008754C7487F0A37432F0A374D8F01200A69A12058677AB
:20BE2000D390084B27E0940090084B26E09400500301C0077F0022900847D6E0FBA3E0FA6B
:20BE4000A3E0F990084B26E0FEA3E0FFE92FF9EA3EFA9008754C7487F0A37434F0A3741123
:20BE6000F090086C5BE0FFA3E09008754FCFF0A3EFF01200A69A90084B27E02FF090084B36
:20BE800026E03EF0E490086C53F0A3F0C390086E8CE09401FF90086E8BE09400FE90086CE0
:20BEA00053E0FCA3E0FDC39FEE6480F8EC648098400301BFDCEDAE047803CEA2E713CE13FB
:20BEC000D8F8FF90086C55EEF0A3EFF0ED5407FF90086C51E4F0A3EFF090086C56E0246129
:20BEE000F582E4346CF583759308E0FD7C0090086C52E0FF74017E00A807088005C333CE3E
:20BF000033CED8F9FFEE5CFEEF5D4E601190086C657487F0A37434F0A3743FF080509008C0
:20BF20006C56E0245DF582E4346CF583759308E0FD7C0090086C52E0FF74017E00A8070823
:20BF40008005C333CE33CED8F9FFEE5CFEEF5D4E90086C65600D7487F0A37434F0A3744191
:20BF6000F0800B7487F0A37432F0A3749FF0900847D6E0FBA3E0FAA3E0F990084B26E0FE0C
:20BF8000A3E0FFE92FF9EA3EFAC002C0019008754C7487F0A37434F0A37443F090086C6537
:20BFA000E0F9A3E0FAA3E09008754FC9F0A3EAF0A3E9F0D001D0021200A69A90084B27E0BB
:20BFC0002FF090084B26E03EF090086C54E004F0700790086C53E004F001BE8C90084E34F8
:20BFE000E0FBA3E0FAA3E0F9E475F00112009549C390084B27E0948490084B26E09403509E
:20C000000301BDC77F00227F0401CCC490087B4EE070289008754C7487F0A37432F0A37476
:20C02000C0F0900847D6E0FBA3E0FAA3E0F91200A69A90084B26EEF0A3EFF090087B4EE0CB
:20C0400070469008754C7487F0A37434F0A3744BF0900847D6E0FBA3E0FAA3E0F91200A618
:20C060009A90084B26EEF0A3EFF090084E34E0FBA3E0FAA3E0F9E475F001120095759008D1
:20C080007B4E7401F001C2E990087B4EE06401600301C2E990086C51F0A3F0E490086C90C1
:20C0A000F090086C52E0FF7B097A6C79571205887F90086C52E0FF12059E55EF60087B876B
:20C0C0007A35790880067B877A35791090087551EBF0A3EAF0A3E9F0900847D6E0FBA3E02B
:20C0E000FAA3E0F990084B26E0FEA3E0FFE92FF9EA3EFA9008754C7487F0A37434F0A37498
:20C10000CAF090086C52E02401FE90086C51E034009008754FF0A3CEF01200A69A90084BC1
:20C1200027E02FF090084B26E03EF090086C52E025E0FF90086C51E033FE749E2FF58274F6
:20C14000783EF583759308E0FEA3E0C39401FFEE940090086C4FF0A3EFF090086C52E02547
:20C16000E0FF90086C51E033FE74AE2FF58274783EF583759308E0FEA3E0FF90086C4FE06D
:20C18000FCA3E0FDC39FEE6480F8EC648098400301C23EEDAE047803CEA2E713CE13D8F816
:20C1A0002457F582746C3EF583759308E0FD7C0090086C50E05407FF74017E00A8070880D6
:20C1C00005C333CE33CED8F9FFEE5CFEEF5D4E605A90086C907401F0900847D6E0FBA3E01D
:20C1E000FAA3E0F990084B26E0FEA3E0FFE92FF9EA3EFA9008754C7487F0A37435F0A37496
:20C2000019F090086C50E02401FE90086C4FE034009008754FF0A3CEF01200A69A90084B75
:20C2200027E02FF090084B26E03EF090086C50E004F0700790086C4FE004F001C15A900847
:20C240006C90E0703C900847D6E0FBA3E0FAA3E0F990084B26E0FEA3E0FFE92FF9EA3EFA31
:20C260009008754C7487F0A37435F0A3741FF01200A69A90084B27E02FF090084B26E03E96
:20C28000F090086C52E004F0700790086C51E004F0C390086C52E0940290086C51E064803C
:20C2A0009480500301C09B900847D6E0FBA3E0FAA3E0F990084B26E0FEA3E0FFE92FF9EACE
:20C2C0003EFA9008754C7487F0A37432F0A374D8F01200A69A90084B27E02FF090084B2666
:20C2E000E03EF07F05120586877F002290087B4EE070289008754C7487F0A37432F0A3747A
:20C30000C0F0900847D6E0FBA3E0FAA3E0F91200A69A90084B26EEF0A3EFF090088181741B
:20C3200009F0A3746CF0A37493F0A37409F0A3746CF0A37491F07B097A6C7992E4FF12056D
:20C3400074A49008754C7487F0A37435F0A37423F090086C91E075F003A42494F582E43453
:20C360006CF583759308E0F9A3E0FAA3E09008754FC9F0A3EAF0A3E9F0900847D6E0FBA3AF
:20C38000E0FAA3E0F91200A69A90084B26EEF0A3EFF090086C91E0701278687C6C7D097BCC
:20C3A000877A32799F12009ACC802A9008754C7487F0A37435F0A374C5F090086C92E0044A
:20C3C000FFF09008754FE4F0A3EFF07B097A6C79681200A69A900847D6E0FBA3E0FAA3E08F
:20C3E000F990084B26E0FEA3E0FFE92FF9EA3EFA9008754C7487F0A37435F0A374CAF0A3B4
:20C400007409F0A3746CF0A37468F01200A69A90084B27E02FF090084B26E03EF090086C57
:20C4200091E0701278687C6C7D097B877A32799F12009ACC802A9008754C7487F0A3743543
:20C44000F0A374C5F090086C93E004FFF09008754FE4F0A3EFF07B097A6C79681200A69A67
:20C46000900847D6E0FBA3E0FAA3E0F990084B26E0FEA3E0FFE92FF9EA3EFA9008754C74CA
:20C4800087F0A37435F0A374FBF0A37409F0A3746CF0A37468F01200A69A90084B27E02F8A
:20C4A000F090084B26E03EF0900847D6E0FBA3E0FAA3E0F990084B26E0FEA3E0FFE92FF972
:20C4C000EA3EFA9008754C7487F0A37432F0A374D8F01200A69A90084B27E02FF090084BA0
:20C4E00026E03EF07F0601CCC490087B4EE070289008754C7487F0A37432F0A374C0F09045
:20C500000847D6E0FBA3E0FAA3E0F91200A69A90084B26EEF0A3EFF01205A14DEF6003010F
:20C52000C5BC90087B4EE07043900847D6E0FBA3E0FAA3E0F990084B26E0FEA3E0FFE92F7C
:20C54000F9EA3EFA9008754C7487F0A37436F0A3742BF01200A69A90084B27E02FF090081A
:20C560004B26E03EF090087B4E7401F0E4FFFE1203A897EF4E6042900847D6E0FBA3E0FA55
:20C58000A3E0F990084B26E0FEA3E0FFE92FF9EA3EFA9008754C7487F0A37432F0A374D817
:20C5A000F01200A69A90084B27E02FF090084B26E03EF07F0A120586877F002290087B4E6A
:20C5C000E07043900847D6E0FBA3E0FAA3E0F990084B26E0FEA3E0FFE92FF9EA3EFA90080B
:20C5E000754C7487F0A37436F0A3744BF01200A69A90084B27E02FF090084B26E03EF090FE
:20C60000087B4E7401F0E4FFFE12043902EF4E6042900847D6E0FBA3E0FAA3E0F990084B67
:20C6200026E0FEA3E0FFE92FF9EA3EFA9008754C7487F0A37432F0A374D8F01200A69A9003
:20C64000084B27E02FF090084B26E03EF07F0A120586877F002290087B4EE0702890087516
:20C660004C7487F0A37432F0A374C0F0900847D6E0FBA3E0FAA3E0F91200A69A90084B269F
:20C68000EEF0A3EFF090087B4EE0600301C7E99008754C7487F0A37436F0A3746CF0900859
:20C6A00047D6E0FBA3E0FAA3E0F91200A69A90084B26EEF0A3EFF07B097A6C79901205A0A4
:20C6C0009490086C90E07041900847D6E0FBA3E0FAA3E0F990084B26E0FEA3E0FFE92FF99E
:20C6E000EA3EFA9008754C7487F0A37436F0A37492F01200A69A90084B27E02FF090084BC0
:20C7000026E03EF07F0701CCC412059FE0C007C00612059FEAC007C00612059FF4C007C04D
:20C720000612059FFE90087555EEF0A3EFF090087553D0E0F0A3D0E0F090087551D0E0F03C
:20C74000A3D0E0F09008754FD0E0F0A3D0E0F0900847D6E0FBA3E0FAA3E0F990084B26E0E5
:20C76000FEA3E0FFE92FF9EA3EFA9008754C7487F0A37436F0A374F3F01200A69A90084B56
:20C7800027E02FF090084B26E03EF0900847D6E0FBA3E0FAA3E0F990084B26E0FEA3E0FF6A
:20C7A000E92FF9EA3EFA9008754C7487F0A37437F0A374DFF01200A69A90084B27E02FF083
:20C7C00090084B26E03EF012053DAE90084E34E0FBA3E0FAA3E0F9E475F00112009575905C
:20C7E000087B4E7401F07F002278A47C6C7D097B817A9079847E007F121200934C90084EEF
:20C8000034E0FBA3E0FAA3E0F9120094FBFFC390086E8CE09401FD90086E8BE09400FCC3E5
:20C82000EF9DE5F09C400301C9FB900847D6E0FBA3E0FAA3E0F990084B26E0FEA3E0FFE918
:20C840002FF9EA3EFA9008754C7487F0A37438F0A37434F01200A69A90084B27E02FF090E5
:20C86000084B26E03EF0E490086C4FF0A3F090084E34E0FBA3E0FAA3E0F9120094FBFFAE3B
:20C88000F0C390086E8CE09401FD90086E8BE09400FCD3EF9DEE9C400301C982C3EF940121
:20C8A000FF7B097A6C79A01205991F90084E34E0FBA3E0FAA3E0F9120094FBC39401FF7BC6
:20C8C000097A6C79A212059B3390084E34E0FBA3E0FAA3E0F9120094FBC39401FF7B097A85
:20C8E0006C79A312059BFF900847D6E0FBA3E0FAA3E0F990084B26E0FEA3E0FFE92FF9EA12
:20C900003EFAC003C002C0019008754C7487F0A37438F0A37448F090084E34E0FBA3E0FA55
:20C92000A3E0F9120094FBFF9008754FE5F0F0A3EFF090086CA0E0FFA3E090087551CFF015
:20C94000A3EFF090086CA2E0FF90087553E4F0A3EFF090086CA3E075F003A424A4F582E464
:20C96000346CF583759308E0F9A3E0FAA3E090087555C9F0A3EAF0A3E9F0D001D002D0032C
:20C98000802A900847D6E0FBA3E0FAA3E0F990084B26E0FEA3E0FFE92FF9EA3EFA900875BB
:20C9A0004C7487F0A37438F0A3746FF01200A69A90084B27E02FF090084B26E03EF0900881
:20C9C0004E34E0FBA3E0FAA3E0F9E475F0011200954990086C50E004F0700790086C4FE0F5
:20C9E00004F0C390086C50E0940490086C4FE064809480500301C86E7F0022900847D6E0C9
:20CA0000FBA3E0FAA3E0F990084B26E0FEA3E0FFE92FF9EA3EFA9008754C7487F0A37432F9
:20CA2000F0A374D8F01200A69A90084B27E02FF090084B26E03EF07F0701CCC490087B4E3D
:20CA4000E070289008754C7487F0A37432F0A374C0F0900847D6E0FBA3E0FAA3E0F912007F
:20CA6000A69A90084B26EEF0A3EFF09008754C7487F0A37438F0A37486F0900847D6E0FB6D
:20CA8000A3E0FAA3E0F91200A69A90084B26EEF0A3EFF01205A0EE90086C90EFF0E0702C4E
:20CAA000900847D6E0FBA3E0FAA3E0F990084B26E0FEA3E0FFE92FF9EA3EFA9008754C7484
:20CAC00087F0A37438F0A3749C01CBF190084E34E0FBA3E0FAA3E0F9E4F5F01200957590CD
:20CAE0000847D6E0FBA3E0FAA3E0F990084B26E0FEA3E0FFE92FF9EA3EFA9008754C74874D
:20CB0000F0A37438F0A374FEF01200A69A90084B27E02FF090084B26E03EF0E4FDFCFFFE95
:20CB200012036F0F90084E34E0FBA3E0FAA3E0F9E4F5F012009575900847D6E0FBA3E0FA82
:20CB4000A3E0F990084B26E0FEA3E0FFE92FF9EA3EFA9008754C7487F0A37439F0A374140E
:20CB6000F01200A69A90084B27E02FF090084B26E03EF0E4FDFCFFFE1203403812059A3B00
:20CB80009008754FEBF0A3EAF0A3E9F0900847D6E0FBA3E0FAA3E0F990084B26E0FEA3E072
:20CBA000FFE92FF9EA3EFA9008754C7487F0A37439F0A37425F01200A69A90084B27E02F28
:20CBC000F090084B26E03EF0900847D6E0FBA3E0FAA3E0F990084B26E0FEA3E0FFE92FF94B
:20CBE000EA3EFA9008754C7487F0A37432F0A374D8F01200A69A90084B27E02FF090084B79
:20CC000026E03EF07F0801CCC490087B4EE070289008754C7487F0A37432F0A374C0F0901B
:20CC20000847D6E0FBA3E0FAA3E0F91200A69A90084B26EEF0A3EFF01205A0DCEF4E600808
:20CC40007B877A3979B780067B877A3079249008754FEBF0A3EAF0A3E9F0900847D6E0FB60
:20CC6000A3E0FAA3E0F990084B26E0FEA3E0FFE92FF9EA3EFA9008754C7487F0A37439F09B
:20CC8000A3742AF01200A69A90084B27E02FF090084B26E03EF07F09802A9008754C74876B
:20CCA000F0A37439F0A374BEF0900847D6E0FBA3E0FAA3E0F91200A69A90084B26EEF0A31A
:20CCC000EFF07F0B120586877F00227F0122EF6402600301CF0F90084B26F0A3F090084B7E
:20CCE00023E0FBA3E0FAA3E02415F9E43AFA120093CAB4075390084B23A3E0FAA3E024162F
:20CD0000F9E43AFA7401120093FFD39405500301E2B690084B23A3E0FAA3E02415F9E43A3B
:20CD2000FAE41200941B90086F8AE0FCA3E0FDA3E0FEA3E02401FFE43EFEE43DFDE43CFCE5
:20CD400090086F8A020097E490084B23E0FBA3E0FAA3E02415F9E43AFA120093CAB4052052
:20CD600090084B23A3E0FAA3E02416F9E43AFA7401120093FFD39405500301E2B601CF0819
:20CD800090084B23E0FBA3E0FAA3E02415F9E43AFA120093CAFF700301E2B620E40301CE18
:20CDA000B490084B23A3E0FAA3E02416F9E43AFA74FF120093FF600301E2B6120511CD90D6
:20CDC000084B23E0FBA3E0FAA3E02417F9E43AFA7401120093E06405705990084B23E0FBA9
:20CDE000A3E0FAA3E02415F9E43AFAE41200941B90086F8AE0FCA3E0FDA3E0FEA3E024012E
:20CE0000FFE43EFEE43DFDE43CFC90086F8A120097E490084A3E7480F0900847D9E0FBA361
:20CE2000E0FAA3E0240DF9E43AFA74141200941B01DDAA90084B23E0FBA3E0FAA3E0241568
:20CE4000F9E43AFA120093CA540F14700301D86524FE603014700301DCE324FE700301DCBF
:20CE6000E324FE700301DCE32406600301E2B6900847D9E0FBA3E0FAA3E0240DF9E43AFA7F
:20CE8000E401D87890084A3E7404F090086F9AE0FCA3E0FDA3E0FEA3E02401FFE43EFEE4AC
:20CEA0003DFDE43CFC90086F9A120097E41205880F01DED090084B23E0FBA3E0FAA3E0248C
:20CEC00015F9E43AFA120093CA540F6403600301E2B690084B23A3E0FAA3E02416F9E43AA0
:20CEE000FA74FF120093FF600301E2B690084B23A3E0FAA3E02417F9E43AFA7401120093B9
:20CF0000E06405600301E2B6120511CD01CDDA90086EB3E0FBA3E0FAA3E0F990084B26E0B9
:20CF2000FEA3E0FFE92FF9EA3EFAE41200941B90084B237409F0A3744AF0A37449F09008ED
:20CF40006EB3E0FBA3E0FAA3E0F9900847D3EBF0A3EAF0A3E9F0240EF9E43AFA900847DF55
:20CF6000EBF0A3EAF0A3E9F01204B018EF6401600301D07790086E6FE0700301D050120500
:20CF80009B1C9008855BEFF075F005A424F5F582E43444F583759308E09008855BF0900821
:20CFA0006EB3E0FBA3E0FAA3E0F990084B20EBF0A3EAF0A3E9F02411F9E43AFA120094FBBE
:20CFC00045F0600301E2B690084B20E0FBA3E0FAA3E02413F9E43AFA120093CA600301E245
:20CFE000B690084B20E0FBA3E0FAA3E02414F9E43AFA120093CA703490084B20A3E0FAA31E
:20D00000E02415F9E43AFA120093CAFF64806010EF6481600BEF64016006EF600301E2B640
:20D020009008855BE0FF1204A921804B90084B20E0FBA3E0FAA3E02414F9E43AFA12009322
:20D04000CAB480339008855BE0FF12058B8B80271205A169BF012090086EB3E0FBA3E0FA62
:20D06000A3E0F990084B20EBF0A3EAF0A3E9F07D347C0012022AE2900847D3E0FBA3E0FA06
:20D08000A3E0240CF9E43AFA120094FBFFAEF0BE0807BF06040204772590086448E0FCA393
:20D0A000E0FDA3E0FEA3E02401FFE43EFEE43DFDE43CFC90086448120097E4900847D3E0AE
:20D0C000FBA3E0FAA3E0240CF9E43AFA120094FB7004E5F06408602190086458E0FCA3E08A
:20D0E000FDA3E0FEA3E02401FFE43EFEE43DFDE43CFC9008645801D236900847DFE0FBA318
:20D10000E0FAA3E02402F9E43AFA120094FBFFAEF090084B26EEF0A3EFF0D394DCEE94050A
:20D1200040219008644CE0FCA3E0FDA3E0FEA3E02401FFE43EFEE43DFDE43CFC9008644C20
:20D1400001D236900847DFE0FBA3E0FAA3E0F9120093CA644560219008644CE0FCA3E0FDF7
:20D16000A3E0FEA3E02401FFE43EFEE43DFDE43CFC9008644C01D236E92406F9E43AFA12A6
:20D180000094FBE5F0543F602190086484E0FCA3E0FDA3E0FEA3E02401FFE43EFEE43DFDD5
:20D1A000E43CFC9008648401D23612059DE5900847DFE0FBA3E0FAA3E02410F9E43AFA1241
:20D1C00000975DC3120096D16042900847DFE0FBA3E0FAA3E02410F9E43AFA12009708747A
:20D1E000FFFBFAF9F8C3120096D1602090086450E0FCA3E0FDA3E0FEA3E02401FFE43EFE9E
:20D20000E43DFDE43CFC90086450802A1204997DEFF47002EEF460259008644CE0FCA3E04F
:20D22000FDA3E0FEA3E02401FFE43EFEE43DFDE43CFC9008644C120097E401DA20900847C0
:20D24000DFE0FBA3E0FAA3E0240CF9E43AFA12009708900847D3E0FBA3E0FAA3E02406F972
:20D26000E43AFA12043B1690086460E0FCA3E0FDA3E0FEA3E02401FFE43EFEE43DFDE43CF1
:20D28000FC90086460120097E4900847DFE0FBA3E0FAA3E02409F9E43AFA120093CA6401FE
:20D2A0007053120093CAFF90084B23E0FBA3E0FAA3E02414F9E43AFAEF1200941B90084784
:20D2C000DFE0FBA3E0FAA3E0240CF9E43AFA1200970890084B23E0FBA3E0FAA3E02404F9A0
:20D2E000E43AFA120097257B817A9079001200A6A0020553BD900847DFE0FBA3E0FAA3E0C1
:20D300002409F9E43AFA120093CA6411600301D42190087A0FE0FCA3E0FDA3E0FEA3E024ED
:20D3200001FFE43EFEE43DFDE43CFC90087A0F120097E4900847DFE0FBA3E0FAA3E0241414
:20D34000F9E43AFA900847DCEBF0A3EAF0A3E9F090086EB3E0FBA3E0FAA3E0F912055CE647
:20D36000900847DFE0FBA3E0FAA3E02409F9E43AFA120093CAFF90084B23E0FBA3E0FAA367
:20D38000E02414F9E43AFAEF1200941B900847DCE0FBA3E0FAA3E02402F9E43AFA12009441
:20D3A000FBFF90084B23E0FBA3E0FAA3E0F9E5F08FF012009575900847DCE0FBA3E0FAA373
:20D3C000E0F9120094FBFF90084B23E0FBA3E0FAA3E02402F9E43AFAE5F08FF0120095754C
:20D3E000900847DFE0FBA3E0FAA3E0240CF9E43AFA1200970890084B23E0FBA3E0FAA3E0C1
:20D400002404F9E43AFA1200972590084B23E0FBA3E0FAA3E0F9120094FBFFAEF002051ACC
:20D4200087900847DFE0FBA3E0FAA3E02409F9E43AFA120093CA64066043E4FFFEFDFC90A8
:20D44000086460E0F8A3E0F9A3E0FAA3E0FBD3120096D1402590086460E0FCA3E0FDA3E0C5
:20D46000FEA3E024FFFFEE34FFFEED34FFFDEC34FFFC90086460120097E401DA20900847EF
:20D48000DFE0FBA3E0FAA3E02414F9E43AFA900847D9EBF0A3EAF0A3E9F090086F92E0FC88
:20D4A000A3E0FDA3E0FEA3E02401FFE43EFEE43DFDE43CFC90086F92120097E41205A0305D
:20D4C000900847D9E0FBA3E0FAA3E02402F9E43AFA120094FB6F7003EE65F0600301DA205E
:20D4E00090088559E4F0A304F090088559E0FEA3E0FFC39405EE9400400301D5C77C007DBE
:20D500002B1200942F74492FF9744A3EFA7B0990084B23EBF0A3EAF0A3E9F02415F9E43A82
:20D52000FA120093CA700301D5B4900847D9E0FBA3E0FAA3E02402F9E43AFA120094FBFF1B
:20D54000AEF090084B23E0FBA3E0FAA3E0F9120094FB6F7003EE65F0705AE92402F9E43A9D
:20D56000FA120094FBFFAEF0900847D9E0FBA3E0FAA3E0F9120094FBB50739E5F0B506348D
:20D5800090084B23E0FBA3E0FAA3E02404F9E43AFA12009708900847DFE0FBA3E0FAA3E027
:20D5A000240CF9E43AFA1200975DC3120096D1700301D97B9008855AE004F0700790088541
:20D5C00059E004F001D4E9900847D9E0FBA3E0FAA3E0240DF9E43AFA120093CA6402600353
:20D5E00001DA2090088559E4F0A304F090088559E0FEA3E0FFC39405EE9400502D90084A3C
:20D600005E75F02BEF12009801EE75F02BA42583F583759308E0605E9008855AE004F070D7
:20D62000CB90088559E004F080C290088559E4F0A304F090088559E0FEA3E0FFC39405EE92
:20D640009400502F90084A5E75F02BEF12009801EE75F02BA42583F583759308E064076050
:20D66000159008855AE004F070C990088559E004F080C001DA2090088559E0FEA3E0FF7C3A
:20D68000007D2B1200942F74492FF9744A3EFA90084B237409F0A3EAF0A3E9F0900847DF08
:20D6A000E0FBA3E0FAA3E02409F9E43AFA120093CAFF90084B23E0FBA3E0FAA3E02414F9D1
:20D6C000E43AFAEF1200941B90084B23E0FBA3E0FAA3E02416F9E43AFA74021200941B908F
:20D6E000084B23E0FBA3E0FAA3E02417F9E43AFAE41200941B900847D9E0FBA3E0FAA3E055
:20D700002402F9E43AFA120094FBFF90084B23E0FBA3E0FAA3E0F9E5F08FF0120095759058
:20D720000847D9E0FBA3E0FAA3E0F9120094FBFF90084B23E0FBA3E0FAA3E02402F9E43A2F
:20D74000FAE5F08FF012009575900847DFE0FBA3E0FAA3E0240CF9E43AFA1200970890083C
:20D760004B23E0FBA3E0FAA3E02404F9E43AFA1200972590084B23E0FBA3E0FAA3E024153F
:20D78000F9E43AFA74111200941B90086F82E0FCA3E0FDA3E0FEA3E02401FFE43EFEE43DE4
:20D7A000FDE43CFC90086F82120097E490084A45E0FCA3E0FDA3E0FEA3E0FF90084B23E0CE
:20D7C000FBA3E0FAA3E0240CF9E43AFA12009725EF2401FFE43EFEE43DFDE43CFC90084BEF
:20D7E00023E0FBA3E0FAA3E02410F9E43AFA12009725900847D9E0FBA3E0FAA3E02404F964
:20D80000E43AFA12009708EF2401FFE43EFEE43DFDE43CFC90084B23E0FBA3E0FAA3E024CD
:20D8200008F9E43AFA1200972590084B23E0FBA3E0FAA3E02422F9E43AFAC003C002C00183
:20D8400090084B23A3E0FAA3E02420F9E43AFA900884DEEBF0A3EAF0A3E9F0D001D002D02C
:20D8600003120578B3900847D9E0FBA3E0FAA3E0240DF9E43AFA74101200941B900847D991
:20D88000E0FBA3E0FAA3E0240DF9E43AFA120093CA44021200941B900847D9E0FBA3E0FAE5
:20D8A000A3E02414F9E43AFA9008855CEBF0A3EAF0A3E9F074021200941B9008855CE0FBC4
:20D8C000A3E0FAA3E02401F9E43AFA74041200941B9008855CE0FBA3E0FAA3E02402F9E482
:20D8E0003AFA74051200941B9008855CE0FBA3E0FAA3E02403F9E43AFA74781200941B90F1
:20D9000008855CE0FBA3E0FAA3E02404F9E43AFA74011200941B9008855CE0FBA3E0FAA360
:20D92000E02405F9E43AFA74011200941B9008855CE0FBA3E0FAA3E02406F9E43AFA740490
:20D940001200941B9008855CE0FBA3E0FAA3E02407F9E43AFA74021200941B90084B26E452
:20D96000F0A37430F0900847D9E0FBA3E0FAA3E0240CF9E43AFA747001E17FE490084A3E63
:20D98000F0900847D9E0FBA3E0FAA3E0240DF9E43AFA120093CA30E26F90084B23E0FBA34E
:20D9A000E0FAA3E02415F9E43AFA120093CAB4012290086F86E0FCA3E0FDA3E0FEA3E02469
:20D9C00001FFE43EFEE43DFDE43CFC90086F86120097E4E41200941B90086F8AE0FCA3E03E
:20D9E000FDA3E0FEA3E02401FFE43EFEE43DFDE43CFC90086F8A120097E490084A3E7420D6
:20DA0000F01205880F01E041900847D9E0FBA3E0FAA3E0240DF9E43AFA120093CA20E403FB
:20DA200001E041900847D9E0FBA3E0FAA3E0240CF9E43AFA120093CAC4540F75F004A4FF4E
:20DA4000AEF090088559EEF0A3EFF02414FFE43EFEC390084B27E09FFF90084B26E09EFE2B
:20DA6000F0A3EFF0D39400EE9400403490084B23E0FBA3E0FAA3E02408F9E43AFA12009710
:20DA800008900847D9E0FBA3E0FAA3E02404F9E43AFA1200975DC3120096D1600301E14BE0
:20DAA00090084B23E0FBA3E0FAA3E02410F9E43AFA12009708900847D9E0FBA3E0FAA3E0FC
:20DAC0002408F9E43AFA1200975DC3120096D1706690084B23E0FBA3E0FAA3E02410F9E4FF
:20DAE0003AFA1200970890084B23A3E0FAA3E0240CF9E43AFA1200972590084B23E0FBA3A8
:20DB0000E0FAA3E02415F9E43AFA120093CAFF30E42590084A3E7401F0EF54EF1200941B3F
:20DB200090084B23E0FBA3E0FAA3E02416F9E43AFA74021200941B90084B23E0FBA3E0FA24
:20DB4000A3E02415F9E43AFA120093CA540F14B40800400301E1479000DB6675F004A4C547
:20DB60008325F0C583730200DB860200DBA20200DC250200DF5C0200E0440200E112020013
:20DB8000E14B0200DF1690084A3EE030E01174031200941B90084A3E7440F01205880F0196
:20DBA000E04190084A3EE030E078900847D9E0FBA3E0FAA3E0240DF9E43AFA120093CA6414
:20DBC00012705F90084B23E0FBA3E0FAA3E02415F9E43AFA74031200941B900847D9E0FB6E
:20DBE000A3E0FAA3E02404F9E43AFA1200970890084B23E0FBA3E0FAA3E02408F9E43AFA1D
:20DC00001200972512009708EF2401FFE43EFEE43DFDE43CFC1200972574421205880201F2
:20DC2000DD5301E04190086F8EE0FCA3E0FDA3E0FEA3E02401FFE43EFEE43DFDE43CFC908F
:20DC4000086F8E120097E4900847D9E0FBA3E0FAA3E0240DF9E43AFA120093CA20E00301EA
:20DC6000DCE690084B27E02401FF90084B26E03400FEE4FCFD90084B23E0FBA3E0FAA3E0FB
:20DC80002408F9E43AFA1200972574101205880290084B23E0FBA3E0FAA3E02410F9E43A28
:20DCA000FA12009708EF2401FFE43EFEE43DFDE43CFC1200972590084B23E0FBA3E0FAA37D
:20DCC000E02415F9E43AFA74181200941B90084B23E0FBA3E0FAA3E02417F9E43AFAE412AA
:20DCE00000941B01DE2AD390084B27E0940090084B26E09400404590084A3EE04402F09053
:20DD0000084B23E0FBA3E0FAA3E02408F9E43AFAC003C002C0011200975D90084B26E0FE42
:20DD2000A3E0FFE4FCFDEB2FFFEA3EFEED39FDEC38FCD001D002D0031200972590084A3E9E
:20DD4000E05403700301DF131205880FEF4E700301E14B90084A3EE030E57490084B23E02C
:20DD6000FBA3E0FAA3E02415F9E43AFAE41200941B900847D9E0FBA3E0FAA3E0240DF9E418
:20DD80003AFA74141200941B90086F8AE0FCA3E0FDA3E0FEA3E02401FFE43EFEE43DFDE4CF
:20DDA0003CFC90086F8A120097E490086FA2E0FCA3E0FDA3E0FEA3E02401FFE43EFEE43D9F
:20DDC000FDE43CFC90086FA2120097E401E16290084A3EE030E46990084B23E0FBA3E0FAD5
:20DDE000A3E02410F9E43AFA12009708EF2401FFE43EFEE43DFDE43CFC1200972590084B8C
:20DE000023E0FBA3E0FAA3E02415F9E43AFA74141200941B90084B23E0FBA3E0FAA3E0246C
:20DE200017F9E43AFAE41200941B900847D9E0FBA3E0FAA3E0240DF9E43AFA741101E15E7B
:20DE4000D390084B27E0940090084B26E09400407790084B23E0FBA3E0FAA3E02415F9E446
:20DE60003AFA120093CA20E45F120093CA44101200941B90084B23E0FBA3E0FAA3E02417FC
:20DE8000F9E43AFAE41200941B90084B23E0FBA3E0FAA3E02410F9E43AFAC003C002C00160
:20DEA0001200975D90084B26E0FEA3E0FFE4FCFDEB2FFFEA3EFEED39FDEC38FCD001D002F1
:20DEC000D003120097258008E490084B26F0A3F0D390084B27E0940090084B26E09400508B
:20DEE0000890084A3EE030E12A90084B27E02428F090084B26E03400F0900847D9E0FBA376
:20DF0000E0FAA3E0240DF9E43AFA74181200941B01E16C01E04190084A3EE020E00301E1C0
:20DF20004790084B23E0FBA3E0FAA3E02415F9E43AFAE41200941B90086F8AE0FCA3E0FDDD
:20DF4000A3E0FEA3E02401FFE43EFEE43DFDE43CFC90086F8A120097E401E147D390084B42
:20DF600027E0940090084B26E09400403D90084B23E0FBA3E0FAA3E02408F9E43AFAC0032B
:20DF8000C002C0011200975D90084B26E0FEA3E0FFE4FCFDEB2FFFEA3EFEED39FDEC38FC30
:20DFA000D001D002D00312009725900847D9E0FBA3E0FAA3E0240DF9E43AFA120093CA30A9
:20DFC000E04990084A3EE090084B2330E027E0FBA3E0FAA3E02415F9E43AFA740712009495
:20DFE0001B90084B23E0FBA3E0FAA3E02416F9E43AFAE4800FE0FBA3E0FAA3E02415F9E476
:20E000003AFA74161200941B01E0D790084A3EE030E01A90084B23E0FBA3E0FAA3E0241585
:20E02000F9E43AFA74051200941B01E147D390084B27E0940090084B26E09400400301E179
:20E040004B01E147D390084B27E0940090084B26E09400403D90084B23E0FBA3E0FAA3E020
:20E060002408F9E43AFAC003C002C0011200975D90084B26E0FEA3E0FFE4FCFDEB2FFFEACE
:20E080003EFEED39FDEC38FCD001D002D00312009725900847D9E0FBA3E0FAA3E0240DF900
:20E0A000E43AFA120093CA30E05590084B23E0FBA3E0FAA3E02415F9E43AFA740712009428
:20E0C0001B90084B23E0FBA3E0FAA3E02416F9E43AFAE41200941B90084B23E0FBA3E0FAF6
:20E0E000A3E02408F9E43AFA12009708EF2401FFE43EFEE43DFDE43CFC12009725804CD3D5
:20E1000090084B27E0940090084B26E09400503B803590084A3EE030E02D90084B23E0FBA6
:20E12000A3E0FAA3E02415F9E43AFA74071200941B90084B23E0FBA3E0FAA3E02416F9E461
:20E140003AFAE41200941B0205A259900847D9E0FBA3E0FAA3E0240DF9E43AFA7410120079
:20E16000941B90084B26E4F0A37428F0900847D9E0FBA3E0FAA3E0240CF9E43AFA7450123A
:20E1800000941B90084B23E0FBA3E0FAA3E02408F9E43AFA12009708900847D9E0FBA3E0EB
:20E1A000FAA3E02408F9E43AFA1200972590084B23E0FBA3E0FAA3E0240CF9E43AFA1200A3
:20E1C0009708900847D9E0FBA3E0FAA3E02404F9E43AFA1200972590084B23E0FBA3E0FAA8
:20E1E000A3E0F9120094FBFF900847D9E0FBA3E0FAA3E0F9E5F08FF01200957590084B2301
:20E20000E0FBA3E0FAA3E02402F9E43AFA120094FBFF900847D9E0FBA3E0FAA3E02402F99A
:20E22000E43AFAE5F08FF012009575900847D9E0FBA3E0FAA3E0240EF9E43AFA740575F0A2
:20E24000781200957590086F96E0FCA3E0FDA3E0FEA3E02401FFE43EFEE43DFDE43CFC901F
:20E26000086F96120097E490086F96E0FCA3E0FDA3E0FEA3E0FFA3E0F8A3E0F9A3E0FAA3F1
:20E28000E0FBC3EF9BFFEE9AFEED99FDEC98FC90086F96120097E47F027E001202D8B69073
:20E2A000084B23E0FBA3E0FAA3E02416F9E43AFA74021200941B229000FFFD1200991EEB29
:20E2C000F0A3EAF0A3E9F09000FF911200991E1205A0EEEF4E7005FEFF01F86390000075B7
:20E2E00012009945E0FBA3E0FAA3E0F9120094FBFDACF0C3940FEC64809480500301F85A30
:20E300009000007212009945E0FBA3E0FAA3E0F9C003C002C001C3ED9401FDEC9400FC90A3
:20E3200000006F12009945E0F9A3E0FAA3E090087FE4C9F0A3EAF0A3E9F09000006F1200E7
:20E340009945E0FBA3E0FAA3E02434F9E43AFA120094FBC39401FEE5F0940090087FE7F04D
:20E36000A3CEF0D001D002D0031204F42AEF4E600301F85A7C007D029000007512009945AF
:20E38000E0FBA3E0FAA3E0F9120094FB25E0FFE5F033FE9000007212009945E0FBA3E0FAB4
:20E3A000A3E02FF9EA3EFAC3E99DF9EA9CFA120094FBFFAEF0855083855182759308EEF0F2
:20E3C000A3EFF0855083855182759308E0FEA3E0FFC39401EE64809480400BD3EF9402EECC
:20E3E00064809480400301F85A85508385518275930874FFF5F0120094CF9000006F1200F1
:20E400009945E0FBA3E0FAA3E02437F9E43AFA120094FBFFAEF0E5F0600301F85AEF24FEFD
:20E42000B40C00400301F85A9000E43775F004A4C58325F0C583730200E4670200E4CF02B2
:20E4400000E62E0200E8180200E9490200EA7A0200EBAF0200EC210200ED2B0200EE5C02F9
:20E4600000EFEE0200F1801205510E9000007B12009945E0FEA3E0FF900000781200994583
:20E48000E0FBA3E0FAA3E0F9C003C002C0017B099000000F12009945A982AA83A801AC02A0
:20E4A000AD03D001D002D0031200934C855083855182759308E0FEA3E0FF7B099000000F02
:20E4C00012009945A982AA831203AED001F8639000007812009945E0FBA3E0FAA3E0F91227
:20E4E000043D26BEFF06BFFF0301F8549000007812009945E0FBA3E0FAA3E0F91200970867
:20E50000855083855182759308E0FAA3E0FB900864EF75F02912009801EA75F029A42583FB
:20E52000F583759308120097E4900864F575F029EB12009801EA75F029A42583F58375936D
:20E5400008E0FEA3E064014E600301F860855083855182A3A3759308F0A3F085508385512C
:20E5600082A3A3759308E0FEA3E0C39402EE64809480400301E603855083855182A3A3758B
:20E580009308A3E0FD7F027E0012057256C001855083855182759308E0FEA3E0FF7C007DA8
:20E5A000291200942F74CE2FF974643EA801FC7D09D00112009A22EF7033855083855182D1
:20E5C000A3A3759308A3E0FF120598C69000007812009945E0FBA3E0FAA3E0F91200975D1C
:20E5E000C3120096D17006FE7F0301F863855083855182A3A3759308E475F001120094CFC8
:20E6000001E55B9000007812009945E0FBA3E0FAA3E0F9120097088550838551827593087C
:20E62000A3E090088650F0120598E401F84E1205A0A6EF4E600301E7169000007812009971
:20E6400045E0FBA3E0FAA3E0F912009708E47B01FAF9F8D3120096D15022900000781200CD
:20E660009945E0FBA3E0FAA3E0F912009708E47BFE7A0FF9F8C3120096D1500301F85485FF
:20E680005083855182A3A3759308E4F0A3F0855083855182A3A3759308E0FEA3E0FFC394D5
:20E6A00040EE6480948050527B099000006512009945A982AA8312056F88EF4E602790006F
:20E6C000007812009945E0FBA3E0FAA3E0F9120097089000006512009945E0FCA3E06F702A
:20E6E00002EC6E6015855083855182A3A3759308E475F001120094CF8094855083855182C0
:20E70000A3A3759308E0FEA3E0C39440EE64809480402601F8549000007812009945E0FB3F
:20E72000A3E0FAA3E0F912009708E4FBFAF9F8C3120096D1600301F8548550838551827554
:20E740009308E0FEA3E0900864F375F02912009801EE75F029A42583F583759308E4F0A3CE
:20E76000F01205A0A6EF4E703D9000007812009945E0FBA3E0FAA3E0F9120097088550838D
:20E78000855182759308E0FCA3E0900864F375F02912009801EC75F029A42583F583759344
:20E7A00008EEF0A3EFF0855083855182759308E0FEA3E0900864F575F02912009801EE7543
:20E7C000F029A42583F583759308E0FEA3E064014E600301F860855083855182759308A319
:20E7E000E0FDE4FFFE12059AEC1205A0A6EF4E70249000007812009945E0FBA3E0FAA3E0BD
:20E80000F912009708855083855182759308A3E0FD12059AEC01F84E855083855182759372
:20E8200008E0FEA3E0900864E375F02912009801EE75F029A42583F583759308E0FCA3E0A8
:20E84000FDA3E0FEA3E0FF9000006112009945120097E49000007812009945E0FBA3E0FAFA
:20E86000A3E0F912009708120098D5E87B00000001E895000000020000E8BC900000611262
:20E88000009945C083C082E0FCA3E0FDA3E0FEA3E0440180189000006112009945C083C0F4
:20E8A00082E0FCA3E0FDA3E0FEA3E054FEFFEC759308D082D083120097E4800301F8549097
:20E8C00000006112009945E0FCA3E0FDA3E0FEA3E0FF855083855182759308E0FAA3E0FB70
:20E8E000900864E375F02912009801EA75F029A42583F583759308120097E4900864F575C1
:20E90000F029EB12009801EA75F029A42583F583759308E0FEA3E064014E600301F860909C
:20E9200000006112009945E0FCA3E0FDA3E0FEA3E0FF855083855182759308A3E0900886C6
:20E9400041F01205983001F84E855083855182759308E0FEA3E0900864EB75F02912009820
:20E9600001EE75F029A42583F583759308E0FCA3E0FDA3E0FEA3E0FF900000611200994506
:20E98000120097E49000007812009945E0FBA3E0FAA3E0F912009708120098D5E9AC000059
:20E9A0000001E9C6000000020000E9ED9000006112009945C083C082E0FCA3E0FDA3E0FE8C
:20E9C000A3E0440180189000006112009945C083C082E0FCA3E0FDA3E0FEA3E054FEFFECD4
:20E9E000759308D082D083120097E4800301F8549000006112009945E0FCA3E0FDA3E0FE47
:20EA0000A3E0FF855083855182759308E0FAA3E0FB900864EB75F02912009801EA75F029C4
:20EA2000A42583F583759308120097E4900864F575F029EB12009801EA75F029A42583F5A7
:20EA400083759308E0FEA3E064014E600301F8609000006112009945E0FCA3E0FDA3E0FE95
:20EA6000A3E0FF855083855182759308A3E09008864BF0120598A801F84E8550838551822A
:20EA8000759308E0FEA3E0900864E775F02912009801EE75F029A42583F583759308E0FCBD
:20EAA000A3E0FDA3E0FEA3E0FF9000006112009945120097E49000007812009945E0FBA3EF
:20EAC000E0FAA3E0F912009708120098D5EADD00000001EAF7000000020000EB1E9000006C
:20EAE0006112009945C083C082E0FCA3E0FDA3E0FEA3E0440280189000006112009945C061
:20EB000083C082E0FCA3E0FDA3E0FEA3E054FDFFEC759308D082D083120097E4800301F8D6
:20EB2000549000006112009945E0FCA3E0FDA3E0FEA3E0FF855083855182759308E0FAA304
:20EB4000E0FB900864E775F02912009801EA75F029A42583F583759308120097E4900864E9
:20EB6000F575F029EB12009801EA75F029A42583F583759308E0FEA3E064014E600301F5C3
:20EB8000859000006112009945E0FCA3E0FDA3E0FEA3E0FF855083855182759308A3E090DD
:20EBA000088646F01205986C120588FB01F585855083855182A3A3759308E4F0A3F0C390A1
:20EBC000086E8CE09401FF90086E8BE09400FE855083855182A3A3759308E0FCA3E0C39FF5
:20EBE000EE6480F8EC6480985034855083855182A3A3759308A3E0FF12059BE990000006A6
:20EC000012009945EEF0A3EFF0855083855182A3A3759308E475F001120094CF80A001F8C6
:20EC20005A855083855182759308E0FEA3E0900864EB75F02912009801EE75F029A4258371
:20EC4000F583759308E0FCA3E0FDA3E0FEA3E0FF9000006112009945120097E49000007857
:20EC600012009945E0FBA3E0FAA3E0F912009708120098D5EC8400000001EC9E00000002A3
:20EC80000000ECC59000006112009945C083C082E0FCA3E0FDA3E0FEA3E04402801890008F
:20ECA000006112009945C083C082E0FCA3E0FDA3E0FEA3E054FDFFEC759308D082D083121B
:20ECC0000097E4800301F8549000006112009945E0FCA3E0FDA3E0FEA3E0FF85508385517B
:20ECE00082759308E0FAA3E0FB900864EB75F02912009801EA75F029A42583F583759308BE
:20ED0000120097E4900864F575F029EB12009801EA75F029A42583F583759308E0FEA3E0A4
:20ED200064014E600301F86001EE32855083855182759308E0FEA3E0900864EB75F029129B
:20ED4000009801EE75F029A42583F583759308E0FCA3E0FDA3E0FEA3E0FF90000061120068
:20ED60009945120097E49000007812009945E0FBA3E0FAA3E0F912009708120098D5ED8EB1
:20ED800000000001EDA8000000020000EDCF9000006112009945C083C082E0FCA3E0FDA3BA
:20EDA000E0FEA3E0440480189000006112009945C083C082E0FCA3E0FDA3E0FEA3E054FBFD
:20EDC000FFEC759308D082D083120097E4800301F8549000006112009945E0FCA3E0FDA356
:20EDE000E0FEA3E0FF855083855182759308E0FAA3E0FB900864EB75F02912009801EA751C
:20EE0000F029A42583F583759308120097E4900864F575F029EB12009801EA75F029A42522
:20EE200083F583759308E0FEA3E064014E600301F8609000006112009945E0FCA3E0FDA317
:20EE4000E0FEA3E0FF855083855182759308A3E09008864BF0120598A801F84E855083853B
:20EE60005182A3A3759308E4F0A3F0C390086E8CE09401FF90086E8BE09400FE8550838559
:20EE80005182A3A3759308E0FCA3E0C39FEE6480F8EC648098400301EFEB85508385518288
:20EEA000A3A3759308A3E0FF12059BE99000000612009945EEF0A3EFF085508385518275D4
:20EEC0009308E0FEA3E0900864E775F02912009801EE75F029A42583F583759308E0FCA34B
:20EEE000E0FDA3E0FEA3E0FF9000006112009945120097E49000007812009945E0FBA3E06E
:20EF0000FAA3E0F912009708120098D5EF1C00000001EF36000000020000EF5D90000061DB
:20EF200012009945C083C082E0FCA3E0FDA3E0FEA3E0440480189000006112009945C083F8
:20EF4000C082E0FCA3E0FDA3E0FEA3E054FBFFEC759308D082D083120097E4800301F854C3
:20EF60009000006112009945E0FCA3E0FDA3E0FEA3E0FF855083855182759308E0FAA3E034
:20EF8000FB900864E775F02912009801EA75F029A42583F583759308120097E4900864F590
:20EFA00075F029EB12009801EA75F029A42583F583759308E0FEA3E064014E702B900000A2
:20EFC0006112009945E0FCA3E0FDA3E0FEA3E0FF855083855182759308A3E090088646F0EA
:20EFE0001205986C120588FB01F58501F85A855083855182A3A3759308E4F0A3F0C39008C6
:20F000006E8CE09401FF90086E8BE09400FE855083855182A3A3759308E0FCA3E0C39FEECA
:20F020006480F8EC648098400301F17D855083855182A3A3759308A3E0FF12059BE9900027
:20F04000000612009945EEF0A3EFF0855083855182759308E0FEA3E0900864E775F02912B6
:20F06000009801EE75F029A42583F583759308E0FCA3E0FDA3E0FEA3E0FF90000061120045
:20F080009945120097E49000007812009945E0FBA3E0FAA3E0F912009708120098D5F0AE6B
:20F0A00000000001F0C8000000020000F0EF9000006112009945C083C082E0FCA3E0FDA351
:20F0C000E0FEA3E0440880189000006112009945C083C082E0FCA3E0FDA3E0FEA3E054F7DA
:20F0E000FFEC759308D082D083120097E4800301F8549000006112009945E0FCA3E0FDA333
:20F10000E0FEA3E0FF855083855182759308E0FAA3E0FB900864E775F02912009801EA75FC
:20F12000F029A42583F583759308120097E4900864F575F029EB12009801EA75F029A425FF
:20F1400083F583759308E0FEA3E064014E702B9000006112009945E0FCA3E0FDA3E0FEA394
:20F16000E0FF855083855182759308A3E090088646F01205986C120588FB01F58501F85A96
:20F180009000007812009945E0FBA3E0FAA3E0F9120097089000000812009945120097E4DD
:20F1A0009000000812009945E0FCA3E0FDA3E0FEA3E0FF120098D5F1D900000001F33E00ED
:20F1C000000002F3CF00000004F3D200000005F504000000060000F3CF1205510E7B099052
:20F1E00000000F12009945A982AA831200B564EF4E601D7B099000000F12009945A982AAEB
:20F20000831200B564D3EF9414EE64809480400301F8549000003612009945E4F0A304F03F
:20F220007B099000000F12009945A982AA83C001855083855182759308E0FEA3E0FF7C0006
:20F240007D291200942F74CE2FF974643EA801FC7D09D0017E007F291200934C7B0990008C
:20F26000000F12009945A982AA83855083855182759308A3E09008859AF07D027C0012053B
:20F2800069F59000002412009945E0FCA3E0FDA3E0FEA3E0FF855083855182759308A3E0CA
:20F2A00090088641F0120598309000002812009945E0FCA3E0FDA3E0FEA3E0FF855083853C
:20F2C0005182759308A3E090088646F01205986C9000002C12009945E0FCA3E0FDA3E0FED0
:20F2E000A3E0FF855083855182759308A3E09008864BF0120598A89000003012009945E009
:20F30000FCA3E0FDA3E0FEA3E0FF855083855182759308A3E090088650F0120598E49000AA
:20F32000003412009945E0FEA3E0FF855083855182759308A3E0FD12059AEC01F84E855050
:20F3400083855182759308E0FEA3E0900864F575F02912009801EE75F029A42583F5837582
:20F360009308E0FCA3E0FD64024C7005FEFF01F863ED64034C7055855083855182759308F1
:20F38000E0FEA3E0FF7C007D291200942F74CE2FF974643EFA7B091200B564EF4E602D859E
:20F3A0005083855182759308E0FEA3E0900864F575F02912009801EE75F029A42583F58347
:20F3C000759308E4F0A37402F001F86001F85401F854855083855182A3A3759308E4F0A3D0
:20F3E000F0855083855182A3A3759308E0FEA3E0FFC39402EE64809480502190000038122D
:20F40000055120EF4E6015855083855182A3A3759308E475F001120094CF80C585508385DD
:20F420005182A3A3759308E0FEA3E0FF4E700E855083855182759308F0A3F08044C3EF942A
:20F4400001FFEE9400FE855083855182759308E0FCA3E0D39FEE6480F8EC648098401F8585
:20F460005083855182A3A3759308E0FFA3E0855083855182759308CFF0A3EFF0800301F82C
:20F48000547E007F297D007B099000003812009945A982AA8312009C8A9000005F1200990F
:20F4A00045E4F0A37403F07B099000003812009945A982AA83A801AC02AD037B817A80791F
:20F4C0000B12009ACC7B099000003812009945A982AA83C001855083855182759308E0FEB6
:20F4E000A3E0FF7C007D291200942F74CE2FF974643EA801FC7D09D0017E007F291200934C
:20F500004C01F860855083855182A3A3759308E4F0A3F0855083855182A3A3759308E0FEF5
:20F52000A3E0FFC39402EE64809480501D1205511CEF4E6015855083855182A3A375930861
:20F54000E475F001120094CF80C9855083855182A3A3759308E0FCA3E0FD4C7005FEFF0182
:20F56000F863C3ED9401FFEC9400FE855083855182759308E0FCA3E0FDD39FEE6480F8EC2A
:20F58000648098400301F860900864F575F029ED12009801EC75F029A42583F583759308EE
:20F5A000E4F0A3F07B817A80790B855083855182759308A3E09008859AF07D027C0012056E
:20F5C00069F5855083855182A3A3759308E4F0A3F0855083855182A3A3759308E0FEA3E0F9
:20F5E000C39402EE64809480400301F84E855083855182A3A3759308A3E0FD7F027E0012AB
:20F600000572569000000C12009945EBF0A3EAF0A3E9F09000000C12009945E0FBA3E0FAD9
:20F62000A3E0F91200B564EF4E600301F838855083855182A3A3759308E0FEA3E02401FFC7
:20F64000E43EFEC3EF9402EE64809480400301F8389000000412009945EEF0A3EFF0900074
:20F66000000412009945E0FEA3E0C39402EE64809480400301F8389000000412009945A35B
:20F68000E0FD7F027E00120572569000000C12009945EBF0A3EAF0A3E9F09000000C1200A1
:20F6A0009945E0FBA3E0FAA3E0F91200B564EF4E700301F8259000000C12009945E0FBA395
:20F6C000E0FAA3E0F9855083855182A3A3759308A3E09008859AF07D027C00120569F590A4
:20F6E00000000412009945A3E0FF120598C6855083855182A3A3759308A3E090088650F038
:20F70000120598E49000000412009945A3E0FF12059B04855083855182A3A3759308A3E011
:20F72000FD12059AEC9000000412009945A3E0FF12059812855083855182A3A3759308A3BF
:20F74000E090088641F0120598309000000412009945A3E0FF1205984E855083855182A345
:20F76000A3759308A3E090088646F01205986C9000000412009945A3E0FF1205988A8550D0
:20F7800083855182A3A3759308A3E09008864BF0120598A87B817A80790B900000041200E5
:20F7A0009945A3E09008859AF07D027C00120569F5E4FFFEFDFC9000000412009945A3E0F0
:20F7C00090088650F0120598E49000000412009945A3E0FDE4FFFE12059AECE4FFFEFDFCDC
:20F7E0009000000412009945A3E090088641F012059830E4FFFEFDFC900000041200994576
:20F80000A3E090088646F01205986CE4FFFEFDFC9000000412009945A3E09008864BF012AA
:20F820000598A880139000000412009945E475F001120094CF01F65E855083855182A3A362
:20F84000759308E475F001120094CF01F5D1120588FB800C7E007F0380097E007F028003E1
:20F86000E4FEFF9000007D0200991E9000FFFD1200991EEBF0A3EAF0A3E9F09000FFC51252
:20F8800000991E1205A0EEEF4E7005FEFF01FFDA9000004112009945E0FBA3E0FAA3E0F9EE
:20F8A000120094FBFDACF0C3940FEC64809480500301FFD19000003E12009945E0FBA3E084
:20F8C000FAA3E0F9C003C002C001C3ED9401FDEC9400FC9000003B12009945E0F9A3E0FA9D
:20F8E000A3E090087FE4C9F0A3EAF0A3E9F09000003B12009945E0FBA3E0FAA3E02434F9F1
:20F90000E43AFA120094FBC39401FEE5F0940090087FE7F0A3CEF0D001D002D0031204F4A0
:20F920002AEF4E600301FFD17C007D029000004112009945E0FBA3E0FAA3E0F9120094FBFB
:20F9400025E0FFE5F033FE9000003E12009945E0FBA3E0FAA3E02FF9EA3EFAC3E99DF9EA8E
:20F960009CFA120094FBFFAEF0855083855182759308EEF0A3EFF0855083855182759308D3
:20F98000E0FEA3E0FFC39401EE64809480400BD3EF9402EE64809480400301FFD1855083D4
:20F9A00085518275930874FFF5F0120094CF9000003B12009945E0FBA3E0FAA3E02437F928
:20F9C000E43AFA120094FBFFAEF0E5F0600301FFD1EF24FD700301FA5B04600301FFD17E39
:20F9E000007F177D007B099000000D12009945A982AA8312009C8A9000004712009945E0AC
:20FA0000FEA3E0FF9000004412009945E0FBA3E0FAA3E0F9C003C002C0017B099000000D67
:20FA200012009945A982AA83A801AC02AD03D001D002D0031200934C855083855182759358
:20FA400008E0FEA3E0FF7B099000000D12009945A982AA8312046CA501FFDA9000004412EE
:20FA6000009945E0FBA3E0FAA3E0F9120097089000000612009945120097E4900000061268
:20FA8000009945E0FCA3E0FDA3E0FEA3E0FF120098D5FAB400000001FB7100000002FC028F
:20FAA00000000004FC0500000005FD1F000000060000FC02855083855182759308E0FEA3DB
:20FAC000E0FF12055D637B099000000D12009945A982AA831200B564EF4E700301FFCB7BE6
:20FAE000099000000D12009945A982AA831200B564D3EF9414EE64809480400301FFCB90FF
:20FB000000002212009945E4F0A304F07B099000000D12009945A982AA83C0018550838561
:20FB20005182759308E0FEA3E0FF7C007D171200942F74942FF974643EA801FC7D09D0015B
:20FB40007E007F171200934C7B099000000D12009945A982AA83855083855182759308A3D4
:20FB6000E09008859AF07D017C00120569F501FFC5855083855182759308E0FEA3E0900811
:20FB800064A975F01712009801EE75F017A42583F583759308E0FCA3E0FD64024C7005FE72
:20FBA000FF01FFDAED64034C7055855083855182759308E0FEA3E0FF7C007D171200942F02
:20FBC00074942FF974643EFA7B091200B564EF4E602D855083855182759308E0FEA3E090BB
:20FBE0000864A975F01712009801EE75F017A42583F583759308E4F0A37402F001FFD701D6
:20FC0000FFCB01FFCB855083855182A3A3759308E4F0A3F0855083855182A3A3759308E0FC
:20FC2000FEA3E0FFC39402EE6480948050219000002412055D67EF4E6015855083855182A3
:20FC4000A3A3759308E475F001120094CF80C5855083855182A3A3759308E0FEA3E0FF4E96
:20FC6000700E855083855182759308F0A3F08044C3EF9401FFEE9400FE8550838551827514
:20FC80009308E0FCA3E0D39FEE6480F8EC648098401F855083855182A3A3759308E0FFA3DF
:20FCA000E0855083855182759308CFF0A3EFF0800301FFCB9000003912009945E4F0A37471
:20FCC00003F07B099000002412009945A982AA83A801AC02AD037B817A80790B12009ACCB8
:20FCE0007B099000002412009945A982AA83C001855083855182759308E0FEA3E0FF7C0027
:20FD00007D171200942F74942FF974643EA801FC7D09D0017E007F171200934C01FFD785D7
:20FD20005083855182A3A3759308E4F0A3F0855083855182A3A3759308E0FEA3E0C394021B
:20FD4000EE64809480505E855083855182A3A3759308A3E0FD7F027E0012057256C0018565
:20FD60005083855182759308E0FEA3E0FF7C007D171200942F74942FF974643EA801FC7D9B
:20FD800009D00112009A22EF7006FE7F0301FFDA855083855182A3A3759308E475F001129A
:20FDA0000094CF8089855083855182A3A3759308E4F0A3F0855083855182A3A3759308E084
:20FDC000FEA3E0FFC39402EE64809480501D12055D63EF4E6015855083855182A3A3759370
:20FDE00008E475F001120094CF80C9855083855182A3A3759308E0FCA3E0FD4C7005FEFFD3
:20FE000001FFDAC3ED9401FFEC9400FE855083855182759308E0FCA3E0FDD39FEE6480F8EE
:20FE2000EC648098400301FFD7900864A975F017ED12009801EC75F017A42583F583759353
:20FE400008E4F0A3F07B817A80790B855083855182759308A3E09008859AF07D017C0012C3
:20FE60000569F5855083855182A3A3759308E4F0A3F0855083855182A3A3759308E0FEA32B
:20FE8000E0C39402EE64809480400301FFC5855083855182A3A3759308A3E0FD7F017E00B7
:20FEA000120572569000000A12009945EBF0A3EAF0A3E9F09000000A12009945E0FBA3E01D
:20FEC000FAA3E0F91200B564EF4E600301FFAF855083855182A3A3759308E0FEA3E02401A6
:20FEE000FFE43EFEC3EF9402EE64809480400301FFAF9000000412009945EEF0A3EFF0904F
:20FF000000000412009945E0FEA3E0C39402EE64809480400301FFAF9000000412009945D7
:20FF2000A3E0FD7F017E00120572569000000A12009945EBF0A3EAF0A3E9F09000000A125A
:20FF4000009945E0FBA3E0FAA3E0F91200B564EF4E60499000000A12009945E0FBA3E0FAFC
:20FF6000A3E0F9855083855182A3A3759308A3E09008859AF07D017C00120569F57B817AF0
:20FF800080790B9000000412009945A3E09008859AF07D017C00120569F580139000000419
:20FFA00012009945E475F001120094CF01FEFF855083855182A3A3759308E475F001120032
:20FFC00094CF01FE72120588FB800C7E007F0380097E007F028003E4FEFF90000049020060
:20FFE000991E74E090087729F0A3F0900877217480F0A3E4F090087727F0A37402F080FE03
:020000040001F9
:20000000E4900887CCF02290087A25EBF0A3EAF0A3E9F01200970890087A2B120097E4E990
:200020002404F9E43AFA1200970890087A2F120097E490087A25E0FBA3E0FAA3E02408F9D1
:20004000E43AFA1200970890087A33120097E490087A25E0FBA3E0FAA3E0240CF9E43AFAB2
:200060001200970890087A37120097E490087A2BE0F8A3E0F9A3E0FAA3E0FBC000C001C02C
:2000800002C00390087A37E0FCA3E0FDA3E0FEA3E0FF90087A33E0F8A3E0F9A3E0FAA3E05A
:2000A0006FFFEA6EFEE96DFDE86CFC90087A2FE0F8A3E0F9A3E0FAA3E05FFFEA5EFEE95D5A
:2000C000FDE85CFC90087A37E0F8A3E0F9A3E0FAA3E06FFFEA6EFEE96DFDE86CFC90087ACD
:2000E00028E0FBA3E0FAA3E0F91200975DEF2BFFEE3AFEED39FDEC38FCEF2478FFEE34A42C
:20010000FEED346AFDEC34D7FCD003D002D001D000EB2FFFEA3EFEE93DFDE83CFC90087A8C
:200120002B120097E490087A2BE0FCA3E0FDA3E0FEA3E0FF7807120096F5C004C005C00600
:20014000C00790087A2BE0FCA3E0FDA3E0FEA3E0FF7819120096E2D003D002D001D000EFEC
:200160004BFFEE4AFEED49FDEC48FC90087A2B120097E490087A2BE0FCA3E0FDA3E0FEA315
:20018000E0FFA3E0F8A3E0F9A3E0FAA3E0FBEF2BFFEE3AFEED39FDEC38FC90087A2B1200BD
:2001A00097E490087A37E0F8A3E0F9A3E0FAA3E0FBC000C001C002C00390087A33E0FCA362
:2001C000E0FDA3E0FEA3E0FF90087A2FE0F8A3E0F9A3E0FAA3E06FFFEA6EFEE96DFDE86C3F
:2001E000FC90087A2BE0F8A3E0F9A3E0FAA3E05FFFEA5EFEE95DFDE85CFC90087A33E0F82E
:20020000A3E0F9A3E0FAA3E06FFFEA6EFEE96DFDE86CFC90087A28E0FBA3E0FAA3E02404BE
:20022000F9E43AFA1200975DEF2BFFEE3AFEED39FDEC38FCEF2456FFEE34B7FEED34C7FD01
:20024000EC34E8FCD003D002D001D000EB2FFFEA3EFEE93DFDE83CFC90087A37120097E4FC
:2002600090087A37E0FCA3E0FDA3E0FEA3E0FF780C120096F5C004C005C006C00790087A8D
:2002800037E0FCA3E0FDA3E0FEA3E0FF7814120096E2D003D002D001D000EF4BFFEE4AFEFD
:2002A000ED49FDEC48FC90087A37120097E490087A37E0FCA3E0FDA3E0FEA3E0FF90087A4B
:2002C0002BE0F8A3E0F9A3E0FAA3E0FBEF2BFFEE3AFEED39FDEC38FC90087A37120097E44C
:2002E00090087A33E0F8A3E0F9A3E0FAA3E0FBC000C001C002C00390087A2FE0FCA3E0FDC7
:20030000A3E0FEA3E0FF90087A2BE0F8A3E0F9A3E0FAA3E06FFFEA6EFEE96DFDE86CFC9052
:20032000087A37E0F8A3E0F9A3E0FAA3E05FFFEA5EFEE95DFDE85CFC90087A2FE0F8A3E0ED
:20034000F9A3E0FAA3E06FFFEA6EFEE96DFDE86CFC90087A28E0FBA3E0FAA3E02408F9E41F
:200360003AFA1200975DEF2BFFEE3AFEED39FDEC38FCEF24DBFFEE3470FEED3420FDEC34E6
:2003800024FCD003D002D001D000EB2FFFEA3EFEE93DFDE83CFC90087A33120097E490080B
:2003A0007A33E0FCA3E0FDA3E0FEA3E0FF7811120096F5C004C005C006C00790087A33E0D0
:2003C000FCA3E0FDA3E0FEA3E0FF780F120096E2D003D002D001D000EF4BFFEE4AFEED49A2
:2003E000FDEC48FC90087A33120097E490087A33E0FCA3E0FDA3E0FEA3E0FFA3E0F8A3E05C
:20040000F9A3E0FAA3E0FBEF2BFFEE3AFEED39FDEC38FC90087A33120097E490087A2FE073
:20042000F8A3E0F9A3E0FAA3E0FBC000C001C002C00390087A2BE0FCA3E0FDA3E0FEA3E0AA
:20044000FF90087A37E0F8A3E0F9A3E0FAA3E06FFFEA6EFEE96DFDE86CFC90087A33E0F87C
:20046000A3E0F9A3E0FAA3E05FFFEA5EFEE95DFDE85CFC90087A2BE0F8A3E0F9A3E0FAA328
:20048000E06FFFEA6EFEE96DFDE86CFC90087A28E0FBA3E0FAA3E0240CF9E43AFA12009716
:2004A0005DEF2BFFEE3AFEED39FDEC38FCEF24EEFFEE34CEFEED34BDFDEC34C1FCD003D014
:2004C00002D001D000EB2FFFEA3EFEE93DFDE83CFC90087A2F120097E490087A2FE0FCA369
:2004E000E0FDA3E0FEA3E0FF7816120096F5C004C005C006C00790087A2FE0FCA3E0FDA39B
:20050000E0FEA3E0FF780A120096E2D003D002D001D000EF4BFFEE4AFEED49FDEC48FC90C7
:20052000087A2F120097E490087A2FE0FCA3E0FDA3E0FEA3E0FFA3E0F8A3E0F9A3E0FAA3C6
:20054000E0FBEF2BFFEE3AFEED39FDEC38FC90087A2F120097E490087A2BE0F8A3E0F9A33C
:20056000E0FAA3E0FBC000C001C002C00390087A37E0FCA3E0FDA3E0FEA3E0FF90087A3330
:20058000E0F8A3E0F9A3E0FAA3E06FFFEA6EFEE96DFDE86CFC90087A2FE0F8A3E0F9A3E088
:2005A000FAA3E05FFFEA5EFEE95DFDE85CFC90087A37E0F8A3E0F9A3E0FAA3E06FFFEA6E34
:2005C000FEE96DFDE86CFC90087A28E0FBA3E0FAA3E02410F9E43AFA1200975DEF2BFFEE13
:2005E0003AFEED39FDEC38FCEF24AFFFEE340FFEED347CFDEC34F5FCD003D002D001D0009F
:20060000EB2FFFEA3EFEE93DFDE83CFC90087A2B120097E490087A2BE0FCA3E0FDA3E0FE74
:20062000A3E0FF7807120096F5C004C005C006C00790087A2BE0FCA3E0FDA3E0FEA3E0FF6A
:200640007819120096E2D003D002D001D000EF4BFFEE4AFEED49FDEC48FC90087A2B120018
:2006600097E490087A2BE0FCA3E0FDA3E0FEA3E0FFA3E0F8A3E0F9A3E0FAA3E0FBEF2BFF58
:20068000EE3AFEED39FDEC38FC90087A2B120097E490087A37E0F8A3E0F9A3E0FAA3E0FB8F
:2006A000C000C001C002C00390087A33E0FCA3E0FDA3E0FEA3E0FF90087A2FE0F8A3E0F9FB
:2006C000A3E0FAA3E06FFFEA6EFEE96DFDE86CFC90087A2BE0F8A3E0F9A3E0FAA3E05FFFC4
:2006E000EA5EFEE95DFDE85CFC90087A33E0F8A3E0F9A3E0FAA3E06FFFEA6EFEE96DFDE899
:200700006CFC90087A28E0FBA3E0FAA3E02414F9E43AFA1200975DEF2BFFEE3AFEED39FDAB
:20072000EC38FCEF242AFFEE34C6FEED3487FDEC3447FCD003D002D001D000EB2FFFEA3EE8
:20074000FEE93DFDE83CFC90087A37120097E490087A37E0FCA3E0FDA3E0FEA3E0FF780C56
:20076000120096F5C004C005C006C00790087A37E0FCA3E0FDA3E0FEA3E0FF7814120096EA
:20078000E2D003D002D001D000EF4BFFEE4AFEED49FDEC48FC90087A37120097E490087A77
:2007A00037E0FCA3E0FDA3E0FEA3E0FF90087A2BE0F8A3E0F9A3E0FAA3E0FBEF2BFFEE3AD6
:2007C000FEED39FDEC38FC90087A37120097E490087A33E0F8A3E0F9A3E0FAA3E0FBC000AE
:2007E000C001C002C00390087A2FE0FCA3E0FDA3E0FEA3E0FF90087A2BE0F8A3E0F9A3E0FF
:20080000FAA3E06FFFEA6EFEE96DFDE86CFC90087A37E0F8A3E0F9A3E0FAA3E05FFFEA5EB1
:20082000FEE95DFDE85CFC90087A2FE0F8A3E0F9A3E0FAA3E06FFFEA6EFEE96DFDE86CFC3B
:2008400090087A28E0FBA3E0FAA3E02418F9E43AFA1200975DEF2BFFEE3AFEED39FDEC38AA
:20086000FCEF2413FFEE3446FEED3430FDEC34A8FCD003D002D001D000EB2FFFEA3EFEE971
:200880003DFDE83CFC90087A33120097E490087A33E0FCA3E0FDA3E0FEA3E0FF78111200ED
:2008A00096F5C004C005C006C00790087A33E0FCA3E0FDA3E0FEA3E0FF780F120096E2D012
:2008C00003D002D001D000EF4BFFEE4AFEED49FDEC48FC90087A33120097E490087A33E0D9
:2008E000FCA3E0FDA3E0FEA3E0FFA3E0F8A3E0F9A3E0FAA3E0FBEF2BFFEE3AFEED39FDEC39
:2009000038FC90087A33120097E490087A2FE0F8A3E0F9A3E0FAA3E0FBC000C001C002C03E
:200920000390087A2BE0FCA3E0FDA3E0FEA3E0FF90087A37E0F8A3E0F9A3E0FAA3E06FFF0D
:20094000EA6EFEE96DFDE86CFC90087A33E0F8A3E0F9A3E0FAA3E05FFFEA5EFEE95DFDE836
:200960005CFC90087A2BE0F8A3E0F9A3E0FAA3E06FFFEA6EFEE96DFDE86CFC90087A28E00D
:20098000FBA3E0FAA3E0241CF9E43AFA1200975DEF2BFFEE3AFEED39FDEC38FCEF2401FF70
:2009A000EE3495FEED3446FDEC34FDFCD003D002D001D000EB2FFFEA3EFEE93DFDE83CFC3D
:2009C00090087A2F120097E490087A2FE0FCA3E0FDA3E0FEA3E0FF7816120096F5C004C0FA
:2009E00005C006C00790087A2FE0FCA3E0FDA3E0FEA3E0FF780A120096E2D003D002D00143
:200A0000D000EF4BFFEE4AFEED49FDEC48FC90087A2F120097E490087A2FE0FCA3E0FDA326
:200A2000E0FEA3E0FFA3E0F8A3E0F9A3E0FAA3E0FBEF2BFFEE3AFEED39FDEC38FC90087AD0
:200A40002F120097E490087A2BE0F8A3E0F9A3E0FAA3E0FBC000C001C002C00390087A37FF
:200A6000E0FCA3E0FDA3E0FEA3E0FF90087A33E0F8A3E0F9A3E0FAA3E06FFFEA6EFEE96D64
:200A8000FDE86CFC90087A2FE0F8A3E0F9A3E0FAA3E05FFFEA5EFEE95DFDE85CFC90087A3B
:200AA00037E0F8A3E0F9A3E0FAA3E06FFFEA6EFEE96DFDE86CFC90087A28E0FBA3E0FAA30F
:200AC000E02420F9E43AFA1200975DEF2BFFEE3AFEED39FDEC38FCEF24D8FFEE3498FEEDCA
:200AE0003480FDEC3469FCD003D002D001D000EB2FFFEA3EFEE93DFDE83CFC90087A2B12A9
:200B00000097E490087A2BE0FCA3E0FDA3E0FEA3E0FF7807120096F5C004C005C006C0078C
:200B200090087A2BE0FCA3E0FDA3E0FEA3E0FF7819120096E2D003D002D001D000EF4BFF7F
:200B4000EE4AFEED49FDEC48FC90087A2B120097E490087A2BE0FCA3E0FDA3E0FEA3E0FF96
:200B6000A3E0F8A3E0F9A3E0FAA3E0FBEF2BFFEE3AFEED39FDEC38FC90087A2B120097E437
:200B800090087A37E0F8A3E0F9A3E0FAA3E0FBC000C001C002C00390087A33E0FCA3E0FD16
:200BA000A3E0FEA3E0FF90087A2FE0F8A3E0F9A3E0FAA3E06FFFEA6EFEE96DFDE86CFC90A6
:200BC000087A2BE0F8A3E0F9A3E0FAA3E05FFFEA5EFEE95DFDE85CFC90087A33E0F8A3E04D
:200BE000F9A3E0FAA3E06FFFEA6EFEE96DFDE86CFC90087A28E0FBA3E0FAA3E02424F9E45B
:200C00003AFA1200975DEF2BFFEE3AFEED39FDEC38FCEF24AFFFEE34F7FEED3444FDEC34BE
:200C20008BFCD003D002D001D000EB2FFFEA3EFEE93DFDE83CFC90087A37120097E49008F7
:200C40007A37E0FCA3E0FDA3E0FEA3E0FF780C120096F5C004C005C006C00790087A37E024
:200C6000FCA3E0FDA3E0FEA3E0FF7814120096E2D003D002D001D000EF4BFFEE4AFEED49F4
:200C8000FDEC48FC90087A37120097E490087A37E0FCA3E0FDA3E0FEA3E0FF90087A2BE08C
:200CA000F8A3E0F9A3E0FAA3E0FBEF2BFFEE3AFEED39FDEC38FC90087A37120097E49008D5
:200CC0007A33E0F8A3E0F9A3E0FAA3E0FBC000C001C002C00390087A2FE0FCA3E0FDA3E0F2
:200CE000FEA3E0FF90087A2BE0F8A3E0F9A3E0FAA3E06FFFEA6EFEE96DFDE86CFC90087A6A
:200D000037E0F8A3E0F9A3E0FAA3E05FFFEA5EFEE95DFDE85CFC90087A2FE0F8A3E0F9A3E9
:200D2000E0FAA3E06FFFEA6EFEE96DFDE86CFC90087A28E0FBA3E0FAA3E02428F9E43AFA7D
:200D40001200975DEF2BFFEE3AFEED39FDEC38FCEF24B1FFEE345BFEED34FFFDEC34FFFC95
:200D6000D003D002D001D000EB2FFFEA3EFEE93DFDE83CFC90087A33120097E490087A3394
:200D8000E0FCA3E0FDA3E0FEA3E0FF7811120096F5C004C005C006C00790087A33E0FCA3F4
:200DA000E0FDA3E0FEA3E0FF780F120096E2D003D002D001D000EF4BFFEE4AFEED49FDEC6E
:200DC00048FC90087A33120097E490087A33E0FCA3E0FDA3E0FEA3E0FFA3E0F8A3E0F9A3BF
:200DE000E0FAA3E0FBEF2BFFEE3AFEED39FDEC38FC90087A33120097E490087A2FE0F8A38B
:200E0000E0F9A3E0FAA3E0FBC000C001C002C00390087A2BE0FCA3E0FDA3E0FEA3E0FF90CC
:200E2000087A37E0F8A3E0F9A3E0FAA3E06FFFEA6EFEE96DFDE86CFC90087A33E0F8A3E09E
:200E4000F9A3E0FAA3E05FFFEA5EFEE95DFDE85CFC90087A2BE0F8A3E0F9A3E0FAA3E06F72
:200E6000FFEA6EFEE96DFDE86CFC90087A28E0FBA3E0FAA3E0242CF9E43AFA1200975DEF0F
:200E80002BFFEE3AFEED39FDEC38FCEF24BEFFEE34D7FEED345CFDEC3489FCD003D002D064
:200EA00001D000EB2FFFEA3EFEE93DFDE83CFC90087A2F120097E490087A2FE0FCA3E0FD74
:200EC000A3E0FEA3E0FF7816120096F5C004C005C006C00790087A2FE0FCA3E0FDA3E0FEB0
:200EE000A3E0FF780A120096E2D003D002D001D000EF4BFFEE4AFEED49FDEC48FC90087A3A
:200F00002F120097E490087A2FE0FCA3E0FDA3E0FEA3E0FFA3E0F8A3E0F9A3E0FAA3E0FB83
:200F2000EF2BFFEE3AFEED39FDEC38FC90087A2F120097E490087A2BE0F8A3E0F9A3E0FA53
:200F4000A3E0FBC000C001C002C00390087A37E0FCA3E0FDA3E0FEA3E0FF90087A33E0F848
:200F6000A3E0F9A3E0FAA3E06FFFEA6EFEE96DFDE86CFC90087A2FE0F8A3E0F9A3E0FAA3D9
:200F8000E05FFFEA5EFEE95DFDE85CFC90087A37E0F8A3E0F9A3E0FAA3E06FFFEA6EFEE900
:200FA0006DFDE86CFC90087A28E0FBA3E0FAA3E02430F9E43AFA1200975DEF2BFFEE3AFEB8
:200FC000ED39FDEC38FCEF2422FFEE3411FEED3490FDEC346BFCD003D002D001D000EB2FD4
:200FE000FFEA3EFEE93DFDE83CFC90087A2B120097E490087A2BE0FCA3E0FDA3E0FEA3E022
:20100000FF7807120096F5C004C005C006C00790087A2BE0FCA3E0FDA3E0FEA3E0FF781972
:20102000120096E2D003D002D001D000EF4BFFEE4AFEED49FDEC48FC90087A2B120097E444
:2010400090087A2BE0FCA3E0FDA3E0FEA3E0FFA3E0F8A3E0F9A3E0FAA3E0FBEF2BFFEE3AC1
:20106000FEED39FDEC38FC90087A2B120097E490087A37E0F8A3E0F9A3E0FAA3E0FBC0000D
:20108000C001C002C00390087A33E0FCA3E0FDA3E0FEA3E0FF90087A2FE0F8A3E0F9A3E04E
:2010A000FAA3E06FFFEA6EFEE96DFDE86CFC90087A2BE0F8A3E0F9A3E0FAA3E05FFFEA5E15
:2010C000FEE95DFDE85CFC90087A33E0F8A3E0F9A3E0FAA3E06FFFEA6EFEE96DFDE86CFC8F
:2010E00090087A28E0FBA3E0FAA3E02434F9E43AFA1200975DEF2BFFEE3AFEED39FDEC38E6
:20110000FCEF2493FFEE3471FEED3498FDEC34FDFCD003D002D001D000EB2FFFEA3EFEE960
:201120003DFDE83CFC90087A37120097E490087A37E0FCA3E0FDA3E0FEA3E0FF780C120041
:2011400096F5C004C005C006C00790087A37E0FCA3E0FDA3E0FEA3E0FF7814120096E2D060
:2011600003D002D001D000EF4BFFEE4AFEED49FDEC48FC90087A37120097E490087A37E028
:20118000FCA3E0FDA3E0FEA3E0FF90087A2BE0F8A3E0F9A3E0FAA3E0FBEF2BFFEE3AFEED18
:2011A00039FDEC38FC90087A37120097E490087A33E0F8A3E0F9A3E0FAA3E0FBC000C001EE
:2011C000C002C00390087A2FE0FCA3E0FDA3E0FEA3E0FF90087A2BE0F8A3E0F9A3E0FAA339
:2011E000E06FFFEA6EFEE96DFDE86CFC90087A37E0F8A3E0F9A3E0FAA3E05FFFEA5EFEE97E
:201200005DFDE85CFC90087A2FE0F8A3E0F9A3E0FAA3E06FFFEA6EFEE96DFDE86CFC9008A0
:201220007A28E0FBA3E0FAA3E02438F9E43AFA1200975DEF2BFFEE3AFEED39FDEC38FCEF4D
:20124000248EFFEE3443FEED3479FDEC34A6FCD003D002D001D000EB2FFFEA3EFEE93DFD79
:20126000E83CFC90087A33120097E490087A33E0FCA3E0FDA3E0FEA3E0FF7811120096F5B2
:20128000C004C005C006C00790087A33E0FCA3E0FDA3E0FEA3E0FF780F120096E2D003D0E0
:2012A00002D001D000EF4BFFEE4AFEED49FDEC48FC90087A33120097E490087A33E0FCA323
:2012C000E0FDA3E0FEA3E0FFA3E0F8A3E0F9A3E0FAA3E0FBEF2BFFEE3AFEED39FDEC38FCBA
:2012E00090087A33120097E490087A2FE0F8A3E0F9A3E0FAA3E0FBC000C001C002C00390F6
:20130000087A2BE0FCA3E0FDA3E0FEA3E0FF90087A37E0F8A3E0F9A3E0FAA3E06FFFEA6E5E
:20132000FEE96DFDE86CFC90087A33E0F8A3E0F9A3E0FAA3E05FFFEA5EFEE95DFDE85CFC4C
:2013400090087A2BE0F8A3E0F9A3E0FAA3E06FFFEA6EFEE96DFDE86CFC90087A28E0FBA3DD
:20136000E0FAA3E0243CF9E43AFA1200975DEF2BFFEE3AFEED39FDEC38FCEF2421FFEE34C2
:2013800008FEED34B4FDEC3449FCD003D002D001D000EB2FFFEA3EFEE93DFDE83CFC9008B0
:2013A0007A2F120097E490087A2FE0FCA3E0FDA3E0FEA3E0FF7816120096F5C004C005C0E3
:2013C00006C00790087A2FE0FCA3E0FDA3E0FEA3E0FF780A120096E2D003D002D001D0004E
:2013E000EF4BFFEE4AFEED49FDEC48FC90087A2F120097E490087A2FE0FCA3E0FDA3E0FE2F
:20140000A3E0FFA3E0F8A3E0F9A3E0FAA3E0FBEF2BFFEE3AFEED39FDEC38FC90087A2F1283
:201420000097E490087A2BE0F8A3E0F9A3E0FAA3E0FBC000C001C002C00390087A33E0FC7E
:20144000A3E0FDA3E0FEA3E0FF90087A2FE0F8A3E0F9A3E0FAA3E06FFFEA6EFEE96DFDE875
:201460006CFC90087A37E0F8A3E0F9A3E0FAA3E05FFFEA5EFEE95DFDE85CFC90087A33E01B
:20148000F8A3E0F9A3E0FAA3E06FFFEA6EFEE96DFDE86CFC90087A28E0FBA3E0FAA3E02438
:2014A00004F9E43AFA1200975DEF2BFFEE3AFEED39FDEC38FCEF2462FFEE3425FEED341E97
:2014C000FDEC34F6FCD003D002D001D000EB2FFFEA3EFEE93DFDE83CFC90087A2B1200974F
:2014E000E490087A2BE0FCA3E0FDA3E0FEA3E0FF7805120096F5C004C005C006C0079008A4
:201500007A2BE0FCA3E0FDA3E0FEA3E0FF781B120096E2D003D002D001D000EF4BFFEE4AF3
:20152000FEED49FDEC48FC90087A2B120097E490087A2BE0FCA3E0FDA3E0FEA3E0FFA3E061
:20154000F8A3E0F9A3E0FAA3E0FBEF2BFFEE3AFEED39FDEC38FC90087A2B120097E4900838
:201560007A37E0F8A3E0F9A3E0FAA3E0FBC000C001C002C00390087A2FE0FCA3E0FDA3E045
:20158000FEA3E0FF90087A2BE0F8A3E0F9A3E0FAA3E06FFFEA6EFEE96DFDE86CFC90087AC1
:2015A00033E0F8A3E0F9A3E0FAA3E05FFFEA5EFEE95DFDE85CFC90087A2FE0F8A3E0F9A345
:2015C000E0FAA3E06FFFEA6EFEE96DFDE86CFC90087A28E0FBA3E0FAA3E02418F9E43AFAE5
:2015E0001200975DEF2BFFEE3AFEED39FDEC38FCEF2440FFEE34B3FEED3440FDEC34C0FC04
:20160000D003D002D001D000EB2FFFEA3EFEE93DFDE83CFC90087A37120097E490087A37E3
:20162000E0FCA3E0FDA3E0FEA3E0FF7809120096F5C004C005C006C00790087A37E0FCA34F
:20164000E0FDA3E0FEA3E0FF7817120096E2D003D002D001D000EF4BFFEE4AFEED49FDECBD
:2016600048FC90087A37120097E490087A37E0FCA3E0FDA3E0FEA3E0FF90087A2BE0F8A3F0
:20168000E0F9A3E0FAA3E0FBEF2BFFEE3AFEED39FDEC38FC90087A37120097E490087A33D9
:2016A000E0F8A3E0F9A3E0FAA3E0FBC000C001C002C00390087A2BE0FCA3E0FDA3E0FEA318
:2016C000E0FF90087A37E0F8A3E0F9A3E0FAA3E06FFFEA6EFEE96DFDE86CFC90087A2FE006
:2016E000F8A3E0F9A3E0FAA3E05FFFEA5EFEE95DFDE85CFC90087A2BE0F8A3E0F9A3E0FA41
:20170000A3E06FFFEA6EFEE96DFDE86CFC90087A28E0FBA3E0FAA3E0242CF9E43AFA120057
:20172000975DEF2BFFEE3AFEED39FDEC38FCEF2451FFEE345AFEED345EFDEC3426FCD003C5
:20174000D002D001D000EB2FFFEA3EFEE93DFDE83CFC90087A33120097E490087A33E0FCA1
:20176000A3E0FDA3E0FEA3E0FF780E120096F5C004C005C006C00790087A33E0FCA3E0FD0C
:20178000A3E0FEA3E0FF7812120096E2D003D002D001D000EF4BFFEE4AFEED49FDEC48FC1A
:2017A00090087A33120097E490087A33E0FCA3E0FDA3E0FEA3E0FFA3E0F8A3E0F9A3E0FA3F
:2017C000A3E0FBEF2BFFEE3AFEED39FDEC38FC90087A33120097E490087A2FE0F8A3E0F9A2
:2017E000A3E0FAA3E0FBC000C001C002C00390087A37E0FCA3E0FDA3E0FEA3E0FF90087A2E
:2018000033E0F8A3E0F9A3E0FAA3E06FFFEA6EFEE96DFDE86CFC90087A2BE0F8A3E0F9A3A6
:20182000E0FAA3E05FFFEA5EFEE95DFDE85CFC90087A37E0F8A3E0F9A3E0FAA3E06FFFEA2F
:201840006EFEE96DFDE86CFC90087A28E0FBA3E0FAA3E0F91200975DEF2BFFEE3AFEED3900
:20186000FDEC38FCEF24AAFFEE34C7FEED34B6FDEC34E9FCD003D002D001D000EB2FFFEA86
:201880003EFEE93DFDE83CFC90087A2F120097E490087A2FE0FCA3E0FDA3E0FEA3E0FF78E3
:2018A00014120096F5C004C005C006C00790087A2FE0FCA3E0FDA3E0FEA3E0FF780C12002B
:2018C00096E2D003D002D001D000EF4BFFEE4AFEED49FDEC48FC90087A2F120097E4900812
:2018E0007A2FE0FCA3E0FDA3E0FEA3E0FFA3E0F8A3E0F9A3E0FAA3E0FBEF2BFFEE3AFEEDC2
:2019000039FDEC38FC90087A2F120097E490087A2BE0F8A3E0F9A3E0FAA3E0FBC000C00196
:20192000C002C00390087A33E0FCA3E0FDA3E0FEA3E0FF90087A2FE0F8A3E0F9A3E0FAA3C9
:20194000E06FFFEA6EFEE96DFDE86CFC90087A37E0F8A3E0F9A3E0FAA3E05FFFEA5EFEE916
:201960005DFDE85CFC90087A33E0F8A3E0F9A3E0FAA3E06FFFEA6EFEE96DFDE86CFC900835
:201980007A28E0FBA3E0FAA3E02414F9E43AFA1200975DEF2BFFEE3AFEED39FDEC38FCEF0A
:2019A000245DFFEE3410FEED342FFDEC34D6FCD003D002D001D000EB2FFFEA3EFEE93DFD90
:2019C000E83CFC90087A2B120097E490087A2BE0FCA3E0FDA3E0FEA3E0FF7805120096F567
:2019E000C004C005C006C00790087A2BE0FCA3E0FDA3E0FEA3E0FF781B120096E2D003D075
:201A000002D001D000EF4BFFEE4AFEED49FDEC48FC90087A2B120097E490087A2BE0FCA3CB
:201A2000E0FDA3E0FEA3E0FFA3E0F8A3E0F9A3E0FAA3E0FBEF2BFFEE3AFEED39FDEC38FC52
:201A400090087A2B120097E490087A37E0F8A3E0F9A3E0FAA3E0FBC000C001C002C003908E
:201A6000087A2FE0FCA3E0FDA3E0FEA3E0FF90087A2BE0F8A3E0F9A3E0FAA3E06FFFEA6EFF
:201A8000FEE96DFDE86CFC90087A33E0F8A3E0F9A3E0FAA3E05FFFEA5EFEE95DFDE85CFCE5
:201AA00090087A2FE0F8A3E0F9A3E0FAA3E06FFFEA6EFEE96DFDE86CFC90087A28E0FBA372
:201AC000E0FAA3E02428F9E43AFA1200975DEF2BFFEE3AFEED39FDEC38FCEF2453FFEE343D
:201AE00014FEED3444FDEC3402FCD003D002D001D000EB2FFFEA3EFEE93DFDE83CFC9008F4
:201B00007A37120097E490087A37E0FCA3E0FDA3E0FEA3E0FF7809120096F5C004C005C078
:201B200006C00790087A37E0FCA3E0FDA3E0FEA3E0FF7817120096E2D003D002D001D000D1
:201B4000EF4BFFEE4AFEED49FDEC48FC90087A37120097E490087A37E0FCA3E0FDA3E0FEB7
:201B6000A3E0FF90087A2BE0F8A3E0F9A3E0FAA3E0FBEF2BFFEE3AFEED39FDEC38FC90083D
:201B80007A37120097E490087A33E0F8A3E0F9A3E0FAA3E0FBC000C001C002C00390087A5B
:201BA0002BE0FCA3E0FDA3E0FEA3E0FF90087A37E0F8A3E0F9A3E0FAA3E06FFFEA6EFEE951
:201BC0006DFDE86CFC90087A2FE0F8A3E0F9A3E0FAA3E05FFFEA5EFEE95DFDE85CFC9008F7
:201BE0007A2BE0F8A3E0F9A3E0FAA3E06FFFEA6EFEE96DFDE86CFC90087A28E0FBA3E0FAF3
:201C0000A3E0243CF9E43AFA1200975DEF2BFFEE3AFEED39FDEC38FCEF2481FFEE34E6FEAF
:201C2000ED34A1FDEC34D8FCD003D002D001D000EB2FFFEA3EFEE93DFDE83CFC90087A33E4
:201C4000120097E490087A33E0FCA3E0FDA3E0FEA3E0FF780E120096F5C004C005C006C021
:201C60000790087A33E0FCA3E0FDA3E0FEA3E0FF7812120096E2D003D002D001D000EF4B25
:201C8000FFEE4AFEED49FDEC48FC90087A33120097E490087A33E0FCA3E0FDA3E0FEA3E035
:201CA000FFA3E0F8A3E0F9A3E0FAA3E0FBEF2BFFEE3AFEED39FDEC38FC90087A33120097C3
:201CC000E490087A2FE0F8A3E0F9A3E0FAA3E0FBC000C001C002C00390087A37E0FCA3E0E2
:201CE000FDA3E0FEA3E0FF90087A33E0F8A3E0F9A3E0FAA3E06FFFEA6EFEE96DFDE86CFCE4
:201D000090087A2BE0F8A3E0F9A3E0FAA3E05FFFEA5EFEE95DFDE85CFC90087A37E0F8A347
:201D2000E0F9A3E0FAA3E06FFFEA6EFEE96DFDE86CFC90087A28E0FBA3E0FAA3E02410F921
:201D4000E43AFA1200975DEF2BFFEE3AFEED39FDEC38FCEF24C8FFEE34FBFEED34D3FDEC11
:201D600034E7FCD003D002D001D000EB2FFFEA3EFEE93DFDE83CFC90087A2F120097E49026
:201D8000087A2FE0FCA3E0FDA3E0FEA3E0FF7814120096F5C004C005C006C00790087A2FB3
:201DA000E0FCA3E0FDA3E0FEA3E0FF780C120096E2D003D002D001D000EF4BFFEE4AFEED14
:201DC00049FDEC48FC90087A2F120097E490087A2FE0FCA3E0FDA3E0FEA3E0FFA3E0F8A301
:201DE000E0F9A3E0FAA3E0FBEF2BFFEE3AFEED39FDEC38FC90087A2F120097E490087A2B82
:201E0000E0F8A3E0F9A3E0FAA3E0FBC000C001C002C00390087A33E0FCA3E0FDA3E0FEA3A8
:201E2000E0FF90087A2FE0F8A3E0F9A3E0FAA3E06FFFEA6EFEE96DFDE86CFC90087A37E09E
:201E4000F8A3E0F9A3E0FAA3E05FFFEA5EFEE95DFDE85CFC90087A33E0F8A3E0F9A3E0FAD1
:201E6000A3E06FFFEA6EFEE96DFDE86CFC90087A28E0FBA3E0FAA3E02424F9E43AFA1200F8
:201E8000975DEF2BFFEE3AFEED39FDEC38FCEF24E6FFEE34CDFEED34E1FDEC3421FCD003D8
:201EA000D002D001D000EB2FFFEA3EFEE93DFDE83CFC90087A2B120097E490087A2BE0FC4A
:201EC000A3E0FDA3E0FEA3E0FF7805120096F5C004C005C006C00790087A2BE0FCA3E0FDB6
:201EE000A3E0FEA3E0FF781B120096E2D003D002D001D000EF4BFFEE4AFEED49FDEC48FCAA
:201F000090087A2B120097E490087A2BE0FCA3E0FDA3E0FEA3E0FFA3E0F8A3E0F9A3E0FAE7
:201F2000A3E0FBEF2BFFEE3AFEED39FDEC38FC90087A2B120097E490087A37E0F8A3E0F93A
:201F4000A3E0FAA3E0FBC000C001C002C00390087A2FE0FCA3E0FDA3E0FEA3E0FF90087ACE
:201F60002BE0F8A3E0F9A3E0FAA3E06FFFEA6EFEE96DFDE86CFC90087A33E0F8A3E0F9A33F
:201F8000E0FAA3E05FFFEA5EFEE95DFDE85CFC90087A2FE0F8A3E0F9A3E0FAA3E06FFFEAD0
:201FA0006EFEE96DFDE86CFC90087A28E0FBA3E0FAA3E02438F9E43AFA1200975DEF2BFF71
:201FC000EE3AFEED39FDEC38FCEF24D6FFEE3407FEED3437FDEC34C3FCD003D002D001D00F
:201FE00000EB2FFFEA3EFEE93DFDE83CFC90087A37120097E490087A37E0FCA3E0FDA3E061
:20200000FEA3E0FF7809120096F5C004C005C006C00790087A37E0FCA3E0FDA3E0FEA3E063
:20202000FF7817120096E2D003D002D001D000EF4BFFEE4AFEED49FDEC48FC90087A371215
:202040000097E490087A37E0FCA3E0FDA3E0FEA3E0FF90087A2BE0F8A3E0F9A3E0FAA3E0CC
:20206000FBEF2BFFEE3AFEED39FDEC38FC90087A37120097E490087A33E0F8A3E0F9A3E0F1
:20208000FAA3E0FBC000C001C002C00390087A2BE0FCA3E0FDA3E0FEA3E0FF90087A37E0FD
:2020A000F8A3E0F9A3E0FAA3E06FFFEA6EFEE96DFDE86CFC90087A2FE0F8A3E0F9A3E0FA33
:2020C000A3E05FFFEA5EFEE95DFDE85CFC90087A2BE0F8A3E0F9A3E0FAA3E06FFFEA6EFE01
:2020E000E96DFDE86CFC90087A28E0FBA3E0FAA3E0240CF9E43AFA1200975DEF2BFFEE3AA0
:20210000FEED39FDEC38FCEF2487FFEE340DFEED34D5FDEC34F4FCD003D002D001D000EB84
:202120002FFFEA3EFEE93DFDE83CFC90087A33120097E490087A33E0FCA3E0FDA3E0FEA371
:20214000E0FF780E120096F5C004C005C006C00790087A33E0FCA3E0FDA3E0FEA3E0FF784B
:2021600012120096E2D003D002D001D000EF4BFFEE4AFEED49FDEC48FC90087A33120097BD
:20218000E490087A33E0FCA3E0FDA3E0FEA3E0FFA3E0F8A3E0F9A3E0FAA3E0FBEF2BFFEEBE
:2021A0003AFEED39FDEC38FC90087A33120097E490087A2FE0F8A3E0F9A3E0FAA3E0FBC082
:2021C00000C001C002C00390087A37E0FCA3E0FDA3E0FEA3E0FF90087A33E0F8A3E0F9A3D5
:2021E000E0FAA3E06FFFEA6EFEE96DFDE86CFC90087A2BE0F8A3E0F9A3E0FAA3E05FFFEA42
:202200005EFEE95DFDE85CFC90087A37E0F8A3E0F9A3E0FAA3E06FFFEA6EFEE96DFDE86CD7
:20222000FC90087A28E0FBA3E0FAA3E02420F9E43AFA1200975DEF2BFFEE3AFEED39FDECE4
:2022400038FCEF24EDFFEE3414FEED345AFDEC3445FCD003D002D001D000EB2FFFEA3EFEB9
:20226000E93DFDE83CFC90087A2F120097E490087A2FE0FCA3E0FDA3E0FEA3E0FF7814120F
:202280000096F5C004C005C006C00790087A2FE0FCA3E0FDA3E0FEA3E0FF780C120096E2EF
:2022A000D003D002D001D000EF4BFFEE4AFEED49FDEC48FC90087A2F120097E490087A2FF7
:2022C000E0FCA3E0FDA3E0FEA3E0FFA3E0F8A3E0F9A3E0FAA3E0FBEF2BFFEE3AFEED39FD4B
:2022E000EC38FC90087A2F120097E490087A2BE0F8A3E0F9A3E0FAA3E0FBC000C001C00221
:20230000C00390087A33E0FCA3E0FDA3E0FEA3E0FF90087A2FE0F8A3E0F9A3E0FAA3E06F52
:20232000FFEA6EFEE96DFDE86CFC90087A37E0F8A3E0F9A3E0FAA3E05FFFEA5EFEE95DFD21
:20234000E85CFC90087A33E0F8A3E0F9A3E0FAA3E06FFFEA6EFEE96DFDE86CFC90087A2803
:20236000E0FBA3E0FAA3E02434F9E43AFA1200975DEF2BFFEE3AFEED39FDEC38FCEF240579
:20238000FFEE34E9FEED34E3FDEC34A9FCD003D002D001D000EB2FFFEA3EFEE93DFDE83CA3
:2023A000FC90087A2B120097E490087A2BE0FCA3E0FDA3E0FEA3E0FF7805120096F5C004DD
:2023C000C005C006C00790087A2BE0FCA3E0FDA3E0FEA3E0FF781B120096E2D003D002D07D
:2023E00001D000EF4BFFEE4AFEED49FDEC48FC90087A2B120097E490087A2BE0FCA3E0FDD7
:20240000A3E0FEA3E0FFA3E0F8A3E0F9A3E0FAA3E0FBEF2BFFEE3AFEED39FDEC38FC9008AD
:202420007A2B120097E490087A37E0F8A3E0F9A3E0FAA3E0FBC000C001C002C00390087ABA
:202440002FE0FCA3E0FDA3E0FEA3E0FF90087A2BE0F8A3E0F9A3E0FAA3E06FFFEA6EFEE9B0
:202460006DFDE86CFC90087A33E0F8A3E0F9A3E0FAA3E05FFFEA5EFEE95DFDE85CFC90084A
:202480007A2FE0F8A3E0F9A3E0FAA3E06FFFEA6EFEE96DFDE86CFC90087A28E0FBA3E0FA46
:2024A000A3E02408F9E43AFA1200975DEF2BFFEE3AFEED39FDEC38FCEF24F8FFEE34A3FE07
:2024C000ED34EFFDEC34FCFCD003D002D001D000EB2FFFEA3EFEE93DFDE83CFC90087A37C6
:2024E000120097E490087A37E0FCA3E0FDA3E0FEA3E0FF7809120096F5C004C005C006C07A
:202500000790087A37E0FCA3E0FDA3E0FEA3E0FF7817120096E2D003D002D001D000EF4B73
:20252000FFEE4AFEED49FDEC48FC90087A37120097E490087A37E0FCA3E0FDA3E0FEA3E084
:20254000FF90087A2BE0F8A3E0F9A3E0FAA3E0FBEF2BFFEE3AFEED39FDEC38FC90087A3725
:20256000120097E490087A33E0F8A3E0F9A3E0FAA3E0FBC000C001C002C00390087A2BE017
:20258000FCA3E0FDA3E0FEA3E0FF90087A37E0F8A3E0F9A3E0FAA3E06FFFEA6EFEE96DFD08
:2025A000E86CFC90087A2FE0F8A3E0F9A3E0FAA3E05FFFEA5EFEE95DFDE85CFC90087A2BD2
:2025C000E0F8A3E0F9A3E0FAA3E06FFFEA6EFEE96DFDE86CFC90087A28E0FBA3E0FAA3E02B
:2025E000241CF9E43AFA1200975DEF2BFFEE3AFEED39FDEC38FCEF24D9FFEE3402FEED34D4
:202600006FFDEC3467FCD003D002D001D000EB2FFFEA3EFEE93DFDE83CFC90087A331200AC
:2026200097E490087A33E0FCA3E0FDA3E0FEA3E0FF780E120096F5C004C005C006C00790B2
:20264000087A33E0FCA3E0FDA3E0FEA3E0FF7812120096E2D003D002D001D000EF4BFFEEE5
:202660004AFEED49FDEC48FC90087A33120097E490087A33E0FCA3E0FDA3E0FEA3E0FFA396
:20268000E0F8A3E0F9A3E0FAA3E0FBEF2BFFEE3AFEED39FDEC38FC90087A33120097E49007
:2026A000087A2FE0F8A3E0F9A3E0FAA3E0FBC000C001C002C00390087A37E0FCA3E0FDA3CC
:2026C000E0FEA3E0FF90087A33E0F8A3E0F9A3E0FAA3E06FFFEA6EFEE96DFDE86CFC900802
:2026E0007A2BE0F8A3E0F9A3E0FAA3E05FFFEA5EFEE95DFDE85CFC90087A37E0F8A3E0F91D
:20270000A3E0FAA3E06FFFEA6EFEE96DFDE86CFC90087A28E0FBA3E0FAA3E02430F9E43AD2
:20272000FA1200975DEF2BFFEE3AFEED39FDEC38FCEF248AFFEE344CFEED342AFDEC348D1A
:20274000FCD003D002D001D000EB2FFFEA3EFEE93DFDE83CFC90087A2F120097E490087AD5
:202760002FE0FCA3E0FDA3E0FEA3E0FF7814120096F5C004C005C006C00790087A2FE0FC6F
:20278000A3E0FDA3E0FEA3E0FF780C120096E2D003D002D001D000EF4BFFEE4AFEED49FDC0
:2027A000EC48FC90087A2F120097E490087A2FE0FCA3E0FDA3E0FEA3E0FFA3E0F8A3E0F984
:2027C000A3E0FAA3E0FBEF2BFFEE3AFEED39FDEC38FC90087A2F120097E490087A2BE0F899
:2027E000A3E0F9A3E0FAA3E0FBC000C001C002C00390087A28E0FBA3E0FAA3E02414F9E432
:202800003AFA1200975DC000C001C00290087A33E0FCA3E0FDA3E0FEA3E0FF90087A2FE076
:20282000F8A3E0F9A3E0FAA3E06FFFEA6EFEE96DFDE86CFC90087A37E0F8A3E0F9A3E0FAA3
:20284000A3E06FFFEA6EFEE96DFDE86CFCD002D001D000EF2BFFEE3AFEED39FDEC38FCEFAA
:202860002442FFEE3439FEED34FAFDEC34FFFCD003D002D001D000EB2FFFEA3EFEE93DFDBF
:20288000E83CFC90087A2B120097E490087A2BE0FCA3E0FDA3E0FEA3E0FF7804120096F599
:2028A000C004C005C006C00790087A2BE0FCA3E0FDA3E0FEA3E0FF781C120096E2D003D0A5
:2028C00002D001D000EF4BFFEE4AFEED49FDEC48FC90087A2B120097E490087A2BE0FCA3FD
:2028E000E0FDA3E0FEA3E0FFA3E0F8A3E0F9A3E0FAA3E0FBEF2BFFEE3AFEED39FDEC38FC84
:2029000090087A2B120097E490087A37E0F8A3E0F9A3E0FAA3E0FBC000C001C002C00390BF
:20292000087A28E0FBA3E0FAA3E02420F9E43AFA1200975DC000C001C00290087A2FE0FC57
:20294000A3E0FDA3E0FEA3E0FF90087A2BE0F8A3E0F9A3E0FAA3E06FFFEA6EFEE96DFDE864
:202960006CFC90087A33E0F8A3E0F9A3E0FAA3E06FFFEA6EFEE96DFDE86CFCD002D001D07C
:2029800000EF2BFFEE3AFEED39FDEC38FCEF2481FFEE34F6FEED3471FDEC3487FCD003D037
:2029A00002D001D000EB2FFFEA3EFEE93DFDE83CFCA3120097E490087A37E0FCA3E0FDA37A
:2029C000E0FEA3E0FF780B120096F5C004C005C006C00790087A37E0FCA3E0FDA3E0FEA398
:2029E000E0FF7815120096E2D003D002D001D000EF4BFFEE4AFEED49FDEC48FC90087A3780
:202A0000120097E490087A37E0FCA3E0FDA3E0FEA3E0FF90087A2BE0F8A3E0F9A3E0FAA3D0
:202A2000E0FBEF2BFFEE3AFEED39FDEC38FC90087A37120097E490087A33E0F8A3E0F9A327
:202A4000E0FAA3E0FBC000C001C002C00390087A28E0FBA3E0FAA3E0242CF9E43AFA120090
:202A6000975DC000C001C00290087A2BE0FCA3E0FDA3E0FEA3E0FF90087A37E0F8A3E0F9E6
:202A8000A3E0FAA3E06FFFEA6EFEE96DFDE86CFC90087A2FE0F8A3E0F9A3E0FAA3E06FFFCC
:202AA000EA6EFEE96DFDE86CFCD002D001D000EF2BFFEE3AFEED39FDEC38FCEF2422FFEE06
:202AC0003461FEED349DFDEC346DFCD003D002D001D000EB2FFFEA3EFEE93DFDE83CFCA3B4
:202AE000120097E490087A33E0FCA3E0FDA3E0FEA3E0FF7810120096F5C004C005C006C071
:202B00000790087A33E0FCA3E0FDA3E0FEA3E0FF7810120096E2D003D002D001D000EF4B78
:202B2000FFEE4AFEED49FDEC48FC90087A33120097E490087A33E0FCA3E0FDA3E0FEA3E086
:202B4000FFA3E0F8A3E0F9A3E0FAA3E0FBEF2BFFEE3AFEED39FDEC38FC90087A3312009714
:202B6000E490087A2FE0F8A3E0F9A3E0FAA3E0FBC000C001C002C00390087A28E0FBA3E043
:202B8000FAA3E02438F9E43AFA1200975DC000C001C00290087A37E0FCA3E0FDA3E0FEA339
:202BA000E0FF90087A33E0F8A3E0F9A3E0FAA3E06FFFEA6EFEE96DFDE86CFC90087A2BE019
:202BC000F8A3E0F9A3E0FAA3E06FFFEA6EFEE96DFDE86CFCD002D001D000EF2BFFEE3AFE68
:202BE000ED39FDEC38FCEF240CFFEE3438FEED34E5FDEC34FDFCD003D002D001D000EB2FA0
:202C0000FFEA3EFEE93DFDE83CFCA3120097E490087A2FE0FCA3E0FDA3E0FEA3E0FF7817ED
:202C2000120096F5C004C005C006C00790087A2FE0FCA3E0FDA3E0FEA3E0FF780912009618
:202C4000E2D003D002D001D000EF4BFFEE4AFEED49FDEC48FC90087A2F120097E490087A9A
:202C60002FE0FCA3E0FDA3E0FEA3E0FFA3E0F8A3E0F9A3E0FAA3E0FBEF2BFFEE3AFEED396F
:202C8000FDEC38FC90087A2F120097E490087A2BE0F8A3E0F9A3E0FAA3E0FBC000C001C07C
:202CA00002C00390087A28E0FBA3E0FAA3E02404F9E43AFA1200975DC000C001C002900820
:202CC0007A33E0FCA3E0FDA3E0FEA3E0FF90087A2FE0F8A3E0F9A3E0FAA3E06FFFEA6EFE8F
:202CE000E96DFDE86CFC90087A37E0F8A3E0F9A3E0FAA3E06FFFEA6EFEE96DFDE86CFCD05D
:202D000002D001D000EF2BFFEE3AFEED39FDEC38FCEF2444FFEE34EAFEED34BEFDEC34A48E
:202D2000FCD003D002D001D000EB2FFFEA3EFEE93DFDE83CFC90087A2B120097E490087AF3
:202D40002BE0FCA3E0FDA3E0FEA3E0FF7804120096F5C004C005C006C00790087A2BE0FCA1
:202D6000A3E0FDA3E0FEA3E0FF781C120096E2D003D002D001D000EF4BFFEE4AFEED49FDCA
:202D8000EC48FC90087A2B120097E490087A2BE0FCA3E0FDA3E0FEA3E0FFA3E0F8A3E0F9A6
:202DA000A3E0FAA3E0FBEF2BFFEE3AFEED39FDEC38FC90087A2B120097E490087A37E0F8AB
:202DC000A3E0F9A3E0FAA3E0FBC000C001C002C00390087A28E0FBA3E0FAA3E02410F9E450
:202DE0003AFA1200975DC000C001C00290087A2FE0FCA3E0FDA3E0FEA3E0FF90087A2BE099
:202E0000F8A3E0F9A3E0FAA3E06FFFEA6EFEE96DFDE86CFC90087A33E0F8A3E0F9A3E0FAC1
:202E2000A3E06FFFEA6EFEE96DFDE86CFCD002D001D000EF2BFFEE3AFEED39FDEC38FCEFC4
:202E400024A9FFEE34CFFEED34DEFDEC344BFCD003D002D001D000EB2FFFEA3EFEE93DFDAC
:202E6000E83CFCA3120097E490087A37E0FCA3E0FDA3E0FEA3E0FF780B120096F5C004C0B6
:202E800005C006C00790087A37E0FCA3E0FDA3E0FEA3E0FF7815120096E2D003D002D0016B
:202EA000D000EF4BFFEE4AFEED49FDEC48FC90087A37120097E490087A37E0FCA3E0FDA352
:202EC000E0FEA3E0FF90087A2BE0F8A3E0F9A3E0FAA3E0FBEF2BFFEE3AFEED39FDEC38FC84
:202EE00090087A37120097E490087A33E0F8A3E0F9A3E0FAA3E0FBC000C001C002C00390D2
:202F0000087A28E0FBA3E0FAA3E0241CF9E43AFA1200975DC000C001C00290087A2BE0FC79
:202F2000A3E0FDA3E0FEA3E0FF90087A37E0F8A3E0F9A3E0FAA3E06FFFEA6EFEE96DFDE872
:202F40006CFC90087A2FE0F8A3E0F9A3E0FAA3E06FFFEA6EFEE96DFDE86CFCD002D001D09A
:202F600000EF2BFFEE3AFEED39FDEC38FCEF2460FFEE344BFEED34BBFDEC34F6FCD003D064
:202F800002D001D000EB2FFFEA3EFEE93DFDE83CFCA3120097E490087A33E0FCA3E0FDA398
:202FA000E0FEA3E0FF7810120096F5C004C005C006C00790087A33E0FCA3E0FDA3E0FEA3B1
:202FC000E0FF7810120096E2D003D002D001D000EF4BFFEE4AFEED49FDEC48FC90087A33A3
:202FE000120097E490087A33E0FCA3E0FDA3E0FEA3E0FFA3E0F8A3E0F9A3E0FAA3E0FBEFBF
:203000002BFFEE3AFEED39FDEC38FC90087A33120097E490087A2FE0F8A3E0F9A3E0FAA396
:20302000E0FBC000C001C002C00390087A28E0FBA3E0FAA3E02428F9E43AFA1200975DC077
:2030400000C001C00290087A37E0FCA3E0FDA3E0FEA3E0FF90087A33E0F8A3E0F9A3E0FA2F
:20306000A3E06FFFEA6EFEE96DFDE86CFC90087A2BE0F8A3E0F9A3E0FAA3E06FFFEA6EFE11
:20308000E96DFDE86CFCD002D001D000EF2BFFEE3AFEED39FDEC38FCEF2470FFEE34BCFE3A
:2030A000ED34BFFDEC34BEFCD003D002D001D000EB2FFFEA3EFEE93DFDE83CFCA312009745
:2030C000E490087A2FE0FCA3E0FDA3E0FEA3E0FF7817120096F5C004C005C006C007900892
:2030E0007A2FE0FCA3E0FDA3E0FEA3E0FF7809120096E2D003D002D001D000EF4BFFEE4A06
:20310000FEED49FDEC48FC90087A2F120097E490087A2FE0FCA3E0FDA3E0FEA3E0FFA3E05D
:20312000F8A3E0F9A3E0FAA3E0FBEF2BFFEE3AFEED39FDEC38FC90087A2F120097E4900838
:203140007A2BE0F8A3E0F9A3E0FAA3E0FBC000C001C002C00390087A28E0FBA3E0FAA3E060
:203160002434F9E43AFA1200975DC000C001C00290087A33E0FCA3E0FDA3E0FEA3E0FF9069
:20318000087A2FE0F8A3E0F9A3E0FAA3E06FFFEA6EFEE96DFDE86CFC90087A37E0F8A3E01F
:2031A000F9A3E0FAA3E06FFFEA6EFEE96DFDE86CFCD002D001D000EF2BFFEE3AFEED39FDDA
:2031C000EC38FCEF24C6FFEE347EFEED349BFDEC3428FCD003D002D001D000EB2FFFEA3ED5
:2031E000FEE93DFDE83CFC90087A2B120097E490087A2BE0FCA3E0FDA3E0FEA3E0FF7804AC
:20320000120096F5C004C005C006C00790087A2BE0FCA3E0FDA3E0FEA3E0FF781C12009623
:20322000E2D003D002D001D000EF4BFFEE4AFEED49FDEC48FC90087A2B120097E490087AB8
:203240002BE0FCA3E0FDA3E0FEA3E0FFA3E0F8A3E0F9A3E0FAA3E0FBEF2BFFEE3AFEED398D
:20326000FDEC38FC90087A2B120097E490087A37E0F8A3E0F9A3E0FAA3E0FBC000C001C08E
:2032800002C00390087A2FE0FCA3E0FDA3E0FEA3E0FF90087A2BE0F8A3E0F9A3E0FAA3E038
:2032A0006FFFEA6EFEE96DFDE86CFC90087A33E0F8A3E0F9A3E0FAA3E06FFFEA6EFEE96DF4
:2032C000FDE86CFC90087A28E0FBA3E0FAA3E0F91200975DEF2BFFEE3AFEED39FDEC38FC0B
:2032E000EF24FAFFEE3427FEED34A1FDEC34EAFCD003D002D001D000EB2FFFEA3EFEE93D0B
:20330000FDE83CFC90087A37120097E490087A37E0FCA3E0FDA3E0FEA3E0FF780B120096E7
:20332000F5C004C005C006C00790087A37E0FCA3E0FDA3E0FEA3E0FF7815120096E2D003F0
:20334000D002D001D000EF4BFFEE4AFEED49FDEC48FC90087A37120097E490087A37E0FC2D
:20336000A3E0FDA3E0FEA3E0FF90087A2BE0F8A3E0F9A3E0FAA3E0FBEF2BFFEE3AFEED39D9
:20338000FDEC38FC90087A37120097E490087A33E0F8A3E0F9A3E0FAA3E0FBC000C001C065
:2033A00002C00390087A28E0FBA3E0FAA3E0240CF9E43AFA1200975DC000C001C002900811
:2033C0007A2BE0FCA3E0FDA3E0FEA3E0FF90087A37E0F8A3E0F9A3E0FAA3E06FFFEA6EFE88
:2033E000E96DFDE86CFC90087A2FE0F8A3E0F9A3E0FAA3E06FFFEA6EFEE96DFDE86CFCD05E
:2034000002D001D000EF2BFFEE3AFEED39FDEC38FCEF2485FFEE3430FEED34EFFDEC34D49F
:20342000FCD003D002D001D000EB2FFFEA3EFEE93DFDE83CFCA3120097E490087A33E0FC77
:20344000A3E0FDA3E0FEA3E0FF7810120096F5C004C005C006C00790087A33E0FCA3E0FD0D
:20346000A3E0FEA3E0FF7810120096E2D003D002D001D000EF4BFFEE4AFEED49FDEC48FC1F
:2034800090087A33120097E490087A33E0FCA3E0FDA3E0FEA3E0FFA3E0F8A3E0F9A3E0FA42
:2034A000A3E0FBEF2BFFEE3AFEED39FDEC38FC90087A33120097E490087A2FE0F8A3E0F9A5
:2034C000A3E0FAA3E0FBC000C001C002C00390087A28E0FBA3E0FAA3E02418F9E43AFA1277
:2034E00000975DC000C001C00290087A37E0FCA3E0FDA3E0FEA3E0FF90087A33E0F8A3E04D
:20350000F9A3E0FAA3E06FFFEA6EFEE96DFDE86CFC90087A2BE0F8A3E0F9A3E0FAA3E06F4B
:20352000FFEA6EFEE96DFDE86CFCD002D001D000EF2BFFEE3AFEED39FDEC38FCEF2405FF87
:20354000EE341DFEED3488FDEC3404FCD003D002D001D000EB2FFFEA3EFEE93DFDE83CFCA0
:20356000A3120097E490087A2FE0FCA3E0FDA3E0FEA3E0FF7817120096F5C004C005C00600
:20358000C00790087A2FE0FCA3E0FDA3E0FEA3E0FF7809120096E2D003D002D001D000EF84
:2035A0004BFFEE4AFEED49FDEC48FC90087A2F120097E490087A2FE0FCA3E0FDA3E0FEA399
:2035C000E0FFA3E0F8A3E0F9A3E0FAA3E0FBEF2BFFEE3AFEED39FDEC38FC90087A2F120045
:2035E00097E490087A2BE0F8A3E0F9A3E0FAA3E0FBC000C001C002C00390087A28E0FBA306
:20360000E0FAA3E02424F9E43AFA1200975DC000C001C00290087A33E0FCA3E0FDA3E0FE89
:20362000A3E0FF90087A2FE0F8A3E0F9A3E0FAA3E06FFFEA6EFEE96DFDE86CFC90087A37C3
:20364000E0F8A3E0F9A3E0FAA3E06FFFEA6EFEE96DFDE86CFCD002D001D000EF2BFFEE3AFB
:20366000FEED39FDEC38FCEF2439FFEE34D0FEED34D4FDEC34D9FCD003D002D001D000EBB6
:203680002FFFEA3EFEE93DFDE83CFC90087A2B120097E490087A2BE0FCA3E0FDA3E0FEA30C
:2036A000E0FF7804120096F5C004C005C006C00790087A2BE0FCA3E0FDA3E0FEA3E0FF78E8
:2036C0001C120096E2D003D002D001D000EF4BFFEE4AFEED49FDEC48FC90087A2B12009746
:2036E000E490087A2BE0FCA3E0FDA3E0FEA3E0FFA3E0F8A3E0F9A3E0FAA3E0FBEF2BFFEE51
:203700003AFEED39FDEC38FC90087A2B120097E490087A37E0F8A3E0F9A3E0FAA3E0FBC00C
:2037200000C001C002C00390087A28E0FBA3E0FAA3E02430F9E43AFA1200975DC000C00142
:20374000C00290087A2FE0FCA3E0FDA3E0FEA3E0FF90087A2BE0F8A3E0F9A3E0FAA3E06F07
:20376000FFEA6EFEE96DFDE86CFC90087A33E0F8A3E0F9A3E0FAA3E06FFFEA6EFEE96DFDA1
:20378000E86CFCD002D001D000EF2BFFEE3AFEED39FDEC38FCEF24E5FFEE3499FEED34DB38
:2037A000FDEC34E6FCD003D002D001D000EB2FFFEA3EFEE93DFDE83CFCA3120097E490087A
:2037C0007A37E0FCA3E0FDA3E0FEA3E0FF780B120096F5C004C005C006C00790087A37E07A
:2037E000FCA3E0FDA3E0FEA3E0FF7815120096E2D003D002D001D000EF4BFFEE4AFEED4948
:20380000FDEC48FC90087A37120097E490087A37E0FCA3E0FDA3E0FEA3E0FF90087A2BE0E0
:20382000F8A3E0F9A3E0FAA3E0FBEF2BFFEE3AFEED39FDEC38FC90087A37120097E4900829
:203840007A33E0F8A3E0F9A3E0FAA3E0FBC000C001C002C00390087A28E0FBA3E0FAA3E051
:20386000243CF9E43AFA1200975DC000C001C00290087A2BE0FCA3E0FDA3E0FEA3E0FF9062
:20388000087A37E0F8A3E0F9A3E0FAA3E06FFFEA6EFEE96DFDE86CFC90087A2FE0F8A3E018
:2038A000F9A3E0FAA3E06FFFEA6EFEE96DFDE86CFCD002D001D000EF2BFFEE3AFEED39FDD3
:2038C000EC38FCEF24F8FFEE347CFEED34A2FDEC341FFCD003D002D001D000EB2FFFEA3EA0
:2038E000FEE93DFDE83CFCA3120097E490087A33E0FCA3E0FDA3E0FEA3E0FF781012009683
:20390000F5C004C005C006C00790087A33E0FCA3E0FDA3E0FEA3E0FF7810120096E2D00313
:20392000D002D001D000EF4BFFEE4AFEED49FDEC48FC90087A33120097E490087A33E0FC4F
:20394000A3E0FDA3E0FEA3E0FFA3E0F8A3E0F9A3E0FAA3E0FBEF2BFFEE3AFEED39FDEC386C
:20396000FC90087A33120097E490087A2FE0F8A3E0F9A3E0FAA3E0FBC000C001C002C003E3
:2039800090087A28E0FBA3E0FAA3E02408F9E43AFA1200975DC000C001C00290087A37E063
:2039A000FCA3E0FDA3E0FEA3E0FF90087A33E0F8A3E0F9A3E0FAA3E06FFFEA6EFEE96DFDD8
:2039C000E86CFC90087A2BE0F8A3E0F9A3E0FAA3E06FFFEA6EFEE96DFDE86CFCD002D001FC
:2039E000D000EF2BFFEE3AFEED39FDEC38FCEF2465FFEE3456FEED34ACFDEC34C4FCD0030B
:203A0000D002D001D000EB2FFFEA3EFEE93DFDE83CFCA3120097E490087A2FE0FCA3E0FDE4
:203A2000A3E0FEA3E0FF7817120096F5C004C005C006C00790087A2FE0FCA3E0FDA3E0FE23
:203A4000A3E0FF7809120096E2D003D002D001D000EF4BFFEE4AFEED49FDEC48FC90087AAF
:203A60002F120097E490087A2FE0FCA3E0FDA3E0FEA3E0FFA3E0F8A3E0F9A3E0FAA3E0FBF8
:203A8000EF2BFFEE3AFEED39FDEC38FC90087A2F120097E490087A2BE0F8A3E0F9A3E0FAC8
:203AA000A3E0FBC000C001C002C00390087A37E0FCA3E0FDA3E0FEA3E0FF120096AE9008EC
:203AC0007A2FE0F8A3E0F9A3E0FAA3E04FFFEA4EFEE94DFDE84CFCA3E0F8A3E0F9A3E0FA8E
:203AE000A3E06FFFEA6EFEE96DFDE86CFC90087A28E0FBA3E0FAA3E0F91200975DEF2BFFAF
:203B0000EE3AFEED39FDEC38FCEF2444FFEE3422FEED3429FDEC34F4FCD003D002D001D007
:203B200000EB2FFFEA3EFEE93DFDE83CFC90087A2B120097E490087A2BE0FCA3E0FDA3E01D
:203B4000FEA3E0FF7806120096F5C004C005C006C00790087A2BE0FCA3E0FDA3E0FEA3E017
:203B6000FF781A120096E2D003D002D001D000EF4BFFEE4AFEED49FDEC48FC90087A2B12C3
:203B80000097E490087A2BE0FCA3E0FDA3E0FEA3E0FFA3E0F8A3E0F9A3E0FAA3E0FBEF2B02
:203BA000FFEE3AFEED39FDEC38FC90087A2B120097E490087A37E0F8A3E0F9A3E0FAA3E036
:203BC000FBC000C001C002C00390087A33E0FCA3E0FDA3E0FEA3E0FF120096AE90087A2BAD
:203BE000E0F8A3E0F9A3E0FAA3E04FFFEA4EFEE94DFDE84CFCA3E0F8A3E0F9A3E0FAA3E093
:203C00006FFFEA6EFEE96DFDE86CFC90087A28E0FBA3E0FAA3E0241CF9E43AFA1200975DD1
:203C2000EF2BFFEE3AFEED39FDEC38FCEF2497FFEE34FFFEED342AFDEC3443FCD003D002EE
:203C4000D001D000EB2FFFEA3EFEE93DFDE83CFC90087A37120097E490087A37E0FCA3E0C3
:203C6000FDA3E0FEA3E0FF780A120096F5C004C005C006C00790087A37E0FCA3E0FDA3E0E7
:203C8000FEA3E0FF7816120096E2D003D002D001D000EF4BFFEE4AFEED49FDEC48FC9008DC
:203CA0007A37120097E490087A37E0FCA3E0FDA3E0FEA3E0FF90087A2BE0F8A3E0F9A3E00A
:203CC000FAA3E0FBEF2BFFEE3AFEED39FDEC38FC90087A37120097E490087A33E0F8A3E074
:203CE000F9A3E0FAA3E0FBC000C001C002C00390087A2FE0FCA3E0FDA3E0FEA3E0FF120018
:203D000096AE90087A37E0F8A3E0F9A3E0FAA3E04FFFEA4EFEE94DFDE84CFC90087A2BE0BE
:203D2000F8A3E0F9A3E0FAA3E06FFFEA6EFEE96DFDE86CFC90087A28E0FBA3E0FAA3E0246F
:203D400038F9E43AFA1200975DEF2BFFEE3AFEED39FDEC38FCEF24A7FFEE3423FEED3494E1
:203D6000FDEC34ABFCD003D002D001D000EB2FFFEA3EFEE93DFDE83CFC90087A33120097C9
:203D8000E490087A33E0FCA3E0FDA3E0FEA3E0FF780F120096F5C004C005C006C0079008C9
:203DA0007A33E0FCA3E0FDA3E0FEA3E0FF7811120096E2D003D002D001D000EF4BFFEE4A2D
:203DC000FEED49FDEC48FC90087A33120097E490087A33E0FCA3E0FDA3E0FEA3E0FFA3E089
:203DE000F8A3E0F9A3E0FAA3E0FBEF2BFFEE3AFEED39FDEC38FC90087A33120097E4900868
:203E00007A2FE0F8A3E0F9A3E0FAA3E0FBC000C001C002C00390087A2BE0FCA3E0FDA3E088
:203E2000FEA3E0FF120096AE90087A33E0F8A3E0F9A3E0FAA3E04FFFEA4EFEE94DFDE84C28
:203E4000FCA3E0F8A3E0F9A3E0FAA3E06FFFEA6EFEE96DFDE86CFC90087A28E0FBA3E0FA76
:203E6000A3E02414F9E43AFA1200975DEF2BFFEE3AFEED39FDEC38FCEF2439FFEE34A0FEE3
:203E8000ED3493FDEC34FCFCD003D002D001D000EB2FFFEA3EFEE93DFDE83CFC90087A2F50
:203EA000120097E490087A2FE0FCA3E0FDA3E0FEA3E0FF7815120096F5C004C005C006C09C
:203EC0000790087A2FE0FCA3E0FDA3E0FEA3E0FF780B120096E2D003D002D001D000EF4BAE
:203EE000FFEE4AFEED49FDEC48FC90087A2F120097E490087A2FE0FCA3E0FDA3E0FEA3E0BB
:203F0000FFA3E0F8A3E0F9A3E0FAA3E0FBEF2BFFEE3AFEED39FDEC38FC90087A2F12009744
:203F2000E490087A2BE0F8A3E0F9A3E0FAA3E0FBC000C001C002C00390087A37E0FCA3E063
:203F4000FDA3E0FEA3E0FF120096AE90087A2FE0F8A3E0F9A3E0FAA3E04FFFEA4EFEE94DBC
:203F6000FDE84CFCA3E0F8A3E0F9A3E0FAA3E06FFFEA6EFEE96DFDE86CFC90087A28E0FBA1
:203F8000A3E0FAA3E02430F9E43AFA1200975DEF2BFFEE3AFEED39FDEC38FCEF24C3FFEE71
:203FA0003459FEED345BFDEC3465FCD003D002D001D000EB2FFFEA3EFEE93DFDE83CFC9024
:203FC000087A2B120097E490087A2BE0FCA3E0FDA3E0FEA3E0FF7806120096F5C004C00567
:203FE000C006C00790087A2BE0FCA3E0FDA3E0FEA3E0FF781A120096E2D003D002D001D036
:2040000000EF4BFFEE4AFEED49FDEC48FC90087A2B120097E490087A2BE0FCA3E0FDA3E0E8
:20402000FEA3E0FFA3E0F8A3E0F9A3E0FAA3E0FBEF2BFFEE3AFEED39FDEC38FC90087A2B4F
:20404000120097E490087A37E0F8A3E0F9A3E0FAA3E0FBC000C001C002C00390087A33E010
:20406000FCA3E0FDA3E0FEA3E0FF120096AE90087A2BE0F8A3E0F9A3E0FAA3E04FFFEA4E54
:20408000FEE94DFDE84CFCA3E0F8A3E0F9A3E0FAA3E06FFFEA6EFEE96DFDE86CFC90087A4F
:2040A00028E0FBA3E0FAA3E0240CF9E43AFA1200975DEF2BFFEE3AFEED39FDEC38FCEF2421
:2040C00092FFEE34CCFEED340CFDEC348FFCD003D002D001D000EB2FFFEA3EFEE93DFDE8FE
:2040E0003CFC90087A37120097E490087A37E0FCA3E0FDA3E0FEA3E0FF780A120096F5C02B
:2041000004C005C006C00790087A37E0FCA3E0FDA3E0FEA3E0FF7816120096E2D003D002E4
:20412000D001D000EF4BFFEE4AFEED49FDEC48FC90087A37120097E490087A37E0FCA3E08E
:20414000FDA3E0FEA3E0FF90087A2BE0F8A3E0F9A3E0FAA3E0FBEF2BFFEE3AFEED39FDEC85
:2041600038FC90087A37120097E490087A33E0F8A3E0F9A3E0FAA3E0FBC000C001C002C09E
:204180000390087A2FE0FCA3E0FDA3E0FEA3E0FF120096AE90087A37E0F8A3E0F9A3E0FA0C
:2041A000A3E04FFFEA4EFEE94DFDE84CFC90087A2BE0F8A3E0F9A3E0FAA3E06FFFEA6EFE40
:2041C000E96DFDE86CFC90087A28E0FBA3E0FAA3E02428F9E43AFA1200975DEF2BFFEE3A83
:2041E000FEED39FDEC38FCEF247DFFEE34F4FEED34EFFDEC34FFFCD003D002D001D000EB82
:204200002FFFEA3EFEE93DFDE83CFC90087A33120097E490087A33E0FCA3E0FDA3E0FEA370
:20422000E0FF780F120096F5C004C005C006C00790087A33E0FCA3E0FDA3E0FEA3E0FF7849
:2042400011120096E2D003D002D001D000EF4BFFEE4AFEED49FDEC48FC90087A33120097BD
:20426000E490087A33E0FCA3E0FDA3E0FEA3E0FFA3E0F8A3E0F9A3E0FAA3E0FBEF2BFFEEBD
:204280003AFEED39FDEC38FC90087A33120097E490087A2FE0F8A3E0F9A3E0FAA3E0FBC081
:2042A00000C001C002C00390087A2BE0FCA3E0FDA3E0FEA3E0FF120096AE90087A33E0F8A9
:2042C000A3E0F9A3E0FAA3E04FFFEA4EFEE94DFDE84CFCA3E0F8A3E0F9A3E0FAA3E06FFF16
:2042E000EA6EFEE96DFDE86CFC90087A28E0FBA3E0FAA3E02404F9E43AFA1200975DEF2B57
:20430000FFEE3AFEED39FDEC38FCEF24D1FFEE345DFEED3484FDEC3485FCD003D002D0011C
:20432000D000EB2FFFEA3EFEE93DFDE83CFC90087A2F120097E490087A2FE0FCA3E0FDA31D
:20434000E0FEA3E0FF7815120096F5C004C005C006C00790087A2FE0FCA3E0FDA3E0FEA3FC
:20436000E0FF780B120096E2D003D002D001D000EF4BFFEE4AFEED49FDEC48FC90087A2FF8
:20438000120097E490087A2FE0FCA3E0FDA3E0FEA3E0FFA3E0F8A3E0F9A3E0FAA3E0FBEF0F
:2043A0002BFFEE3AFEED39FDEC38FC90087A2F120097E490087A2BE0F8A3E0F9A3E0FAA3EB
:2043C000E0FBC000C001C002C00390087A37E0FCA3E0FDA3E0FEA3E0FF120096AE90087AEC
:2043E0002FE0F8A3E0F9A3E0FAA3E04FFFEA4EFEE94DFDE84CFCA3E0F8A3E0F9A3E0FAA33C
:20440000E06FFFEA6EFEE96DFDE86CFC90087A28E0FBA3E0FAA3E02420F9E43AFA12009742
:204420005DEF2BFFEE3AFEED39FDEC38FCEF244FFFEE347EFEED34A8FDEC346FFCD003D0AA
:2044400002D001D000EB2FFFEA3EFEE93DFDE83CFC90087A2B120097E490087A2BE0FCA3B1
:20446000E0FDA3E0FEA3E0FF7806120096F5C004C005C006C00790087A2BE0FCA3E0FDA3EF
:20448000E0FEA3E0FF781A120096E2D003D002D001D000EF4BFFEE4AFEED49FDEC48FC90F8
:2044A000087A2B120097E490087A2BE0FCA3E0FDA3E0FEA3E0FFA3E0F8A3E0F9A3E0FAA30F
:2044C000E0FBEF2BFFEE3AFEED39FDEC38FC90087A2B120097E490087A37E0F8A3E0F9A375
:2044E000E0FAA3E0FBC000C001C002C00390087A33E0FCA3E0FDA3E0FEA3E0FF120096AE64
:2045000090087A2BE0F8A3E0F9A3E0FAA3E04FFFEA4EFEE94DFDE84CFCA3E0F8A3E0F9A389
:20452000E0FAA3E06FFFEA6EFEE96DFDE86CFC90087A28E0FBA3E0FAA3E0243CF9E43AFA31
:204540001200975DEF2BFFEE3AFEED39FDEC38FCEF24E0FFEE34E6FEED342CFDEC34FEFC77
:20456000D003D002D001D000EB2FFFEA3EFEE93DFDE83CFC90087A37120097E490087A3754
:20458000E0FCA3E0FDA3E0FEA3E0FF780A120096F5C004C005C006C00790087A37E0FCA3BF
:2045A000E0FDA3E0FEA3E0FF7816120096E2D003D002D001D000EF4BFFEE4AFEED49FDEC2F
:2045C00048FC90087A37120097E490087A37E0FCA3E0FDA3E0FEA3E0FF90087A2BE0F8A361
:2045E000E0F9A3E0FAA3E0FBEF2BFFEE3AFEED39FDEC38FC90087A37120097E490087A334A
:20460000E0F8A3E0F9A3E0FAA3E0FBC000C001C002C00390087A2FE0FCA3E0FDA3E0FEA384
:20462000E0FF120096AE90087A37E0F8A3E0F9A3E0FAA3E04FFFEA4EFEE94DFDE84CFC9031
:20464000087A2BE0F8A3E0F9A3E0FAA3E06FFFEA6EFEE96DFDE86CFC90087A28E0FBA3E05A
:20466000FAA3E02418F9E43AFA1200975DEF2BFFEE3AFEED39FDEC38FCEF2414FFEE34435D
:20468000FEED3401FDEC34A3FCD003D002D001D000EB2FFFEA3EFEE93DFDE83CFC90087A64
:2046A00033120097E490087A33E0FCA3E0FDA3E0FEA3E0FF780F120096F5C004C005C00623
:2046C000C00790087A33E0FCA3E0FDA3E0FEA3E0FF7811120096E2D003D002D001D000EF27
:2046E0004BFFEE4AFEED49FDEC48FC90087A33120097E490087A33E0FCA3E0FDA3E0FEA340
:20470000E0FFA3E0F8A3E0F9A3E0FAA3E0FBEF2BFFEE3AFEED39FDEC38FC90087A331200EF
:2047200097E490087A2FE0F8A3E0F9A3E0FAA3E0FBC000C001C002C00390087A2BE0FCA3AC
:20474000E0FDA3E0FEA3E0FF120096AE90087A33E0F8A3E0F9A3E0FAA3E04FFFEA4EFEE91D
:204760004DFDE84CFCA3E0F8A3E0F9A3E0FAA3E06FFFEA6EFEE96DFDE86CFC90087A28E047
:20478000FBA3E0FAA3E02434F9E43AFA1200975DEF2BFFEE3AFEED39FDEC38FCEF24A1FF7A
:2047A000EE3411FEED3408FDEC344EFCD003D002D001D000EB2FFFEA3EFEE93DFDE83CFC70
:2047C00090087A2F120097E490087A2FE0FCA3E0FDA3E0FEA3E0FF7815120096F5C004C0BD
:2047E00005C006C00790087A2FE0FCA3E0FDA3E0FEA3E0FF780B120096E2D003D002D00104
:20480000D000EF4BFFEE4AFEED49FDEC48FC90087A2F120097E490087A2FE0FCA3E0FDA3E8
:20482000E0FEA3E0FFA3E0F8A3E0F9A3E0FAA3E0FBEF2BFFEE3AFEED39FDEC38FC90087A92
:204840002F120097E490087A2BE0F8A3E0F9A3E0FAA3E0FBC000C001C002C00390087A37C1
:20486000E0FCA3E0FDA3E0FEA3E0FF120096AE90087A2FE0F8A3E0F9A3E0FAA3E04FFFEAB6
:204880004EFEE94DFDE84CFCA3E0F8A3E0F9A3E0FAA3E06FFFEA6EFEE96DFDE86CFC900873
:2048A0007A28E0FBA3E0FAA3E02410F9E43AFA1200975DEF2BFFEE3AFEED39FDEC38FCEFBF
:2048C0002482FFEE347EFEED3453FDEC34F7FCD003D002D001D000EB2FFFEA3EFEE93DFD69
:2048E000E83CFC90087A2B120097E490087A2BE0FCA3E0FDA3E0FEA3E0FF7806120096F517
:20490000C004C005C006C00790087A2BE0FCA3E0FDA3E0FEA3E0FF781A120096E2D003D026
:2049200002D001D000EF4BFFEE4AFEED49FDEC48FC90087A2B120097E490087A2BE0FCA37C
:20494000E0FDA3E0FEA3E0FFA3E0F8A3E0F9A3E0FAA3E0FBEF2BFFEE3AFEED39FDEC38FC03
:2049600090087A2B120097E490087A37E0F8A3E0F9A3E0FAA3E0FBC000C001C002C003903F
:20498000087A33E0FCA3E0FDA3E0FEA3E0FF120096AE90087A2BE0F8A3E0F9A3E0FAA3E01C
:2049A0004FFFEA4EFEE94DFDE84CFCA3E0F8A3E0F9A3E0FAA3E06FFFEA6EFEE96DFDE86CAE
:2049C000FC90087A28E0FBA3E0FAA3E0242CF9E43AFA1200975DEF2BFFEE3AFEED39FDEC11
:2049E00038FCEF2435FFEE34F2FEED343AFDEC34BDFCD003D002D001D000EB2FFFEA3EFE74
:204A0000E93DFDE83CFC90087A37120097E490087A37E0FCA3E0FDA3E0FEA3E0FF780A1241
:204A20000096F5C004C005C006C00790087A37E0FCA3E0FDA3E0FEA3E0FF7816120096E215
:204A4000D003D002D001D000EF4BFFEE4AFEED49FDEC48FC90087A37120097E490087A371F
:204A6000E0FCA3E0FDA3E0FEA3E0FF90087A2BE0F8A3E0F9A3E0FAA3E0FBEF2BFFEE3AFE0C
:204A8000ED39FDEC38FC90087A37120097E490087A33E0F8A3E0F9A3E0FAA3E0FBC000C0E9
:204AA00001C002C00390087A2FE0FCA3E0FDA3E0FEA3E0FF120096AE90087A37E0F8A3E0D6
:204AC000F9A3E0FAA3E04FFFEA4EFEE94DFDE84CFC90087A2BE0F8A3E0F9A3E0FAA3E06FF6
:204AE000FFEA6EFEE96DFDE86CFC90087A28E0FBA3E0FAA3E02408F9E43AFA1200975DEF77
:204B00002BFFEE3AFEED39FDEC38FCEF24BBFFEE34D2FEED34D7FDEC342AFCD003D002D093
:204B200001D000EB2FFFEA3EFEE93DFDE83CFC90087A33120097E490087A33E0FCA3E0FDAF
:204B4000A3E0FEA3E0FF780F120096F5C004C005C006C00790087A33E0FCA3E0FDA3E0FEF6
:204B6000A3E0FF7811120096E2D003D002D001D000EF4BFFEE4AFEED49FDEC48FC90087A76
:204B800033120097E490087A33E0FCA3E0FDA3E0FEA3E0FFA3E0F8A3E0F9A3E0FAA3E0FBBF
:204BA000EF2BFFEE3AFEED39FDEC38FC90087A33120097E490087A2FE0F8A3E0F9A3E0FA8F
:204BC000A3E0FBC000C001C002C00390087A2BE0FCA3E0FDA3E0FEA3E0FF120096AE9008C7
:204BE0007A33E0F8A3E0F9A3E0FAA3E04FFFEA4EFEE94DFDE84CFCA3E0F8A3E0F9A3E0FA59
:204C0000A3E06FFFEA6EFEE96DFDE86CFC90087A28E0FBA3E0FAA3E02424F9E43AFA12002A
:204C2000975DEF2BFFEE3AFEED39FDEC38FCEF2491FFEE34D3FEED3486FDEC34EBFCD003EA
:204C4000D002D001D000EB2FFFEA3EFEE93DFDE83CFC90087A2F120097E490087A2FE0FC74
:204C6000A3E0FDA3E0FEA3E0FF7815120096F5C004C005C006C00790087A2FE0FCA3E0FDD4
:204C8000A3E0FEA3E0FF780B120096E2D003D002D001D000EF4BFFEE4AFEED49FDEC48FCEC
:204CA00090087A2F120097E490087A2FE0FCA3E0FDA3E0FEA3E0FFA3E0F8A3E0F9A3E0FA12
:204CC000A3E0FBEF2BFFEE3AFEED39FDEC38FC90087A2F120097E490087A25E0FBA3E0FA77
:204CE000A3E0F9C002C0011200970890087A2BE0F8A3E0F9A3E0FAA3E02FFFEA3EFEE93DF9
:204D0000FDE83CFCD001D0021200972590087A25E0FBA3E0FAA3E02404F9E43AFAC002C038
:204D2000011200970890087A2FE0F8A3E0F9A3E0FAA3E02FFFEA3EFEE93DFDE83CFCD001C4
:204D4000D0021200972590087A25E0FBA3E0FAA3E02408F9E43AFAC002C0011200970890A0
:204D6000087A33E0F8A3E0F9A3E0FAA3E02FFFEA3EFEE93DFDE83CFCD001D0021200972522
:204D800090087A25E0FBA3E0FAA3E0240CF9E43AFAC002C0011200970890087A37E0F8A3C8
:204DA000E0F9A3E0FAA3E02FFFEA3EFEE93DFDE83CFCD001D00202009725900847D9E0FB8F
:204DC000A3E0FAA3E02414F9E43AFA900847D6EBF0A3EAF0A3E9F090084B23E0FBA3E0FAA3
:204DE000A3E02424F9E43AFA90084E37EBF0A3EAF0A3E9F090084B23A3E0FAA3E02423F9A0
:204E0000E43AFA90084B2BEBF0A3EAF0A3E9F090084B23A3E0FAA3E02418F9E43AFA9008AD
:204E20004E29EBF0A3EAF0A3E9F090084B23A3E0FAA3E0241AF9E43AFA90084B28EBF0A349
:204E4000EAF0A3E9F090084B23A3E0FAA3E0241CF9E43AFA90084E34EBF0A3EAF0A3E9F0B7
:204E600090084B23A3E0FAA3E0241EF9E43AFA90084E2CEBF0A3EAF0A3E9F090084A3EE0F3
:204E8000FD30E65490084E37E0FBA3E0FAA3E0F9E41200941B90084E37E0FBA3E0FAA3E01D
:204EA0002402F9E43AFAE4F5F01200957590084E29E0FBA3E0FAA3E0F9E475F00112009502
:204EC0007590084E34E0FBA3E0FAA3E0F9E475F00112009575216068ED30E70321606890A0
:204EE000084A3EE020E103215E7790084E37E0FBA3E0FAA3E0F9120093CA6003215E7790FF
:204F000008844B7481F0A374ADF0A37448F0A3E4F0A37404F0900847D6E0FBA3E0FAA3E0C0
:204F2000F9120558E7EF6003214FB2900874FDF0900847D6E0FBA3E0FAA3E02405F9E43AE5
:204F4000FA900874FDE0FF7C0029F9EC3AFAA3EBF0A3EAF0A3E9F0120093CAFE64206004E5
:204F6000EEB43F1174012FF582E43475F583759308E4F08019900874FDE0FF04F074012F22
:204F8000F582E43475F583759308EEF080A27B097A7579011200B564EF4E60032150517893
:204FA000017C757D097B817AAD794D12009ACC215051900880667481F0A374ADF0A37457D1
:204FC000F0900847D6E0FBA3E0FAA3E0F912051DE2900874FEEBF0A3EAF0A3E9F090087458
:204FE000FEE0FBA3E0FAA3E04A4B701C90084E2FE064037003215424900847D6E0FBA3E03C
:20500000FAA3E0F902035C3890087A687481F0A374ADF0A37457F0A37481F0A374ADF0A331
:205020007461F0A37409F0A37475F0A37401F0900874FEE0FBA3E0FAA3E0F912049F5090A4
:20504000084E37E0FBA3E0FAA3E0F974011200941B9008844B7481F0A374ADF0A37463F04F
:20506000A3E4F0A3740AF07B097A757901120558E7EF704990084B23E0FBA3E0FAA3E024B8
:2050800004F9E43AFA1200970890084E30E0F8A3E0F9A3E0FAA3E0FBC3120096D170032115
:2050A0005133E4FFFEFDFC90084E30E0F8A3A3A3E0C3120096D1600321522A80769008848D
:2050C0004B7481F0A374ADF0A3746EF0A3E4F0A3740AF07B097A757901120558E7EF70103D
:2050E00078017C757D097B817AAD797912009ACC9008844B7481F0A374ADF0A37486F0A303
:20510000E4F0A37404F07B097A757901120558E7EF70032151E9900882D17409F0A37474CD
:20512000F0A374F8F07B097A75790112051631EF4E702078017C757D097B817AAD798B123F
:20514000009ACC90084E2F7401F0E4FFFEFDFCA32153D290084E37E0FBA3E0FAA3E0F97447
:20516000021200941B900874F8E0FBA3E0FAA3E0F9C003C002C00190084E37E0FBA3E0FAD9
:20518000A3E02404F9E43AFA1200982A900874FBE0FEA3E0FF90084E37E0FBA3E0FAA3E020
:2051A0002402F9E43AFAEE8FF01200957512059DC5C004C005C006C0071205A09DE4FCFD6F
:2051C0007B587A02F9F812009591D003D002D001D000EB2FFFEA3EFEE93DFDE83CFC9008F7
:2051E0004B2E120097E4215F9B90084B23E0FBA3E0FAA3E02404F9E43AFA1200970890082B
:205200004E30E0F8A3E0F9A3E0FAA3E0FBC3120096D1603EE4FFFEFDFC90084E30E0F8A37C
:20522000A3A3E0C3120096D16028900882AD7481F0A374ADF0A3749BF0A37481F0A374AD36
:20524000F0A3748BF07B817AAD799512053E5321606890084E37E0FBA3E0FAA3E0F9120007
:2052600093CA640160032153D99008844B7481F0A374ADF0A374B3F0A3E4F0A3740AF07BFF
:20528000097A757901120558E7EF60032153D9900847D6E0FBA3E0FAA3E0F91205420EEFC8
:2052A0004E600321537912059E15E4FBFAF9F8C3120096D1604512059E25EF5402FFE4FEDB
:2052C000FDFC7B02FAF9F8C3120096D1702D90084B23E0FBA3E0FAA3E02404F9E43AFA1268
:2052E000009708900883E2120097E4E4900883E6F0A3F07FEA7E03120434D11205A0EEEF84
:205300004E604E1205A080EF4E604612059EB5EF5402FFE4FEFDFC7B02FAF9F8C31200961B
:20532000D1702E90084B23E0FBA3E0FAA3E02404F9E43AFA12009708900883E2120097E4A9
:20534000900883E6E4F0A304F07FEA7E03120434D1900882AD7481F0A374ADF0A374BEF0B7
:20536000A37481F0A374ADF0A3748BF07B817AAD799512053E5321606890084B23E0FBA319
:20538000E0FAA3E02404F9E43AFA1200970890084E30120097E490084E2F7402F012059DF4
:2053A000C5C004C005C006C0071205A09DE4FCFD7B587A02F9F812009591D003D002D001F3
:2053C000D000EB2FFFEA3EFEE93DFDE83CFC90084B2E120097E4215B189008844B7481F0FD
:2053E000A374ADF0A3748BF0A3E4F0A37409F07B097A757901120558E7EF700990084E2F20
:2054000004F0215B1890084E2FE0B4010F78017C757D097B817AAD798B215ADD90084E2FC7
:20542000E0B40339900882AD7481F0A374ADF0A374CDF0A37481F0A374ADF0A3748BF07B1F
:20544000817AAD799512053E5390084E2F7401F0E4FFFEFDFCA3120097E421606890084E9B
:2054600037E0FBA3E0FAA3E0F9120093CA64016003215B189008844B7481F0A374ADF0A3B3
:2054800074DBF0A3E4F0A37408F07B097A757901120558E7EF701A900847D6E0FBA3E0FA7E
:2054A000A3E0F912040C5CEF4E6003215B18215ACD9008844B7481F0A374ADF0A374E4F08B
:2054C000A3E4F0A37407F07B097A757901120558E7EF701A900847D6E0FBA3E0FAA3E0F902
:2054E00012057DB7EF4E6003215B18215ACD9008844B7481F0A374ADF0A374ECF0A3E4F07B
:20550000A3740AF07B097A757901120558E7EF701A900847D6E0FBA3E0FAA3E0F91204CB54
:20552000DEEF4E6003215B18215ACD9008844B7481F0A374ADF0A374F7F0A3E4F0A374077E
:20554000F07B097A757901120558E7EF701A900847D6E0FBA3E0FAA3E0F91204C597EF4E67
:205560006003215B18215ACD9008844B7481F0A374ADF0A374FFF0A3E4F0A37409F07B09DB
:205580007A757901120558E7EF701A900847D6E0FBA3E0FAA3E0F91204E125EF4E6003216D
:2055A0005B18215ACD9008844B7481F0A374AEF0A37409F0A3E4F0A3740BF07B097A7579AA
:2055C00001120558E7EF7026900847D6E0FBA3E0FAA3E0F9120473ABEF4E7003215ACD78C2
:2055E000017C757D097B817AAE7915215ADD9008844B7481F0A374AEF0A37415F0A3E4F095
:20560000A37408F07B097A757901120558E7EF701A900847D6E0FBA3E0FAA3E0F9120443DD
:205620004EEF4E6003215B18215ACD9008844B7481F0A374AEF0A3741EF0A3E4F0A37409E3
:20564000F07B097A757901120558E7EF701A900847D6E0FBA3E0FAA3E0F91203C416EF4EE9
:205660006003215B18215ACD9008844B7481F0A374AEF0A37428F0A3E4F0A3740AF07B09AF
:205680007A757901120558E7EF701A900847D6E0FBA3E0FAA3E0F912048742EF4E600321A9
:2056A0005B18215ACD9008844B7481F0A374AEF0A37433F0A3E4F0A37411F07B097A757979
:2056C00001120558E7EF701A900847D6E0FBA3E0FAA3E0F9120501F7EF4E6003215B18210D
:2056E0005ACD9008844B7481F0A374AEF0A37445F0A3E4F0A37407F07B097A7579011205AD
:2057000058E7EF701A900847D6E0FBA3E0FAA3E0F912029E06EF4E6003215B18215ACD9084
:2057200008844B7481F0A374AEF0A3744DF0A3E4F0A37407F07B097A757901120558E7EFED
:20574000701A900847D6E0FBA3E0FAA3E0F91202AEB6EF4E6003215B18215ACD9008844BDB
:205760007481F0A374AEF0A37455F0A3E4F0A37408F07B097A757901120558E7EF701A9061
:205780000847D6E0FBA3E0FAA3E0F9120471EBEF4E6003215B18215ACD9008844B7481F0D6
:2057A000A374AEF0A3745EF0A3E4F0A37408F07B097A757901120558E7EF701A900847D6D8
:2057C000E0FBA3E0FAA3E0F912037D7AEF4E6003215B18215ACD9008844B7481F0A374AE5C
:2057E000F0A37467F0A3E4F0A3740DF07B097A757901120558E7EF7026900847D6E0FBA3C5
:20580000E0FAA3E0F91204EF0BEF4E7003215ACD78017C757D097B817AAE7975215ADD9040
:2058200008844B7481F0A374AEF0A37483F0A3E4F0A37410F07B097A757901120558E7EFAD
:20584000701A900847D6E0FBA3E0FAA3E0F9120562A9EF4E6003215B18215ACD9008844B30
:205860007481F0A374AEF0A37494F0A3E4F0A37410F07B097A757901120558E7EF7026900D
:205880000847D6E0FBA3E0FAA3E0F912021CFAEF4E7003215ACD78017C757D097B817AAED9
:2058A0007975215ADD9008844B7481F0A374AEF0A374A5F0A3E4F0A37410F07B097A75797B
:2058C00001120558E7EF7026900847D6E0FBA3E0FAA3E0F91203F5BBEF4E7003215ACD782E
:2058E000017C757D097B817AAE7975215ADD9008844B7481F0A374AEF0A374B6F0A3E4F091
:20590000A37411F07B097A757901120558E7EF7026900847D6E0FBA3E0FAA3E0F91202C941
:2059200036EF4E7003215ACD78017C757D097B817AAE79C8215ADD9008844B7481F0A37429
:20594000AEF0A374D7F0A3E4F0A37411F07B097A757901120558E7EF7026900847D6E0FBE4
:20596000A3E0FAA3E0F912032B8AEF4E7003215ACD78017C757D097B817AAE79C8215ADDBF
:205980009008844B7481F0A374AEF0A374E9F0A3E4F0A3740CF07B097A757901120558E749
:2059A000EF7026900847D6E0FBA3E0FAA3E0F91204BDAFEF4E7003215ACD78017C757D096F
:2059C0007B817AAE7915215ADD9008844B7481F0A374AEF0A374F6F0A3E4F0A37408F07BBE
:2059E000097A757901120558E7EF701A900847D6E0FBA3E0FAA3E0F912042E73EF4E600386
:205A0000215B18215ACD9008844B7481F0A374AEF0A374FFF0A3E4F0A3740AF07B097A75A8
:205A20007901120558E7EF7026900847D6E0FBA3E0FAA3E0F91203C701EF4E7003215ACDB3
:205A400078017C757D097B817AAF790A215ADD9008844B7481F0A374AFF0A37412F0A3E4B4
:205A6000F0A3740AF07B097A757901120558E7EF7024900847D6E0FBA3E0FAA3E0F91203C1
:205A80009F25EF4E7002804578017C757D097B817AAF790A80479008844B7481F0A374AF5D
:205AA000F0A3741DF0A3E4F0A3740AF07B097A757901120558E7EF702A900847D6E0FBA34B
:205AC000E0FAA3E0F912046586EF4E7004FE7F012278017C757D097B817AAF790A12009ADA
:205AE000CC80359008844B7481F0A374AFF0A37428F0A3E4F0A37409F07B097A757901126E
:205B00000558E7EF701290086E75F0A304F090084A3E7410F02160689008844B7481F0A362
:205B200074AEF0A37415F0A3E4F0A37408F07B097A757901120558E7EF70181205A0A6EFAB
:205B40004E701078017C757D097B817AAF790A12009ACCE4900874FDF09008844B7481F03E
:205B6000A374AFF0A37432F0A3E4F0A3740BF07B097A757901120558E7EF701412055BEA9B
:205B800078017C757D097B817AAF793E12009ACC9008844B7481F0A374AFF0A3744AF0A3CB
:205BA000E4F0A3740BF07B097A757901120558E7EF701A900887AAF0A304F078017C757D0C
:205BC000097B817AAF795612009ACC8008E4900887AAF0A3F0E490088618F0A3F0900884DF
:205BE0004B7481F0A374AEF0A374FFF0A3E4F0A3740AF07B097A757901120558E7EF70454B
:205C0000900873F67481F0A374AFF0A37462F0A37409F0A37486F0A37418F07B097A7579D7
:205C2000011200AA7978017C757D097B817AAF790A12009ACC90088619E024FFF0900886D6
:205C400018E034FFF09008844B7481F0A374AFF0A37470F0A3E4F0A37411F07B097A757935
:205C600001120558E7EF7017900886FEF0A304F078017C757D097B817AAE79B6215DC6909D
:205C800008844B7481F0A374AEF0A374B6F0A3E4F0A37411F07B097A757901120558E7EF15
:205CA0007003215D869008844B7481F0A374AEF0A374D7F0A3E4F0A37411F07B097A757913
:205CC00001120558E7EF7003215D869008844B7481F0A374AEF0A374C8F0A3E4F0A3740E9B
:205CE000F07B097A757901120558E7EF7016900886FCF0A3F078017C757D097B817AAF79D1
:205D000082215DC69008844B7481F0A374AFF0A3748BF0A3E4F0A37410F07B097A757901AE
:205D2000120558E7EF7017900886FEF0A304F078017C757D097B817AAE7994215DC69008F7
:205D4000844B7481F0A374AEF0A37494F0A3E4F0A37410F07B097A757901120558E7EF700F
:205D60000280239008844B7481F0A374AEF0A374A5F0A3E4F0A37410F07B097A7579011244
:205D80000558E7EF7009900886FEF0A3F0803B9008844B7481F0A374AEF0A37475F0A3E4F9
:205DA000F0A3740DF07B097A757901120558E7EF7018900886FCF0A304F078017C757D0994
:205DC0007B817AAF798212009ACC900874FDE0FD75F017A42432F582E5F0344BF583759384
:205DE00008E0FBA3E0FAA3E04A4B700A90084A3E7410F0216068ED75F017A42435F9744B16
:205E000035F0FA7B091200B5649008844EEEF0A3EFF0900874FDE075F017A42435F9744BD0
:205E200035F0FA9008844B7409F0A3EAF0A3E9F07B097A757901120558E7EF703090084EBE
:205E400037E0FBA3E0FAA3E0F974031200941B900874FDE0FF90084E37E0FBA3E0FAA3E01F
:205E60002401F9E43AFAEF1200941B800A900874FDE004F0215DCA90084E37E0FBA3E0FA18
:205E8000A3E0F9120093CA64036003215F9B90084B26F0A3F090084A3EE0B4043C90084BCF
:205EA00028E0FBA3E0FAA3E0F9120094FBFF90084E29E0FBA3E0FAA3E0F9E5F08FF01200FD
:205EC000957590084E2CE0FBA3E0FAA3E0F9120094FBFF90084E34803A90084E29E0FBA3D1
:205EE000E0FAA3E0F9120094FBFF90084B28E0FBA3E0FAA3E0F9E5F08FF0120095759008C5
:205F00004E34E0FBA3E0FAA3E0F9120094FBFF90084E2CE0FBA3E0FAA3E0F9E5F08FF0123F
:205F200000957590084E37E0FBA3E0FAA3E02401F9E43AFA120093CA75F017A42432F582CD
:205F4000E5F0344BF583759308E0FBA3E0FAA3E0F912009911EF600790084A3E7410F012D9
:205F6000059DC5C004C005C006C0071205A09DE4FCFD7B587A02F9F812009591D003D00256
:205F8000D001D000EB2FFFEA3EFEE93DFDE83CFC90084B2E120097E421606890084A3EE057
:205FA00030E07A90084E37E0FBA3E0FAA3E02402F9E43AFA120094FBC39478E5F09405400A
:205FC0002A74FA75F0881200954990084E37E0FBA3E0FAA3E02404F9E43AFA09E970010AAE
:205FE000740575F07812009549803290084E37E0FBA3E0FAA3E02402F9E43AFAE4F5F0129F
:2060000000957590084E37E0FBA3E0FAA3E0F9120093CAB4020790084A3E7410F090084EDF
:2060200037E0FBA3E0FAA3E02402F9E43AFA120094FBFFAEF0D39478EE940590084B26402A
:20604000097405F0A37478F08005EEF0A3EFF090084E37E0FBA3E0FAA3E02404F9E43AFA39
:206060001200980D1205948F7E007F012278057C577D097B817A90790C7E007F3D120093CF
:206080004C78427C577D097B817A9079497E007F2F1200934C90084E29E0FBA3E0FAA3E0D2
:2060A000F9E475F0011200951FAFF0FE6003216F18EF24FE700321619C14700321659B14D1
:2060C00070032168AD147003216C1B24046003216F18900880667487F0A37484F0A374F0BA
:2060E000F0900847D6E0FBA3E0FAA3E0F912051DE29008582DEBF0A3EAF0A3E9F090085830
:206100002DE0FBA3E0FAA3E04A4B70037F0122900873F67487F0A37484F0A374F8F0A37440
:2061200009F0A37458F0A37430F09008582DE0FBA3E0FAA3E0F91200AA799008754C748756
:20614000F0A37485F0A37402F090085830E0FEA3E0FF9008754FEEF0A3EFF02401FFE43E38
:20616000A3F0A3EFF0900847D6E0FBA3E0FAA3E0F91200A69A90084B26EEF0A3EFF090082E
:206180005830E0F9A3E0FF90084E34E0FBA3E0FAA3E0C98FF012009575216F1B90084E34FE
:2061A000E0FBA3E0FAA3E0F9120094FBFF7B097A5879401204B2D990084E34E0FBA3E0FA49
:2061C000A3E0F9120094FBFF12059BE9EF64044E701B90084E34E0FBA3E0FAA3E0F91200D8
:2061E00094FBFF120594D8EF4E7002803490084E34E0FBA3E0FAA3E0F9120094FBFF120586
:206200009BE9EF64034E702A90084E34E0FBA3E0FAA3E0F9120094FBFF120594D8EF4E70FE
:2062200011FE7FBCFD7B097A57797112009C8A2162CA7E007FBC7D007B097A5779711200CC
:206240009C8A90084E34E0FBA3E0FAA3E0F9120094FBFF7B097A577971900885E27401F0E7
:2062600012059F0390084E34E0FBA3E0FAA3E0F9120094FBFF7B097A577971900885E27425
:2062800003F012059F0390084E34E0FBA3E0FAA3E0F9120094FBFF7B097A57797190088568
:2062A000E27405F012059F0390084E34E0FBA3E0FAA3E0F9120094FBFF7B097A577971907D
:2062C0000885E27406F012059F0390085840E0C4F854F0C8A3E0C4540F48540F64077026FE
:2062E000FFFEFDFC90085809120097E4E4FFFEFDFC9008578D120097E4E4FFFEFDFC9008CD
:206300005819120097E49008754C7409F0A37457F0A37405F0A37487F0A37486F0A3741B02
:20632000F090085809E0FCA3E0FDA3E0FEA3E0FF90087552120097E4900847D6E0FBA3E016
:20634000FAA3E0F91200A69A90084B26EEF0A3EFF0900847D6E0FBA3E0FAA3E0F990084BA0
:2063600026E0FEA3E0FFE92FF9EA3EFAC0039008754C7487F0A37486F0A3741EF0900857BC
:206380008DE0FCA3E0FDA3E0FEA3E0FF9008754F120097E490085819E0FCA3E0FDA3E0FE42
:2063A000A3E0FF90087553120097E4D0031200A69A90084B27E02FF090084B26E03EF09099
:2063C000085830E4F0A304F090085830E0FEA3E0FFD39403EE648094804003216F1BEE60B6
:2063E000032164B5EF24FE604514607D240260032164B5900858327487F0A37486F0A37445
:2064000089F090085795E0FCA3E0FDA3E0FEA3E0FF90085838120097E4900858357487F05B
:20642000A37486F0A37497F0900857C98074900858327487F0A37486F0A374A3F090085752
:2064400091E0FCA3E0FDA3E0FEA3E0FF90085838120097E4900858357487F0A37486F0A357
:2064600074B1F0900857CD8039900858327487F0A37486F0A374C4F090085799E0FCA3E046
:20648000FDA3E0FEA3E0FF90085838120097E4900858357487F0A37486F0A374D9F0900832
:2064A00057D1E0FCA3E0FDA3E0FEA3E0FF9008583C120097E490085840E0C4F854F0C8A321
:2064C000E0C4540F48540F64077019FFFEFDFC90085838120097E4E4FFFEFDFC9008583C65
:2064E000120097E4900847D6E0FBA3E0FAA3E0F990084B26E0FEA3E0FFE92FF9EA3EFAC02A
:2065000003C002C0019008754C7409F0A37457F0A37442F090085832E0F9A3E0FAA3E090FD
:2065200008754FC9F0A3EAF0A3E9F090085838E0FCA3E0FDA3E0FEA3E0FF900875521200E5
:2065400097E490085835E0F9A3E0FAA3E090087556C9F0A3EAF0A3E9F09008583CE0FCA302
:20656000E0FDA3E0FEA3E0FF90087559120097E4D001D002D0031200A69A90084B27E02F67
:20658000F090084B26E03EF090085831E004F0700790085830E004F02163C890084E34E04E
:2065A000FBA3E0FAA3E0F9120094FBFF12059BE9EF64044E701B90084E34E0FBA3E0FAA367
:2065C000E0F9120094FBFF120594D8EF4E7002803490084E34E0FBA3E0FAA3E0F9120094C8
:2065E000FBFF12059BE9EF64034E702990084E34E0FBA3E0FAA3E0F9120094FBFF12059490
:20660000D8EF4E7010FE7FBCFD7B097A57797112009C8A80547E007FBC7D007B097A577960
:206620007112009C8A90084E34E0FBA3E0FAA3E0F9120094FBFF7B097A577971900885E2E5
:206640007403F012059F0390084E34E0FBA3E0FAA3E0F9120094FBFF7B097A5779719008B5
:2066600085E27406F012059F0390085830E4F0A304F090085830E0FEA3E0FFD39404EE64C8
:206680008094804003216F1BEE60032167C7EF24FE604E14700321671C1470032167622459
:2066A0000360032167C7900858327487F0A37486F0A374EDF09008581DE0FCA3E0FDA3E0AB
:2066C000FEA3E0FF90085838120097E4900858357487F0A37486F0A374FDF0900857D580A0
:2066E00074900858327487F0A37487F0A37411F090085821E0FCA3E0FDA3E0FEA3E0FF9073
:20670000085838120097E4900858357487F0A37487F0A37425F0900857D9803990085832E7
:206720007487F0A37487F0A3743AF090085825E0FCA3E0FDA3E0FEA3E0FF900858381200F1
:2067400097E4900858357487F0A37487F0A3744DF0900857DDE0FCA3E0FDA3E0FEA3E0FFA1
:20676000805D900858327487F0A37487F0A37463F090085829E0FCA3E0FDA3E0FEA3E0FFBF
:2067800090085838120097E4900858357487F0A37487F0A37471F0900857E5E0FCA3E0FDFE
:2067A000A3E0FEA3E0FF900857E1E0F8A3E0F9A3E0FAA3E02FFFEA3EFEE93DFDE83CFC908B
:2067C00008583C120097E490085840E0C4F854F0C8A3E0C4540F48540F64077019FFFEFD75
:2067E000FC90085838120097E4E4FFFEFDFC9008583C120097E4900847D6E0FBA3E0FAA3A5
:20680000E0F990084B26E0FEA3E0FFE92FF9EA3EFAC003C002C0019008754C7409F0A374E0
:2068200057F0A37442F090085832E0F9A3E0FAA3E09008754FC9F0A3EAF0A3E9F0900858CF
:2068400038E0FCA3E0FDA3E0FEA3E0FF90087552120097E490085835E0F9A3E0FAA3E09027
:20686000087556C9F0A3EAF0A3E9F09008583CE0FCA3E0FDA3E0FEA3E0FF90087559120090
:2068800097E4D001D002D0031200A69A90084B27E02FF090084B26E03EF090085831E00490
:2068A000F0700790085830E004F021667290084E34E0FBA3E0FAA3E0F9120094FBFF1205DF
:2068C0009BE9EF64044E701B90084E34E0FBA3E0FAA3E0F9120094FBFF120594D8EF4E7046
:2068E00002803490084E34E0FBA3E0FAA3E0F9120094FBFF12059BE9EF64034E70299008E4
:206900004E34E0FBA3E0FAA3E0F9120094FBFF120594D8EF4E7010FE7FBCFD7B097A57793D
:206920007112009C8A80757E007FBC7D007B097A57797112009C8A90084E34E0FBA3E0FA9A
:20694000A3E0F9120094FBFF7B097A577971E4900885E2F012059F0390084E34E0FBA3E0D8
:20696000FAA3E0F9120094FBFF7B097A577971900885E27402F012059F0390084E34E0FBAF
:20698000A3E0FAA3E0F9120094FBFF7B097A577971900885E27405F012059F039008754CA5
:2069A0007409F0A37457F0A37405F0A37487F0A37487F0A37486F090085811E0FCA3E0FDFA
:2069C000A3E0FEA3E0FF90087552120097E4900847D6E0FBA3E0FAA3E0F91200A69A900855
:2069E0004B26EEF0A3EFF090085830E4F0A304F090085830E0FEA3E0FFD39405EE648094E9
:206A0000804003216F1BEE6003216B64EF24FE6055147003216AA2147003216ADD147003D7
:206A2000216B1824046003216B64900858327487F0A37487F0A37489F090085771E0FCA32D
:206A4000E0FDA3E0FEA3E0FF90085838120097E4900858357487F0A37487F0A37495F090D7
:206A60000857C1216B51900858327487F0A37486F0A37489F090085779E0FCA3E0FDA3E0A8
:206A8000FEA3E0FF90085838120097E4900858357487F0A37487F0A374A5F0900857C521A2
:206AA0006B51900858327487F0A37486F0A374A3F090085775E0FCA3E0FDA3E0FEA3E0FF13
:206AC00090085838120097E4900858357487F0A37486F0A37497F09008579D807490085856
:206AE000327487F0A37486F0A374C4F09008577DE0FCA3E0FDA3E0FEA3E0FF90085838121C
:206B00000097E4900858357487F0A37486F0A374B1F0900857A18039900858327487F0A3AC
:206B20007487F0A374B4F0900857B9E0FCA3E0FDA3E0FEA3E0FF90085838120097E490085B
:206B400058357487F0A37486F0A374D9F0900857A5E0FCA3E0FDA3E0FEA3E0FF9008583C31
:206B6000120097E4900847D6E0FBA3E0FAA3E0F990084B26E0FEA3E0FFE92FF9EA3EFAC0A3
:206B800003C002C0019008754C7409F0A37457F0A37442F090085832E0F9A3E0FAA3E09077
:206BA00008754FC9F0A3EAF0A3E9F090085838E0FCA3E0FDA3E0FEA3E0FF9008755212005F
:206BC00097E490085835E0F9A3E0FAA3E090087556C9F0A3EAF0A3E9F09008583CE0FCA37C
:206BE000E0FDA3E0FEA3E0FF90087559120097E4D001D002D0031200A69A90084B27E02FE1
:206C0000F090084B26E03EF090085831E004F0700790085830E004F02169F090084E34E099
:206C2000FBA3E0FAA3E0F9120094FBFF12059BE9EF64044E701B90084E34E0FBA3E0FAA3E0
:206C4000E0F9120094FBFF120594D8EF4E7002803490084E34E0FBA3E0FAA3E0F912009441
:206C6000FBFF12059BE9EF64034E702990084E34E0FBA3E0FAA3E0F9120094FBFF12059409
:206C8000D8EF4E7010FE7FBCFD7B097A57797112009C8A80537E007FBC7D007B097A5779DB
:206CA0007112009C8A90084E34E0FBA3E0FAA3E0F9120094FBFF7B097A577971E49008855D
:206CC000E2F012059F0390084E34E0FBA3E0FAA3E0F9120094FBFF7B097A5779719008853F
:206CE000E27402F012059F0390085830E4F0A304F090085830E0FEA3E0FFD39404EE64804B
:206D000094804003216EDAEE6003216E23EF24FE604F147003216D9C147003216DD724032C
:206D20006003216E23900858327487F0A37487F0A374C2F0900857BDE0FCA3E0FDA3E0FE51
:206D4000A3E0FF90085838120097E4900858357487F0A37486F0A374FDF0900857A9216E34
:206D600010900858327487F0A37487F0A374CFF090085781E0FCA3E0FDA3E0FEA3E0FF9033
:206D8000085838120097E4900858357487F0A37487F0A37425F0900857AD80749008583252
:206DA0007487F0A37487F0A374D9F090085785E0FCA3E0FDA3E0FEA3E0FF9008583812006D
:206DC00097E4900858357487F0A37487F0A3744DF0900857B18039900858327487F0A374C9
:206DE00087F0A374E9F090085789E0FCA3E0FDA3E0FEA3E0FF90085838120097E4900858B0
:206E0000357487F0A37487F0A374F6F0900857B5E0FCA3E0FDA3E0FEA3E0FF9008583C1286
:206E20000097E4900847D6E0FBA3E0FAA3E0F990084B26E0FEA3E0FFE92FF9EA3EFAC003EF
:206E4000C002C0019008754C7409F0A37457F0A37442F090085832E0F9A3E0FAA3E09008AF
:206E6000754FC9F0A3EAF0A3E9F090085838E0FCA3E0FDA3E0FEA3E0FF900875521200970D
:206E8000E490085835E0F9A3E0FAA3E090087556C9F0A3EAF0A3E9F09008583CE0FCA3E070
:206EA000FDA3E0FEA3E0FF90087559120097E4D001D002D0031200A69A90084B27E02FF00E
:206EC00090084B26E03EF090085831E004F0700790085830E004F0216CF1900847D6E0FB2D
:206EE000A3E0FAA3E0F990084B26E0FEA3E0FFE92FF9EA3EFA9008754C7487F0A37488F02A
:206F0000A3740BF01200A69A90084B27E02FF090084B26E03EF080037F01227F0022900097
:206F2000FFFD1200991EEBF0A3EAF0A3E9F09000FFD61200991E1205A0A6EF64014E700615
:206F4000FE7F02217DC79000003012009945E0FBA3E0FAA3E0F9120094FBFDACF0C3940F29
:206F6000EC648094805003217DBE9000002D12009945E0FBA3E0FAA3E0F9C003C002C001B7
:206F8000C3ED9401FDEC9400FC9000002A12009945E0F9A3E0FAA3E090087FE4C9F0A3EA6F
:206FA000F0A3E9F09000002A12009945E0FBA3E0FAA3E02434F9E43AFA120094FBC394017E
:206FC000FEE5F0940090087FE7F0A3CEF0D001D002D0031204F42AEF4E6003217DBE7C00D9
:206FE0007D029000003012009945E0FBA3E0FAA3E0F9120094FB25E0FFE5F033FE90000053
:207000002D12009945E0FBA3E0FAA3E02FF9EA3EFAC3E99DF9EA9CFA120094FBFFAEF085A9
:207020005083855182759308EEF0A3EFF0855083855182759308E0FEA3E0FFC39401EE94BB
:20704000004009D3EF94FEEE940F4003217DBE7E007F047D007B099000001E12009945A91A
:2070600082AA8312009C8A9000002A12009945E0FBA3E0FAA3E02437F9E43AFA120094FB97
:20708000FFAEF0E5F06003217DBEEF24FC70032175E314700321795E24026003217DBE90D0
:2070A00000003612009945E0FEA3E0D39404EE648094804003217A307E007F047D007B09E8
:2070C0009000001A12009945A982AA8312009C8A9000003612009945E0FEA3E0FF900000E0
:2070E0003312009945E0FBA3E0FAA3E0F9C003C002C0017B099000001A12009945A982AA60
:2071000083A801AC02AD03D001D002D0031200934C7B099000001A12009945A982AA837D8B
:20712000047C001204F924BEFF06BFFF03217A30855083855182A3A3759308E4F0A3F0855B
:207140005083855182A3A3759308E0FEA3E0FFC39440EE64809480506C7B099000000E12E1
:20716000009945A982AA8312056F88EF4E60409000000E12009945E0FEA3E0FF8550838523
:207180005182759308E0FCA3E0B50723ECB5061F855083855182A3A3759308E0FEA3E0FFA2
:2071A0009000000412009945EEF0A3EFF08016855083855182A3A3759308E475F0011200F3
:2071C00094CF21713F855083855182A3A3759308E0FEA3E0C39440EE648094804003217DB6
:2071E000BE855083855182759308E0FEA3E0FF9000000E12009945EEF0A3EFF07B099000AF
:20720000001A12009945A982AA83C003C002C0017B099000002612009945A982AA839008AC
:207220008580EBF0A3EAF0A3E9F0D001D002D00312052F877E007F047D007B09900000227E
:2072400012009945A982AA8312009C8A855083855182A3A3759308E4F0A3F0C390086E8CEC
:20726000E09401FF90086E8BE09400FE855083855182A3A3759308E0FCA3E0FDC39FEE6481
:2072800080F8EC6480984003217374EDAE047803CEA2E713CE13D8F8FF9000001012009944
:2072A00045E5822FF582E5833EF583759308E0FF855083855182A3A3759308A3E05407FE8D
:2072C0007401A806088002C333D8FCFD5F600321735E855083855182A3A3759308E0FEA3FF
:2072E000E07803CEA2E713CE13D8F8FF9000002612009945E5822FF582E5833EF583759340
:2073000008E05D6059855083855182A3A3759308E0FEA3E07803CEA2E713CE13D8F8FF90E3
:2073200000002212009945E5822FF582E5833EF583C083C082759308E0FF855083855182EC
:20734000A3A3759308A3E05407FE7401A806088002C333D8FC4F759308D082D083F08550BB
:2073600083855182A3A3759308E475F001120094CF21725B855083855182A3A3759308E445
:20738000F0A3F0C390086E8CE09401FF90086E8BE09400FE855083855182A3A3759308E0B8
:2073A000FCA3E0FDC39FEE6480F8EC648098400321749CEDAE047803CEA2E713CE13D8F814
:2073C000FF9000002612009945E5822FF582E5833EF583759308E0FF855083855182A3A3F8
:2073E000759308A3E05407FE7401A806088002C333D8FCFD5F700321748685508385518290
:20740000A3A3759308E0FEA3E07803CEA2E713CE13D8F8FF9000001412009945E5822FF501
:2074200082E5833EF583759308E05D6059855083855182A3A3759308E0FEA3E07803CEA254
:20744000E713CE13D8F8FF9000002212009945E5822FF582E5833EF583C083C08275930820
:20746000E0FF855083855182A3A3759308A3E05407FE7401A806088002C333D8FC4F75937D
:2074800008D082D083F0855083855182A3A3759308E475F001120094CF2173837B0990005F
:2074A000002612009945A982AA83C003C002C0017B099000001012009945A982AA83A80103
:2074C000AC02AD03D001D002D0037E007F041200934C7B099000002212009945A982AA8368
:2074E000C003C002C0017B099000001412009945A982AA83A801AC02AD03D001D002D00359
:207500007E007F041200934C855083855182A3A3759308E4F0A3F0C390086E8CE09401FD45
:2075200090086E8BE09400FC855083855182A3A3759308E0FEA3E0FFC39DEC6480F8EE646A
:2075400080984003217BD77B099000001812009945A982AA83120589389000000E120099C8
:2075600045E0FEA3E0FF9000001812009945E0540FFCA3E06F7002EE6C70528550838551E1
:2075800082A3A3759308E0FEA3E07803CEA2E713CE13D8F8FF9000001012009945E5822FF7
:2075A000F582E5833EF583759308E0FF855083855182A3A3759308A3E05407FE7401A80642
:2075C000088002C333D8FC5F700321793F855083855182A3A3759308E475F001120094CFE7
:2075E0002175179000003612009945E0FEA3E0D39404EE648094804003217A307E007F0467
:207600007D007B099000001A12009945A982AA8312009C8A9000003612009945E0FEA3E028
:20762000FF9000003312009945E0FBA3E0FAA3E0F9C003C002C0017B099000001A120099A5
:2076400045A982AA83A801AC02AD03D001D002D0031200934C7B099000001A12009945A958
:2076600082AA837D047C001204F924BEFF06BFFF03217A30855083855182A3A3759308E4F2
:20768000F0A3F0855083855182A3A3759308E0FEA3E0FFC39440EE64809480506C7B0990B4
:2076A00000000E12009945A982AA8312056F88EF4E60409000000E12009945E0FEA3E0FF9B
:2076C000855083855182759308E0FCA3E0B50723ECB5061F855083855182A3A3759308E000
:2076E000FEA3E0FF9000000412009945EEF0A3EFF08016855083855182A3A3759308E47531
:20770000F001120094CF217683855083855182A3A3759308E0FEA3E0C39440EE6480948005
:207720004003217DBE855083855182759308E0FEA3E0FF9000000E12009945EEF0A3EFF09C
:207740007B099000001A12009945A982AA83C003C002C0017B099000002212009945A9821C
:20776000AA8390088580EBF0A3EAF0A3E9F0D001D002D00312052F87855083855182A3A332
:20778000759308E4F0A3F0C390086E8CE09401FF90086E8BE09400FE855083855182A3A3B0
:2077A000759308E0FCA3E0FDC39FEE6480F8EC6480984003217847EDAE047803CEA2E71322
:2077C000CE13D8F8FF9000002212009945E5822FF582E5833EF583759308E0FF8550838560
:2077E0005182A3A3759308A3E05407FE7401A806088002C333D8FCFD5F60368550838551ED
:2078000082A3A3759308E0FEA3E07803CEA2E713CE13D8F8FF9000001012009945E5822F74
:20782000F582E5833EF583759308E05D700321793F855083855182A3A3759308E475F001CA
:20784000120094CF2177877B099000002212009945A982AA83C003C002C0017B09900000BC
:207860001412009945A982AA83A801AC02AD03D001D002D0037E007F041200934C855083E5
:20788000855182A3A3759308E4F0A3F0C390086E8CE09401FD90086E8BE09400FC855083B3
:2078A000855182A3A3759308E0FEA3E0FFC39DEC6480F8EE648098400321795B7B099000DC
:2078C000001812009945A982AA83120589389000000E12009945E0FEA3E0FF9000001812C8
:2078E000009945E0540FFCA3E06F7002EE6C7055855083855182A3A3759308E0FEA3E07809
:2079000003CEA2E713CE13D8F8FF9000001012009945E5822FF582E5833EF583759308E09F
:20792000FF855083855182A3A3759308A3E05407FE7401A806088002C333D8FC5F7006FE1C
:207940007F03217DC7855083855182A3A3759308E475F001120094CF21788C217BD7900053
:20796000003312009945E0FBA3E0FAA3E0F912009708120098D5799E000000017BF9000054
:2079800000027BF9000000037A33000000047BF9000000057BFC0000000600007BF985507E
:2079A00083855182A3A3759308E4F0A3F0855083855182A3A3759308E0FEA3E0FFC3944032
:2079C000EE64809480504F7B099000000E12009945A982AA8312056F88EF4E603990000044
:2079E0000E12009945E0FEA3E0FF855083855182759308E0FCA3E0B50707ECB50603217DFF
:207A0000C4855083855182A3A3759308E475F001120094CF8097855083855182A3A37593C8
:207A200008E0FEA3E0C39440EE64809480217DB8217DB8855083855182A3A3759308E4F0DA
:207A4000A3F0855083855182A3A3759308E0FEA3E0FFC39440EE64809480506F7B099000DD
:207A6000000E12009945A982AA8312056F88EF4E701F855083855182A3A3759308E0FEA34F
:207A8000E0FF9000000412009945EEF0A3EFF0803A9000000E12009945E0FEA3E0FF8550A6
:207AA00083855182759308E0FCA3E0B50707ECB50603217DB8855083855182A3A3759308B3
:207AC000E475F001120094CF217A42855083855182A3A3759308E0FEA3E0C39440EE64803A
:207AE00094804003217DBE855083855182759308E0FEA3E0FF9000000E12009945EEF0A3A4
:207B0000EFF0855083855182A3A3759308E4F0A3F0C390086E8CE09401FF90086E8BE0944B
:207B200000FE855083855182A3A3759308E0FCA3E0FDC39FEE6480F8EC6480985063EDAE03
:207B4000047803CEA2E713CE13D8F8FF9000001012009945E5822FF582E5833EF583C0838E
:207B6000C082759308E0FF855083855182A3A3759308A3E05407FE7401A806088002C3334F
:207B8000D8FC4F759308D082D083F0855083855182A3A3759308E475F001120094CF217BBC
:207BA000117B099000001012009945A982AA83C003C002C0017B099000001412009945A941
:207BC00082AA83A801AC02AD03D001D002D0037E007F041200934C9000000412009945E023
:207BE000FEA3E0FF7B099000000E12009945A982AA831205A229217DB2217DB87E007F080E
:207C00007D007B099000000612009945A982AA8312009C8A855083855182A3A3759308E463
:207C2000F0A3F0855083855182A3A3759308E0FEA3E0FFC39440EE64809480506C7B09900E
:207C400000000E12009945A982AA8312056F88EF4E60409000000E12009945E0FEA3E0FFF5
:207C6000855083855182759308E0FCA3E0B50723ECB5061F855083855182A3A3759308E05A
:207C8000FEA3E0FF9000000412009945EEF0A3EFF08016855083855182A3A3759308E4758B
:207CA000F001120094CF217C23855083855182A3A3759308E0FEA3E0C39440EE64809480BA
:207CC0004003217DC4855083855182A3A3759308E4F0A3F0C390086E8CE09401FD90086EC5
:207CE0008BE09400FC855083855182A3A3759308E0FEA3E0FFC39DEC6480F8EE6480985041
:207D00004C7B099000001812009945A982AA83120589389000000E12009945E0FEA3E0FFDD
:207D20009000001812009945E0540FFCA3E0B50707EEB50403217DB8855083855182A3A330
:207D4000759308E475F001120094CF80879000000412009945E0FEA3E07803CEA2E713CEB5
:207D600013D8F8FF9000000612009945E5822FF582E5833EF583C083C082759308E0FF906C
:207D800000000412009945A3E05407FE7401A806088002C333D8FC4F759308D082D083F0A8
:207DA0007B099000000612009945A982AA8312049694120588FB800C7E007F0380097E00F4
:207DC0007F028003E4FEFF900000380200991E9000FFFD1200991EEBF0A3EAF0A3E9F09084
:207DE00000FEAC1200991E9000015412009945E0FBA3E0FAA3E0F9C003C002C001855083C9
:207E0000855182759308A982AA83900883EB7409F0A3EAF0A3E9F09000015412009945E081
:207E2000FBA3E0FAA3E02434F9E43AFA120094FB25E0FEE5F033900883EEF0A3CEF0D00107
:207E4000D002D003120576279000015412009945E0FBA3E0FAA3E02434F9E43AFA1200940A
:207E6000FB25E0FFE5F033FE9000015412009945E0FBA3E0FAA3E02FF9EA3EFA120094FB62
:207E8000FFAEF09000008212009945EEF0A3EFF09000008012009945E4F0A304F0900000E8
:207EA0008212009945E0FEA3E0FF9000008012009945E0FCA3E0FDD39FEE6480F8EC648088
:207EC00098400321800C9000015412009945E0FBA3E0FAA3E02434F9E43AFA120094FBC39D
:207EE0009401FFE5F09400FEEF25E0FFEE33FE759308E5512FF582E5503EF583759308ECA2
:207F0000F0A3EDF09000008212009945E0FEA3E0B5052FECB5062B120094FBC39401FFE5F6
:207F2000F09400FEEF25E0FFEE33FE759308E5512FF582E5503EF5837593087402F0A37449
:207F40005CF09000015712009945E0FBA3E0FAA3E0F9C003C002C0019000015A1200994508
:207F6000E0FBA3E0FAA3E0F9120094FBFDACF0855083855182759308A982AA8390087FE4E0
:207F80007409F0A3EAF0A3E9F09000015412009945E0FBA3E0FAA3E02434F9E43AFA120050
:207FA00094FBFF90087FE7E5F0F0A3EFF0D001D002D0031204F42A9000008412009945EE52
:207FC000F0A3EFF09000015D12009945E0FEA3E0FF4E600F9000008412009945E0FCA3E0D1
:207FE0004C6029EF4E70129000008412009945E0FEC3EE6480948040139000008012009954
:2080000045E475F001120094CF217E9D9000008212009945E0FEA3E0FF9000008012009903
:2080200045E0FCA3E0D39FEE6480F8EC6480984003218B787B09855083855182759308A9A4
:2080400082AA83C003C002C0019000015712009945E0F9A3E0FAA3E0900883EBC9F0A3EA2E
:20806000F0A3E9F09000015412009945E0FBA3E0FAA3E02434F9E43AFA120094FB25E0FED7
:20808000E5F033900883EEF0A3CEF0D001D002D003120576279000015412009945E0FBA301
:2080A000E0FAA3E02434F9E43AFA120094FBFFAEF09000015A12009945E0FBA3E0FAA3E006
:2080C000F9EE8FF0120095759000016212009945E0FBA3E0FAA3E0F9E4F5F01200957590F2
:2080E00000015412009945E0FBA3E0FAA3E02437F9E43AFA120094FBFFAEF0E5F06003215D
:2081000084F9EF24FBB4100040032184F99001811C75F004A4C58325F0C583730201815CFC
:20812000020184F9020181C20201815C020184F90201820D02018233020182330201829BF7
:2081400002018305020184F9020183B70201842102018421020184F90201848990000082E5
:2081600012009945E0FEA3E0FF9000008012009945E0FCA3E0B50727ECB506239000008093
:2081800012009945A3E0C39401FF7B099000008612009945A982AA831205907A2184F990E4
:2081A00000008012009945A3E0C39401FF7B099000008612009945A982AA831205A21921A0
:2081C00084F99000008212009945E0FEA3E0FF9000008012009945E0FCA3E0C39FEE64802D
:2081E000F8EC64809840032184F99000008012009945A3E0C39401FF7B09900001461200F7
:208200009945A982AA831204B2D92184F99000008212009945E0FEA3E0FF90000080120065
:208220009945E0FCA3E0B50707ECB506032183D72183FC9000008212009945E0FEA3E0FF17
:208240009000008012009945E0FCA3E0B50728ECB506249000008012009945A3E0C3940135
:20826000FF7B099000008A12009945A982AA83E49008863C2184CB9000008012009945A3C8
:20828000E0C39401FF7B099000008A12009945A982AA83E4900885E22184F4900000821221
:2082A000009945E0FEA3E0FF9000008012009945E0FCA3E0B50729ECB5062590000080124E
:2082C000009945A3E0C39401FF7B099000008A12009945A982AA839008863C74042184CBBE
:2082E0009000008012009945A3E0C39401FF7B099000008A12009945A982AA83900885E2BF
:2083000074042184F49000008212009945E0FEA3E0FF9000008012009945E0FCA3E06F70AC
:2083200002EC6E90000080704712009945A3E0C39401FF7B099000008A12009945A982AAED
:2083400083E49008863CF012059C6B9000008012009945A3E0C39401FF7B099000008A12C4
:20836000009945A982AA839008863C74022184CB12009945A3E0C39401FF7B099000008A1F
:2083800012009945A982AA83E4900885E2F012059F039000008012009945A3E0C39401FF2F
:2083A0007B099000008A12009945A982AA83900885E274022184F49000008212009945E0E7
:2083C000FEA3E0FF9000008012009945E0FCA3E0B50729ECB506259000008012009945A36A
:2083E000E0C39401FF7B099000008A12009945A982AA839008863C74052184CB900000800D
:2084000012009945A3E0C39401FF7B099000008A12009945A982AA83900885E2740521848F
:20842000F49000008212009945E0FEA3E0FF9000008012009945E0FCA3E0B50728ECB506FC
:20844000249000008012009945A3E0C39401FF7B099000008A12009945A982AA839008861A
:208460003C740180669000008012009945A3E0C39401FF7B099000008A12009945A982AA28
:2084800083900885E27401806B9000008212009945E0FEA3E0FF9000008012009945E0FCBC
:2084A000A3E0B5072DECB506299000008012009945A3E0C39401FF7B099000008A1200995D
:2084C00045A982AA839008863C7406F012059C6B80279000008012009945A3E0C39401FF9C
:2084E0007B099000008A12009945A982AA83900885E27406F012059F0390000154120099E4
:2085000045E0FBA3E0FAA3E02437F9E43AFA120094FBFFAEF0E5F06003218B78EF24FCB472
:2085200012004003218B789001853675F004A4C58325F0C583730201857E020185EF0201D1
:208540008659020186E50201875202018B78020187A4020187E40201882402018881020192
:20856000895202018AE302018A0602018A4602018A8602018AE302018B1402018AE3900025
:20858000015F12009945E0FBA3E0FAA3E0F9E475F004120095759000008212009945E0FE6E
:2085A000A3E0FF9000008012009945E0FCA3E0B5071AECB50616E47FDC7E05FDFC900001FB
:2085C0004A12009945120097E42187499000008012009945A3E0C39401FF7B099000014AAA
:2085E00012009945A982AA83120584DA2187499000015F12009945E0FBA3E0FAA3E0F9E435
:2086000075F004120095759000008612009945E0C4F854F0C8A3E0C4540F48540F60191445
:20862000600C14600924FE600304701680147F007EE17DF57C0580127F007ECA7D9A7C3BB6
:2086400080087F807E967D987C009000014A12009945120097E421874990000082120099E8
:2086600045E0FEA3E0FF9000008012009945E0FCA3E0B50730ECB5062C9000015F1200999C
:2086800045E0FBA3E0FAA3E0F9E475F006120095757B099000014E12009945A982AA831299
:2086A0000591B380379000015F12009945E0FBA3E0FAA3E0F9E4F5F0120095759000008011
:2086C00012009945A3E0C39401FF7B099000014E12009945A982AA831205A2027B09900056
:2086E000014E218B6E9000015F12009945E0FBA3E0FAA3E0F9E475F0041200957590000064
:208700008212009945E0FEA3E0FF9000008012009945E0FCA3E0B50709ECB50605E47F0153
:2087200080189000014612009945A3E0540F64066005E47F018003E47F02FEFDFC90000151
:208740004A12009945120097E47B099000014A218B6E9000015F12009945E0FBA3E0FAA3FE
:20876000E0F9E475F004120095759000008612009945E0C4F854F0C8A3E0C4540F48540FB4
:2087800064076005E47F018003E47F02FEFDFC9000014A12009945120097E47B0990000159
:2087A0004A218B6E9000015F12009945E0FBA3E0FAA3E0F9E475F004120095759000012A7D
:2087C00012009945E0FCA3E0FDA3E0FEA3E0FF9000014A12009945120097E47B09900001DD
:2087E0004A218B6E9000015F12009945E0FBA3E0FAA3E0F9E475F004120095759000008ADE
:2088000012009945E0FCA3E0FDA3E0FEA3E0FF9000014A12009945120097E47B099000019C
:208820004A218B6E9000015F12009945E0FBA3E0FAA3E0F9E475F004120095759000009295
:2088400012009945E0FCA3E0FDA3E0FEA3E0FF9000008E12009945E0F8A3E0F9A3E0FAA347
:20886000E02FFFEA3EFEE93DFDE83CFC9000014A12009945120097E47B099000014A218B1E
:208880006E9000015F12009945E0FBA3E0FAA3E0F9E475F004120095759000010E12009903
:2088A00045E0FCA3E0FDA3E0FEA3E0FF9000010A12009945E0F8A3E0F9A3E0FAA3E02FFF07
:2088C000EA3EFEE93DFDE83CFC9000011212009945E0F8A3E0F9A3E0FAA3E02FFFEA3EFEF4
:2088E000E93DFDE83CFC9000011612009945E0F8A3E0F9A3E0FAA3E02FFFEA3EFEE93DFDD3
:20890000E83CFC9000011A12009945E0F8A3E0F9A3E0FAA3E02FFFEA3EFEE93DFDE83CFCB1
:208920009000011E12009945E0F8A3E0F9A3E0FAA3E02FFFEA3EFEE93DFDE83CFC9000011C
:208940004A12009945120097E47B099000014A218B6E9000015F12009945E0FBA3E0FAA3FC
:20896000E0F9E475F004120095759000009E12009945E0FCA3E0FDA3E0FEA3E0FF900000A8
:208980009A12009945E0F8A3E0F9A3E0FAA3E02FFFEA3EFEE93DFDE83CFC900000A212001E
:2089A0009945E0F8A3E0F9A3E0FAA3E02FFFEA3EFEE93DFDE83CFC900000DA12009945E0B4
:2089C000F8A3E0F9A3E0FAA3E02FFFEA3EFEE93DFDE83CFC900000DE12009945E0F8A3E0D3
:2089E000F9A3E0FAA3E02FFFEA3EFEE93DFDE83CFC9000014A12009945120097E47B09907B
:208A000000014A218B6E9000015F12009945E0FBA3E0FAA3E0F9E475F00412009575900044
:208A2000012212009945E0FCA3E0FDA3E0FEA3E0FF9000014A12009945120097E47B099058
:208A400000014A218B6E9000015F12009945E0FBA3E0FAA3E0F9E475F00412009575900004
:208A600000A612009945E0FCA3E0FDA3E0FEA3E0FF9000014A12009945120097E47B099095
:208A800000014A218B6E9000015F12009945E0FBA3E0FAA3E0F9E475F004120095759000C4
:208AA00000AA12009945E0FCA3E0FDA3E0FEA3E0FF900000AE12009945E0F8A3E0F9A3E0B8
:208AC000FAA3E02FFFEA3EFEE93DFDE83CFC9000014A12009945120097E47B099000014ACB
:208AE000218B6E9000015F12009945E0FBA3E0FAA3E0F9E475F00412009575E4FFFEFDFC65
:208B00009000014A12009945120097E47B099000014A805A9000015F12009945E0FBA3E086
:208B2000FAA3E0F9E475F004120095759000014212009945E0FCA3E0FDA3E0FEA3E0FF90A4
:208B400000013E12009945E0F8A3E0F9A3E0FAA3E02FFFEA3EFEE93DFDE83CFC9000014A20
:208B600012009945120097E47B099000014A12009945A982AA8380067B007A00790090004D
:208B800001650200991E9000FFFD1200991EEBF0A3EAF0A3E9F09000FFEA1200991E9000BB
:208BA000002212009945E0FEA3E0FF9000002212009945EEF0A3EFF09000001C12009945A5
:208BC000E0FBA3E0FAA3E0F9120094FBFDACF0C3940FEC64809480500321963E900000194C
:208BE00012009945E0FBA3E0FAA3E0F9C003C002C001C3ED9401FDEC9400FC9000001612F5
:208C0000009945E0F9A3E0FAA3E090087FE4C9F0A3EAF0A3E9F09000001612009945E0FB7F
:208C2000A3E0FAA3E02434F9E43AFA120094FBC39401FEE5F0940090087FE7F0A3CEF0D04C
:208C400001D002D0031204F42AEF4E600321963E7C007D029000001C12009945E0FBA3E0B0
:208C6000FAA3E0F9120094FB25E0FFE5F033FE9000001912009945E0FBA3E0FAA3E02FF937
:208C8000EA3EFAC3E99DF9EA9CFA120094FBFFAEF0855083855182759308EEF0A3EFF0850D
:208CA0005083855182759308E0FEA3E0FFC39401EE64809480400BD3EF9401EE6480948053
:208CC000400321963E85508385518275930874FFF5F0120094CF9000001612009945E0FB5E
:208CE000A3E0FAA3E02437F9E43AFA120094FBFFAEF0E5F0600321963EEF24FD7003218F6A
:208D00001B14700321908F1470032192712403600321963E9000001F12009945E0FBA3E04A
:208D2000FAA3E0F912009708E4FBFAF9F8C3120096D19000001F705512009945E0FBA3E044
:208D4000FAA3E0F912009708855083855182759308E0FCA3E0FD9008812375F0071200987E
:208D600001EC75F007A42583F583759308EFF09008812975F007ED12009801EC75F007A4A5
:208D80002583F583759308E054FEF0805312009945E0FBA3E0FAA3E0F912009708855083E1
:208DA000855182759308E0FCA3E0FD9008812375F00712009801EC75F007A42583F583750B
:208DC0009308EFF09008812975F007ED12009801EC75F007A42583F583759308E04401F092
:208DE000855083855182759308E0FEA3E09008812775F00712009801EE75F007A42583F560
:208E000083759308E0FEA3E064014E60032196449000001F12009945E0FBA3E0FAA3E0F9DA
:208E200012009708E4FBFAF9F8C3120096D1707A855083855182759308E0FEA3E0FF9008D9
:208E4000812575F00712009801EE75F007A42583F583759308E4F09008812675F007EF12A7
:208E6000009801EE75F007A42583F583759308E4F09008812975F007EF12009801EE75F0BC
:208E800007A42583F583759308E4F09008812775F007EF12009801EE75F007A42583F583BF
:208EA000759308E4F0A3F0219203855083855182759308E0FEA3E0FF9008812675F00712A8
:208EC000009801EE75F007A42583F583759308E0FD9008812575F007EF12009801EE75F057
:208EE00007A42583F583759308E0B50503219638855083855182759308E0FEA3E0900881D1
:208F00002975F00712009801EE75F007A42583F583759308E04401F02192038550838551EA
:208F200082759308E0FEA3E0FF9008812575F00712009801EE75F007A42583F583759308BC
:208F4000E4F09008812975F007EF12009801EE75F007A42583F583759308E054FDF0900016
:208F6000001F12009945E0FBA3E0FAA3E0F912009708E47B01FAF9F8D3120096D15031C382
:208F800090086E7CE09401FF90086E7BE09400FE3395E0FDFC9000001F12009945E0FBA32A
:208FA000E0FAA3E0F91200975DD3120096D140032196389000001F12009945E0FBA3E0FAE0
:208FC000A3E0F912009708C3EF9401FBEE9400FAED9400F9EC9400F88550838551827593FC
:208FE00008E0FEA3E09008812675F00712009801EE75F007A42583F583759308E0FFE4FCC5
:20900000FDFEC3120096D1700321917D9000001F12009945E0FBA3E0FAA3E0F91200970853
:20902000C3EF9401FF855083855182759308E0FCA3E0FD9008812575F00712009801EC7518
:20904000F007A42583F583759308EFF09008812975F007ED12009801EC75F007A42583F587
:2090600083759308E04402F09008812775F007ED12009801EC75F007A42583F583759308D7
:20908000E0FEA3E064014E6003219644219203855083855182759308E0FEA3E0FF9008816F
:2090A0002675F00712009801EE75F007A42583F583759308E4F09008812975F007EF1200C2
:2090C0009801EE75F007A42583F583759308E054FBF09000001F12009945E0FBA3E0FAA310
:2090E000E0F912009708E47B01FAF9F8D3120096D15031C390086E7CE09401FF90086E7B94
:20910000E09400FE3395E0FDFC9000001F12009945E0FBA3E0FAA3E0F91200975DD31200DE
:2091200096D140032196389000001F12009945E0FBA3E0FAA3E0F912009708C3EF9401FB30
:20914000EE9400FAED9400F9EC9400F8855083855182759308E0FEA3E09008812575F007D6
:2091600012009801EE75F007A42583F583759308E0FFE4FCFDFEC3120096D17006FE7F032A
:209180002196479000001F12009945E0FBA3E0FAA3E0F912009708C3EF9401FF855083858A
:2091A0005182759308E0FCA3E0FD9008812675F00712009801EC75F007A42583F5837593F6
:2091C00008EFF09008812975F007ED12009801EC75F007A42583F583759308E04404F0908E
:2091E00008812775F007ED12009801EC75F007A42583F583759308E0FEA3E064014E600318
:20920000219644855083855182759308E0FEA3E0FF9008812575F00712009801EE75F00784
:20922000A42583F583759308E0FD9008812675F007EF12009801EE75F007A42583F58375A5
:209240009308E0FB9008812375F007EF12009801EE75F007A42583F583759308E09008862A
:2092600083F0855083855182759308A3E0FF21962E9000001F12009945E0FBA3E0FAA3E0DA
:20928000F9120097089000000412009945120097E49000000412009945E0FCA3E0FDA3E0B0
:2092A000FEA3E0FF120098D592CA00000001935A0000000293D60000000493D90000000585
